:100000000C940F2A0C94852A0C94852A0C94852A2A
:100010000C94852A0C94852A0C94852A0C94852AA4
:100020000C94852A0C94852A0C94852A0C94852A94
:100030000C94852A0C94292D0C94682D0C94062B75
:100040000C94852A0C94852A0C94852A0C94852A74
:100050000C94852A0C94852A0C94852A0C94852A64
:100060000C94852A0C94852A0C94852A0C94852A54
:10007000CE442C433243354338433B433E43414314
:100080004443CB442F43A045BB45E545F5450A46CF
:100090002246554674465A55012001010038080091
:1000A0000000000000000000000000000000000050
:1000B000000000000000810045005DFF5E1027FF8A
:1000C0002AD22B7D210C22FB850084008903888D98
:1000D00081096F02444247004501B083B300B1017A
:1000E00024B925578A1D8B03FB35FE351A3A35375F
:1000F0002C3707360C3611361A37143617361A369F
:100100005B365E36613600408891D2E4ADB5B6BE4E
:10011000BFFF1409000000000001000203040500F5
:100120000000000000000000000000060708090AA7
:100130000B0C0D0E0F101100000000000000121338
:100140001415161718191A1B1C1D1E1F202100003C
:100150000022232425262728292A2B2C2D00002E97
:100160002F300000313233333435363738393A3BAB
:100170003C3D3E3F404142434445464748494A4B47
:100180004C4D4E4F505152535455565758595A5B37
:100190005C5D5E5F606162636465666768696A6B27
:1001A0000000000000000000006C6D6E6F70717246
:1001B000737475760000000000000000000000006D
:1001C000007778797A7B7C0004047E8081828F902E
:1001D0008787968787879D87879E04048384857E8B
:1001E00087879192878787979F8787A00404868750
:1001F000878893878787989987877EA2A3A404041A
:100200008987878A8787879487879A9BA5A6A77EF1
:1002100004048B87878C8B87878C8B87878C8B8755
:10022000878C04048D8D8D8D878787878787878747
:10023000A8A8A8A80000000000000000000000001E
:1002400000000000000000000000000000000000AE
:10025000000000000000000000000000000000009E
:10026000000000000000000000000000000000008E
:10027000000000000000000000000000000000007E
:10028000000000000000000000000000000000006E
:10029000000000000000000000000000000000005E
:1002A000000000000000000000000000000101004C
:1002B000000000000000000000000000000000003E
:1002C000000000000000000000000000000000002E
:1002D000000000000000000000000000000000001E
:1002E000000009640000000000005B6400000000E2
:1002F000005B64BF00000000000000000000000080
:100300000000095B000000095B64646400095B6431
:100310006464B6BF5B64646DBFBFBFBF6464BFBFCE
:10032000BFBFBFBFBFBFBFBFBFBFBFBFBFBFBFBFDD
:10033000BFBFB6B6000000095B5B00005B5BB6BFE9
:10034000BF645B00B6BFBFBFBFBF645BBFBFBFBF03
:10035000BFBFB65BBFBFBFBF645BBFB6BFBFB66446
:100360005BB6BFBFB6645B5B64BFBFBF5B5B0900CE
:100370000064BFBF0000000000000000000000009B
:1003800000000000090000000000000064090000F7
:10039000000000005B6400000000000064645B007B
:1003A00000000000BF64640000000000BFBF5B09E4
:1003B000000000000000000000000000000000003D
:1003C000000000000000000000000000000000002D
:1003D0000000010200000000020304050000000309
:1003E00004030202000000000203040500000204EE
:1003F00005050505000000000000000000000000E9
:1004000000000002000000000000010400000000E5
:1004100000020305020000000102050502020201BC
:10042000010205040505050504040202050505058C
:10043000050505040304040302010000030303038C
:100440000303020104040403030202020404050579
:10045000050404030303020305060505030304045E
:100460000302050503020001020303020202020067
:100470000000020300000000000000000000000077
:100480000000000001000000000000000200000069
:1004900000000000040302000000005B05050403E7
:1004A00000095BB604050505095BB6BF0204050437
:1004B0005BB6BFBF000000005BB6BFBF00000964B1
:1004C000BFBFBFBF000964BFBFBFBFBF5B6DBFBFC2
:1004D000BFBFBFBFB6BFBFBFBFBFBF64BFBFBFBF90
:1004E000BFBF6464BFBFBFBFBF645B09BFBFBFBF47
:1004F00064090000BFBFBFBFBFB6645BBFBFBFB66C
:10050000645B0900BFB664645B0000006464640956
:1005100000000000645B0900000000005B000000B8
:1005200000000000000000000000000000000000CB
:10053000000009B609000000000964BF00000000C7
:10054000000009BF0000000000095B64000000001B
:100550005B64646400000964BFBFBF64005BBFBF2D
:10056000BFBFBFBF64BFBFBFBFBFBFBF64BFBFBF51
:10057000BFBFBFBFBFBF645B09000000BFBFB65BAA
:100580005B5B0900BFBFBFB66464645B6DBFBFBF88
:10059000BFB6BFBFB6BFBFBFBFBF6D64BFBFBFBF2A
:1005A000645B0952BFBF645B09000052BF5B5B091B
:1005B000000000000000000000000000000000003B
:1005C000000000005B5B090000000000BF645B00EE
:1005D00000005B645B5B09095B64B664525264B6FD
:1005E000BF645B64525BBF64095BB6BF52645B5B14
:1005F000B6BFBFBF000000000000000900000000FF
:10060000005B5B5B00095B6464BFB6646464BFBF8E
:10061000BFBFBFB664BFBFBFBFBFBFBFBFBFBFBF4E
:10062000BFBFBFBFBFBFBFBFBFBFBFBFBFBFBFBFDA
:10063000BFBFBFBF00000000000000006464645B37
:100640005B5B09006464B6B664646464B6B6B664A1
:1006500065646464BFBFBFBFBFBFBFB6BFBFBFBF1E
:10066000BFBFBFBFBFBFBFBFBFBFBFBFBFBFBFBF9A
:10067000BFBFBF64000000000000000000000000D9
:10068000000000005B090000000000006464645B7F
:1006900000000000B664B66400000000BFB65B094D
:1006A00000000000645B09000052520064640052C4
:1006B0005200005200000000000000000000000096
:1006C000000000000000000000000000000000002A
:1006D0000000005200000000000052520000000024
:1006E00000525252000000005252525200000000CC
:1006F0005252520000000204050505050052510245
:1007000003040505525252010204040452525200DD
:10071000000203045200000000000000000000007E
:1007200000000000000000000000000000000000C9
:10073000000000000505050505050505050505057D
:100740000505050504050505050505050403030460
:100750000505050500000001020405050000000074
:1007600002020204000000000000535200000000DA
:100770000000ADA405040203010000000505050505
:10078000040200000505050505050301050505052D
:10079000050505040505050505050505050505050A
:1007A00005050505030505050505050502040505FF
:1007B000040403020203035C64BFBFBF00000964BA
:1007C000BFBFBFBF00005BB6BFBFBFBF0303646452
:1007D000BFBFBFBF0505B75BBFBFBFBF0505665B3A
:1007E000BFBFBFBF05055E5BBFBFBFBF0303015BEC
:1007F000BFBFBFBFBFBFBF6400000000BFBF64007A
:1008000000000000BF6D5B0000000000BF5B64647F
:1008100000000000BFB65BBF09000000BFBF5BBFA8
:100820005B00005BBFBF656464005B1EBFBFBF5B56
:10083000645B1E3700000000005BBFBF00000000CB
:100840005BBF1E1E000000641E1E373700091E1EFF
:1008500037373737641E3737373737371E3737372D
:100860003737373737373737373737373737373718
:10087000373737376464BFBFBFBFBF641E1EBFBFFB
:10088000BF5B090037371EBF640000003737371ED3
:1008900000000000373737371E1E00003737373764
:1008A00037371E00373737373737371E3737373741
:1008B0003737371E5B5B00000000000000000000BF
:1008C000000000090000000000005BB6000000000E
:1008D000005BBFBF0000000064BFBFBF000000643A
:1008E000BFBFBFBF000964BFBFBFBFBF0964BFBFF9
:1008F000BFBFBFBF005BB6BFBFBFBFBF64BFBFBF8F
:10090000BFBFBFBFBFBFBFBFBFBFBFBFBFBFBFBFF7
:10091000BFBFBFBFBFBFBFBFBFBFBFBFBFBFBFBFE7
:10092000BFBFBFBFBFBFBFBFBFBFBFBFBFBFBFBFD7
:10093000BFBFBFBFBFBFBFBFBFBFBFBFBFBFBFBFC7
:10094000BFBFBFBFBFBFBFBFBFBFBFBFBFBFBFBFB7
:10095000BFBFBFBFBFBFBFBFBFBFBFBFBFBFBFBFA7
:10096000BFBFBFBFBFBFBFBFBFBFBF64BFBFBFBFF2
:10097000BFBF645BBFBFBFBFBFB6646DBFBFBFBFFC
:100980006409645BBFBFBF6409000000BFB6646454
:1009900000000000BF64640900000000645B0900FF
:1009A000000000005B0900000000000009000000DA
:1009B000000000005B0000005252520000000000E6
:1009C0000000525200000000000000520000000031
:1009D0000000000000000000000000000000000017
:1009E0000000000000000000000000000000000007
:1009F000000000005200000000000000525252525D
:100A00000000000052525252520000005252525204
:100A100052520000005252525252520000005252A2
:100A200052525252000000525252525200000000E4
:100A300000525252000000000000000000000000C0
:100A400000000000000000000000000000000000A6
:100A500000000000000000000000096452000000D7
:100A6000000964BF525200000964BFBF525200091E
:100A70005BB6B6BF000000000000000000000000F0
:100A80000000000000000000000000000000000066
:100A9000000000005B5B090000000000BF64090962
:100AA00000000000BFBF5B5B00000000BF64646427
:100AB0000000000000000000000000000000000036
:100AC00000000000000000000000000000000052D4
:100AD0000000000100525252000000025252000079
:100AE0000001040452000000020405050000000398
:100AF0000505050500000052525200000000525248
:100B00005200000000015301000000000302040431
:100B1000030100000304050505040302040505059F
:100B20000505050505050505050505050505050575
:100B300005050505000000000000000000000000A1
:100B400000000000000000000000000000000000A5
:100B50000000000001000000000000000404020189
:100B60000000000005050505040302010505050553
:100B700005050504000000000052ADA400000000BF
:100B800000A4AD5B0000000052ADAD5200000000BB
:100B90005BADA45300000000ADAD5B02000000524D
:100BA000ADAD53040100005BADA402050303025385
:100BB000AD5B030502050503025201000305045263
:100BC0005BA452000305045BAD5B00000405035BFE
:100BD000AD5B00000505035BAD520000050502A4F6
:100BE000A4010001050503035302030405050504E0
:100BF000050505050000005BB6BFBFBF000000B6DD
:100C000064BFBFBF000000BF64BFBFBF0000005B88
:100C100064BF00000101000064BF00000404030081
:100C20005BBF0000050505035B0000000505050529
:100C30005B000000BFBFBF5B5B1E3737BFBFBF6538
:100C40001E373737BFBFBF1E3737373700001E3755
:100C50003737373700001E373737373700001E3732
:100C6000373737370000001E37373737000000FFAF
:100C70001E37371E373737373737371E373737374F
:100C800037371E0037373737371E5BA43737371EE5
:100C90001E00001E37371E000000001E371E000019
:100CA0000000001E1EFF000000001E37FF000000B5
:100CB00000001E371E3737373737371E1E37373796
:100CC0003737371E1E3737373737371E37373737FF
:100CD0003737371E373737373737371E37373737D6
:100CE0003737371E3737373737371EB63737373747
:100CF00037371E6464BFBFBFBFBFBFBFBFBFBFBF6B
:100D0000BFBFBFBFBFB6B6B6B6B6B6B664655B5BAF
:100D10005B09095B5B640000000000000900000043
:100D2000000000005B000000000000005B0000000D
:100D300000000000BFBFBFBFBFBFBFBFBFBFBFBFBF
:100D4000BFBFBFBFBFBFBFBFBFBFBFBF5B5B646431
:100D50006464B6BF005252525B5B09640052525B3E
:100D6000A4A4525B0000000000525B52000000008F
:100D700000005B52BFBFBFBFBF645B09BFBFBFB650
:100D80005B5B5B00BFBFB65B5BADA400B6645B5B47
:100D9000A4A45200BF5B5BADADA40000BF645BAD1B
:100DA000ADAD0000B6BF5B5BADAD5B00ADBFB65B8C
:100DB000A4ADAD520000000000005252000000003F
:100DC00000000052000000000000000000000000D1
:100DD000000000000000000000000009000000000A
:100DE000000009090000000000005B640000000032
:100DF000095B64B65252005B5B655BBF52525B6439
:100E00005B5B64B6005BB6BF646464640064646486
:100E1000B6B6095B095B64B6BFBF646464B6BFBFA6
:100E2000B6BFB65BBFBFB66464BFBFB6B6645B6D2A
:100E3000BFBFBFBFB65BBF090000000064B65B0068
:100E40000000000064640000000000005B0000007F
:100E50000000000009000000000000005B5B0900CA
:100E6000000000005B5B645B09000000BF645B6422
:100E7000645B0000000000000000000100000000B2
:100E8000000000010000000000020002000000015C
:100E900004025CA60000010453ADFFFF00000454EF
:100EA000ADFFFFFF000304ADFFADA4AD000503AD32
:100EB000AD5BADAD000103050505050502040505A3
:100EC0000505050505050505050505055605050581
:100ED00005050505FFFF5E0505050505FFFFFFAFDD
:100EE00005050505FFFFFFFF55050505ADADADFF88
:100EF000FF050505050505050505050505050505A8
:100F00000505050505050505050505050505050591
:100F10000505050505050505050505050505050581
:100F20000505050505050505050505050505050571
:100F30000505050505050403530205050505050519
:100F40000404050505050505050504530505050506
:100F5000050453FF050505050501A4FF0505050565
:100F600002ADADAD050505045BAD5BAD05050553F3
:100F7000AD5B5BA405050505050505050302030436
:100F8000050505055B52020103050505AD52AD528D
:100F9000020505055BADFFAD5C020503A4ADFFAD29
:100FA000A5020203AD5BAD5BA4000102ADAD5B52D7
:100FB00052005200050505055B000000050505050A
:100FC0005B000000050505045BFFFFFF0505050448
:100FD00064FFFFFF0405050164FFFFFF0504010036
:100FE000FFFFFFFF0200005BFFFFFFFF0000005B51
:100FF000FFFFFFFF000000FF1E371EFF000000FF85
:10100000FF1EFFFFFFFFFF0000000000FFFFFF00CB
:1010100000000000FFFFFF0000000000FFFF0000D5
:1010200000000000FFFF000000000000FFFF0000C4
:1010300000000000FF000000001E3737FF00000026
:101040001E37373700FFFFFF1E37373700FFFF1E01
:101050003737373700FFFF1E37373737FFFF1E3769
:1010600037373737FF1E373737373737FF1E3737B2
:10107000373737373737373737371E5B37373737F5
:10108000371EBF0937373737371EB65B3737373725
:101090001EBF6464373737371EBF5B643737371E70
:1010A00064BF5BBF3737371E5BBF5BBF37371E0080
:1010B0005BBF5BB6B600000000000000BF00000090
:1010C00000000000B6000000000000006400000006
:1010D000000000005B0000000000000009000000AC
:1010E0000000000000000000000000000000000000
:1010F00000000000000000000000005B0000000095
:101100000000005B000000000000005B0000000029
:10111000000000520000000000000052000000002B
:1011200000000000000000000000000000000000BF
:101130000000005B5BB6BF6452ADAD5B52B6BFBF93
:101140005B5BADAD5B5BBFBFB652ADADA45BBFBF7C
:10115000BF525BADA45B64BFBFB652A4AD525BBFD0
:10116000BFBFB6525B5B5BBFBFBFBF645B64BFBF4B
:10117000BFBFBFBF00000000000000005200000021
:1011800000000000A452000000000000AD5B000061
:1011900000000000ADAD000000000000ADAD5B0040
:1011A0000000000052ADAD52000000005BA4ADADE8
:1011B0000000000900000000000000000000000026
:1011C000000000000000000000000000000000001F
:1011D00000005BBF000000000064BFBF0000005BB8
:1011E000BFBFBFBF005BB6BFBFBFBFBF64BFBFBF96
:1011F000B664B6BF00000964BFBFBF640064BFBF70
:10120000BFBF645B5B5B645B095B64BFBFBFBFBFA9
:10121000BFBFBFBFBFBFBFBFBFBFBFBFBFBFBFBFDE
:10122000BFBFBFBFBFBFBFBFBFBFBFBFBFBFBFBFCE
:10123000BFBFBFBF5B64BFBFBFBFBFBFB6BFBFBF86
:10124000BFBFBFBFBFBFBFBFBFBFBFBFBFBFBFBFAE
:10125000BFBFBFBFBFBFBFBFBFBFBFBFBFBFBFBF9E
:10126000BFBFBFBFBFBFBFBFBFBFBFBFBFBFBFBF8E
:10127000BFBFBFBFBFBFBF645B5B0952BFBFBFBFC4
:10128000645B0900BFBFBFBFBFB65B00BFBFBFBFCE
:10129000BFBFBF5BBFBFBFBFBFBFBFBFBFBFBFBFC2
:1012A000BFBFBFBFBFBFBFBFBFBFBFBFBFBFBFBF4E
:1012B000BFBFBFBF5252000000000000000000008E
:1012C000000000000000000000000000000000001E
:1012D000000000000900000000000000BF0900003D
:1012E00000000000BFB6000000000000BFBF645255
:1012F0005B5252520000000000000000000000009D
:1013000000000000000000000000000000000000DD
:10131000000000000000000000000000AD5B520073
:1013200000000000FFFFFFAD5200000052FFFFFF72
:10133000FF520000020553FF5BADFFFF040454FFA2
:10134000A45BADAD030304AFFFFFFFAD00020505D5
:10135000AFFFFFFF000305050555AEAE0003050511
:101360000505030300010304040404040000000154
:1013700003040404FFADADFFFF560505ADADADFFA1
:10138000FF550505AD5BADFFAE050505FFFFFFAFE2
:10139000050505055D555605050505050305050407
:1013A00004040505050505040303030404040505F9
:1013B00005050505050505050505050505040505DE
:1013C000050505AF03010305050556FF03020405E6
:1013D00005055DFF05040505050556FF0505050521
:1013E000050505AE05050404040505050505050309
:1013F0000405050555AFAEAF5E050505FFFFFFFF10
:10140000FFFF5E05FFADADADFFFFFF55FF5B5BADC1
:10141000ADADFFFFAD5BADFFFF5BA4FFFFADADADBD
:10142000ADADADFFAFFFFFFEADADAEA7035DAFAF9E
:10143000A65D5605050503ADAD5BADFF0505015B7A
:10144000AD5BFFFF05050100520052525604020039
:10145000000000005E0304010000000056040300C9
:101460000000000005040400005200000304020014
:10147000005200005BAD5B52000052005B52000066
:10148000000000000000000000000000000000005C
:10149000000000000000000000000000000000004C
:1014A0005200000000000052520000000052525250
:1014B0000000000000000009000000000000000023
:1014C000000000000000000000000000000000001C
:1014D000000000000000000000000000000000000C
:1014E00000000000000000FFFFFFFFFF000000FF02
:1014F000FFFFFFFF0000FFFFFFFFFFFF0000FFFFF8
:10150000FFFFFF1E0000FFFFFFFF1E3700FFFFFF72
:10151000FF1E373700FFFFFFFF1E373700FFFFFFBB
:101520001E373737FF0000001E373737FF00000037
:101530001E3737371E37373737373737373737376D
:10154000373737373737373737373737373737372B
:101550003737371E373737373737371E373737374D
:10156000373737373737373737373737373737370B
:1015700037373737371EFFFF64BF6465371EFFFFFD
:10158000BFB664641EFFFFFFBFBF5B64FFFFFF00C9
:10159000BFBFB6B61E1E1E1E1E1E5B643737373712
:1015A00037371E64373737373737371E37373737D0
:1015B000373737370000000000000000000000004F
:1015C00000000000645B090000000000B6B6B664CD
:1015D00064646464B6BFBFBFBFBFBFBF6464B6BF4F
:1015E000BFBFB6B6646464B6656464641E6464BFF9
:1015F000BFBFB6B6000000000000645B0000000042
:1016000009095B6400095B5BB6B65BBF646464B6E2
:10161000BF5BB6BFBFBFBFBFBF5B6464B6B6BFBF73
:10162000BFB664646464BFBFBFBFBFBFB6B6BFBF51
:10163000BFBFBFBF64646464646464B6BFB6B6B65B
:10164000645B5BB6BFBFBFBF64646464BFBF6464F8
:1016500064B6645B6464645B6464BFBF64B6BFBF4C
:10166000BFBFBFBFBFBFBFBFBFBFBFBFBFBFBFBF8A
:10167000BFBFBFBFB65BA4AD52005BB6BF645BA487
:101680005264BFBFB6BF5B5BB6BFB66464BFBFBFCB
:10169000BFB66464BFBFBFBFBFB6BFBFBFBFBFBF22
:1016A000BFBFBFBFBFBFBFBFBFBFBFBFBFBFBFBF4A
:1016B000BFBFBFBFBFBFB66464B6BFBF6D645B646E
:1016C000BFBFBFBF5B64BFBFBFBFBFBFBFBFBFBFE9
:1016D000BFBFBFBFBFBFBFBFBFBFBFBFBF646DBFC7
:1016E000BFBFBFBFBFB664BFBFBFBFBFBFBF645B2D
:1016F000BFBFBFBFBFBFBFBFBFBFBFBFBFBFBFBFFA
:10170000BFBFBFBFBFBFBFBFBFBFBFBFBFBFBFBFE9
:10171000BFBFBFBFBFBFBFBFBFBFBFBFBFBFBFBFD9
:10172000BFBFBFBFBFBFBFBFBFBFBFB6BFBFBFBFD2
:10173000BFBFFFFFBFBFBFBFBFBFBFBFBFBFBFBF39
:10174000BFBFBFBFBFBFBFBFBFBFBFBFBFBFBFBFA9
:10175000BFBFBFBFBFBFBFBFB7BFBFBFBFB6FFFF2A
:10176000FFFFFFB6FFFFFFFFFFFFFFFFFFFFFFFFD2
:10177000FFFFFFFFBFBFBFBFBFBFBFBFBFBFBFBF79
:10178000BFBFBFBFBFBFBFBFBFBFBFBFBFBFBFBF69
:10179000BFBFBFBFBFBFBFBFBFBFBFBFBFBFBFBF59
:1017A000BFBFBFBFB66464BFBFBFBFBFA4645BBFE2
:1017B000BFBFBFBFBFBFBFADAD5B52ADBFBFFFFFC0
:1017C0005BAD00ADBFB6FFFF5B5B5252BFFFFFAD2D
:1017D00052525B00B6AD5BADAD5B5B00B6AD00FFDA
:1017E000ADAD5B00FFFFAD5BADADAD00ADADFF5B83
:1017F000525BAD5B00ADFFFFFFAD00000052FFFF8D
:10180000FFFF52005200FFFFFFFFAD005B00ADFF86
:10181000FFFFAD005B52ADFFFFFFFF00525BADFF6E
:10182000FFFFAD0052ADFFFFFFFF520000ADFFFF15
:10183000FFAD0000000000000103040400000000F0
:101840000000010300000000000000000000000094
:101850000000000000000000000000000000000088
:101860000000000000000000000000000000000078
:101870000000000004040303030404050505050536
:101880000504030200010203040405050000000032
:101890000000000000000000000000000000000048
:1018A0000000000000000000000000000000000038
:1018B00000000000050505050505050502020304F5
:1018C00005050505050403020101020301020203E7
:1018D00003040303000000000000000000000000FB
:1018E00000000000000000000000000000000000F8
:1018F00000000000030303050505050305040405B6
:10190000050504020405050505050205020202039A
:1019100003020301000102020200000000000000B7
:1019200000000000000000000000000000000000B7
:1019300000000000030400000052525205020000A3
:101940000000000003000000000000000000000094
:101950000000000000000000000000000000000087
:101960000000000000000000000000000000000077
:1019700000000000525200000000000000000000C3
:101980000000000000000000000000000000000057
:101990000000000000000000000000000000000047
:1019A0000000000000000000000000000000000037
:1019B00000000000000000FFFFFFFFFF0000FFFF2E
:1019C000FFFFFFFF0000FFFFFFFFFFFF0000FFFF23
:1019D000FFFFFFFF0000000000000000000000000B
:1019E00000000000000000000000000000000000F7
:1019F000000000FFFF000000001E3737000000005D
:101A0000001E373700000000001E373700000000BE
:101A100000001E37FFFFFFFFFFFF001EFFFFFFFF5D
:101A2000FFFF0000FFFFFFFFFFFF0000FFFFFFFFC2
:101A3000FF00000037373737373737373737373713
:101A40003737373737373737373737371E1E1E1E8A
:101A50001E1E1E1E0000000000FFFFFF0000000011
:101A600000FFFFFF0000000000FFFFFF000000007C
:101A7000FFFFFFFF373737373737373737373737D6
:101A80003737373737373737373737371E1E1E1E4A
:101A90001E1E1E1EFFFFFFBFBF5B0964FFFFFFBFCF
:101AA000BF64BFBFFFFFFFBFBFBFBFBFFFFF645B20
:101AB00064BFBFBF1EBFBFBFBFBFBFBF1E64BFBF2E
:101AC000BFBFBFBF1EBFBFBFBFBFBFBF64BFBFBF22
:101AD000BFBFBFBFBFBFBFBFBFBFBFBFBFBFBFBF16
:101AE000BFBFBFBFBFBFBFBFBFBFBFBFBFBFBFBF06
:101AF000BFBFBFBFBFBFBFBFBFBFBFBFBFBFBFBFF6
:101B0000BFBFBFBFBFBFBFBFBFBFBFBFBFBFBFBFE5
:101B1000BFBFBFBFBFBFBFBFBFBFBFBFBFBFBFBFD5
:101B2000BFBFBFBFBFBFBFBFBFBFBFBFBFBFBFBFC5
:101B3000BFBFBFBFBFBFBFBFBFBF6464BFBFBFBF6B
:101B4000645B5BADBFBFBF5B00005252BFB65B00C2
:101B50000000FF5BB60900000000FFADB65B5B0054
:101B60000000ADADBF6D5B000000ADADBFBF5B0061
:101B700000005BFF5BADADB6BFBFBFBF5B5BADAD94
:101B8000AD64BFBF5B5B5200005B5B09ADFFFFFF55
:101B900052520000ADFFFF5BADAD52525BAD5BAD8D
:101BA000AD52ADFF5BADADFF5BADFFFFADADFF5B1C
:101BB000ADFFFFFFBFBFBF6464BFBFBFBFBFBFBF3D
:101BC0005BB6BFBF64BFBFBF6D09BFBF0064BFBF0F
:101BD000BF5B64BF000064BFBFBF5BB65B0000B605
:101BE000BFBF6D5BFFAD0009BFBFBFADFFFF5B00B7
:101BF00009BFBFB6BFBFBFBFB7FFFFFFBFBFBFB605
:101C0000FFFFFFFFBFBFFFFFFFFFFFFFBFFFFFFFA4
:101C1000FFFFFFFFFFFFFFFFFFFFFFADFFFFFFFF26
:101C2000FFAD5B52A4ADAD5B52525BADAD5B5200FC
:101C30005BFFFFFFFFFFFFFFFFFFFFFFFFFFFFFF58
:101C4000FFFFFFFFFFFFFF5BFFFFFFFFFFAD525BEB
:101C5000FFFFFFFF525BAD00ADFFADAD5BFFA4A486
:101C600052AD5BADFFFF5BAD5B5BFFFFFFFF5BFF5B
:101C7000AD5BFFFF52AD0964BFBFB65BAD5BB65B4A
:101C8000BF645B64FFADBF645B64BFBFFFAD5B64FB
:101C9000BFBFBFBF5BADFFBFBFBFBFBFFFFFFFFF8A
:101CA000BFBFBF65FFFFFFFFBFBFB65BFFFFFFFF0B
:101CB0006DBFBFBF5BADFFAD52ADFFFFB6FFFFFF16
:101CC000FFADADFFBFFFFFFFAD52ADFFBFFFFFADEB
:101CD00052FFFFFFBFADFFFFFFFFFFB65B64B6B66D
:101CE000B6B6BFBF65BFBFBFBFBFBF5BBFBFBFBFD4
:101CF000BFBFBFB6525BFFFFAD520000AD00FFFF9C
:101D000052000000FF525B5200000000FFAD0000D7
:101D100000000000BFBF090000000000646409006B
:101D2000000000005B5B0900000000005B5B6409D1
:101D3000000000000000000000095BB60000000089
:101D40000000000000000000000000000000000093
:101D50000000000000000000000000000000000083
:101D60000000000000000000000000000000000073
:101D700000000000BFBFBFBFBFBFBFBF0964B6BF89
:101D8000BFBFBFBF0909095B64B6B6BF005B645B38
:101D90005B095B640000095B5B5B5B5B0000000050
:101DA000000900000000000000000000000000002A
:101DB00000000000BFBFBFBFBFBFBFBFBFBFBFBF2F
:101DC000BFBFBFBFBFBFBFBFBFBFBFBF64B66DB6E2
:101DD000B6B6BFBF5B5B6464646464BF095B646484
:101DE000646464640000095B6464B6B600000000CB
:101DF00000095B64BFBF5B00000052FFBFBF5B0018
:101E0000000000ADBFBF5B0052000052BFBF6400C6
:101E100052000000BFBFB6095200000064646409AC
:101E200000000000B6B66464000000006464645BF7
:101E300000000000FFFF5BADFFFFFFFFFFFF5BAD9A
:101E4000FFFFFFADFFFF5BADADADAD5BADFFAD5BCC
:101E50005B5B5BAD52ADFFFFFFFFFFFF005BFFFF72
:101E6000FFFFADAD00005BAD5B5B5200000000000A
:101E700000000000FFFFAD000064BFB6ADAD000084
:101E800000006DBFADAD000000005BBFFF52000061
:101E9000000009B65B0000000000006400000000C4
:101EA00000520009000000000000000900000000CE
:101EB00000000000FFFFAD52FFFFFFFFFFFFFF52DA
:101EC000FFFFFFFFFFFFFFAD5BFFFFADFFFFFFFF6A
:101ED00052AD5B52B6FFFFFFAD5BADFFBFB6FFFF7C
:101EE000FFFFFFFF6DBFB6FFFFFFFFFF5BBFBFB68A
:101EF000FFFFFFFFFFFF5B52005BFFFFFF5B52AD89
:101F0000FFFFFFFF525BFFFFFFFFFFADADFFFFFFD6
:101F1000FFFFAD52FFFFFFFFFFAD52ADFFFFFFFF21
:101F2000FFADADB6FFFFFFFFFFFFBFBFFFFFFFB677
:101F3000BFB6BFBFFFFFFF5B5BBFBFBFFFFF5B6401
:101F4000BFBFBFBFFFFFB6BFBFBFBFBFADFFBFBFFC
:101F5000BFBFBFBFB6BFBFBFBFBFBFBFBFBFBFBF9A
:101F6000BFBFBFBFBFBFBFBFBFBFBFBFBFBFBFBF81
:101F7000BFBFBF64BFBFBFBFBFBFBFBFBFBFBFBFCC
:101F8000BFBFBFBFBFBFBFBFBFBFBFBFBFBFBFBF61
:101F9000BFBFBF64BFBFBFBFBF645B00BFBFB6648E
:101FA0005B090000B664645B09000000645B090023
:101FB0000000000064B6BF5B00000000BFBFB609B0
:101FC00000000000BF6D090000000000640900006F
:101FD0000000000000000000000000000000000001
:101FE00000000000000000000000000000000000F1
:101FF00000000000000000000000000000000000E1
:10200000520000000000000000000000000000007E
:102010000000005200525252525252000000000082
:1020200000000000000000000000000000000000B0
:1020300000000000000000000052520000520000AA
:1020400052525200525252525200000052525252B8
:102050000000000000000000000000000000000080
:102060000000000000000000000000000000000070
:1020700000000000000964BFBFB7B6B60000005BF7
:10208000BFBFBFBF000000000964BFBF0000000069
:10209000000064BF000000000000005B00000000C2
:1020A0000000000000000000000000000000000030
:1020B00000000000B6B7BFBF5B5BBFBFBFBF645BC4
:1020C00064646DBFBF5B645B5B5B64BF645BB66491
:1020D0005B64BFBFBF64B664BFBF645B64BFB6640C
:1020E0005B095BB600095B5B5B6DBF6400000009C8
:1020F0005B090000BFBFBFBFBFB65B64BFBFBFBF50
:10210000645B645BBFBF645B6464090064646464B3
:102110005B00000064BF640900000000B65B0000C3
:1021200000000000090000000000000000000000A6
:10213000000000005B09000000000000000000003B
:10214000000000000000000000000000000000008F
:10215000000000000000000000000000000000007F
:10216000000000000000000000000000000000006F
:10217000000000005B0900000000000000000000FB
:10218000000000000000000000000000000000004F
:10219000000000000000000000000000000000003F
:1021A000000000000000000000000000000000002F
:1021B0000000000029292929292929292929292933
:1021C000292929292929292929292929292929297F
:1021D000292929292929292929292929292929296F
:1021E000292929292929292929292929292929295F
:1021F000292929290000070707070000000707070A
:102200000707070007070707070707070707070765
:10221000070707070707070707070707070707074E
:10222000070707070007070707070700000007075A
:1022300007070000292929292929292929292929A4
:1022400029292929292929292929292929292929FE
:1022500029292929292929292929292929292929EE
:10226000292929FF29292929290606522929292925
:10227000FF5252522929292929292929292929297D
:10228000292929FF29292929FF060652292906FF7C
:1022900052525252FF0652525252525252525252BD
:1022A000525252525252525252525252525252520E
:1022B00052525252292929FFFF0606FFFF060652F5
:1022C00052525252525252525252525252525252EE
:1022D00052525252525252525252525252525252DE
:1022E00052525252525252525252525252525252CE
:1022F00052525252FF0606FFFF29292952525252CA
:10230000520606FF52525252525252525252525298
:10231000525252525252525252525252525252529D
:10232000525252525252525252525252525252528D
:10233000525252522929292929292929FF29292993
:1023400029292929520606FF2929292952525252A0
:10235000FF06292952525252525206FF52525252ED
:10236000525252525252525252525252525252524D
:102370005252525229292929292929292929292929
:1023800029292929292929292929292929292929BD
:1023900029292929292929292929292906292929D0
:1023A000292929295206FF29292929295252520669
:1023B00029292929FF52525252525252FF52525247
:1023C0005252525206525252525252520652525285
:1023D00052525252FF5252525252525229FF5252AC
:1023E00052525252290652525252525229065252B7
:1023F00052525252525252525252525252525252BD
:1024000052525252525252525252525252525252AC
:10241000525252525252525252525252525252529C
:10242000525252525252525252525252525252528C
:1024300052525252525252525252520652525252C8
:10244000525252525252525252525252525252526C
:10245000525252525252525252525252525252525C
:10246000525252525252525252525252525252524C
:102470005252525206525252525252525252525288
:10248000525252525252525252525252525252522C
:10249000525252525252525252525252525252521C
:1024A000525252525252525252525252525252520C
:1024B0005252525252525252525252FF525252524F
:1024C000525252FF5252525252525206525252528B
:1024D0005252520652525252525252FF525252527B
:1024E00052520629525252525252062952525252B6
:1024F0005252FF29065252525252525206525252D0
:102500005252525206525252525252520652525243
:102510005252525206525252525252520652525233
:102520005252525206525252525252520652525223
:1025300052525252525252525252520652525252C7
:102540005252520652525252525252065252525203
:1025500052525206525252525252520652525252F3
:1025600052525206525252525252520652525252E3
:1025700052525206060606060606060652525252E7
:10258000525252525252525252525252525252522B
:10259000525252525252525252525252525252521B
:1025A000525252525252525252525252525252520B
:1025B000525252520000181818180000001818182B
:1025C00018181800181818181818181818181818A3
:1025D000181818181818181818181818181818187B
:1025E00018181818001818181818180000001818CB
:1025F00018180000292929292929292929292929BF
:10260000292929292929292929292929292929293A
:10261000292929292929292929292906292929294D
:102620002929FF5229292929292906522929292915
:102630002906525229292906525252522929065254
:102640005252525229FF5252525252520652525232
:10265000525252525252525252525252525252525A
:10266000525252525252525252525252525252524A
:102670005252525252525252062929295252525201
:1026800052FF2929525252525252FF29525252524B
:102690005252520652525252525252525252525266
:1026A000525252525252525252525252525252520A
:1026B00052525252292929292929292929292929E6
:1026C000292929292929292929292929292929297A
:1026D00029292929062929292929292952FF29298E
:1026E0002929292952FF292929292929525206292C
:1026F0002929292929FF5252525252522929FF527F
:1027000052525252292906525252525229290652E5
:1027100052525252292929FF52525252292929FF35
:10272000525252522929292906525252292929291D
:1027300006525252525252525252FF295252525241
:1027400052062929525252525206292952525252A5
:1027500052FF292952525252FF29292952525252CC
:10276000062929295252520629292929525252FF53
:102770002929292900003A3A3A3A0000003A3A3A1F
:102780003A3A3A003A3A3A3A3A3A3A3A3A3A3A3AE3
:102790003A3A3A3A3A3A3A3A3A3A3A3A3A3A3A3A99
:1027A0003A3A3A3A003A3A3A3A3A3A0000003A3A71
:1027B0003A3A000029292929FF5252522929292968
:1027C000FF525252292929065252525229292906CA
:1027D000525252522929FF52525252522929FF5223
:1027E00052525252292906525252525229065252DC
:1027F000525252525252520629292929525252FFFC
:102800002929292952525252FF292929525252521A
:1028100006292929525252525206292952525252FD
:1028200052FF29295252525252FF292952525252D2
:10283000525206292929292929FF525229292929B1
:1028400029290652292929292929065229292929EC
:10285000292929FF29292929292929292929292912
:1028600029292929292929292929292929292929D8
:1028700029292929525252525252525252525252DC
:102880005252525252525252525252525252525228
:1028900052525252FF5252525252525229065252E0
:1028A000525252522929065252525252292929FF74
:1028B00052525252525252525252525252525252F8
:1028C00052525252525252525252525252525252E8
:1028D0005252525252525252525252065252525224
:1028E000525206295252525252FF292952525252E2
:1028F000FF2929295252FF29292929295206292944
:10290000292929295206292929292929FF2929295B
:102910002929292929292929292929292929292927
:102920002929292929292929292929292929292917
:1029300029292929000004040404000000040404D7
:10294000040404000404040404040404040404044B
:102950000404040404040404040404040404040437
:102960000404040400040404040404000000040437
:102970000404000029FF52525252525229FF52526F
:1029800052525252290652525252525206525252E8
:1029900052525252FF52525252525252FF525252BD
:1029A000525252520652525252525252065252529F
:1029B00052525252525252525252525252525252F7
:1029C00052525252525252525252525252525252E7
:1029D00052525252525252525252525252525252D7
:1029E00052525252525252525252525252525252C7
:1029F0005252520652525252525252525252525203
:102A000052525252525252525252525252525252A6
:102A10005252525252525252525252525252525296
:102A200052525252525252525252525206525252D2
:102A300052525252525252525252FF2952525252F2
:102A40005252FF2952525252525206295252525257
:102A50005252520652525252525252FF52525252F5
:102A6000525252FF525252525252520652525252E5
:102A70005252520600000000FFFFFFFF000000005E
:102A8000FFFFFFFF00000000FFFFFFFF000000004E
:102A9000FFFFFFFFFFFFFFFF00000000FFFFFFFF42
:102AA00000000000FFFFFFFF00000000FFFFFFFF2E
:102AB0000000000029292929FF52525229292929D9
:102AC0002906065229292929292929FF29292929BD
:102AD0002929292929292929292929292929292966
:102AE0002929292929292929292929292929292956
:102AF000292929295252525252525252525252525A
:102B0000525252525252525252525252FF06525244
:102B100052525252292906FF52525252292929292A
:102B2000FF06065229292929292929FF2929292986
:102B30002929292952525252525252525252525219
:102B40005252525252525252525252525252525265
:102B50005252525252525252525252525252525255
:102B600052525252FF06065252525252292929FFFE
:102B7000FF0606FF52525252525252525252525273
:102B80005252525252525252525252525252525225
:102B90005252525252525252525252525252525215
:102BA000525252525252525252FF0606FF0606FF2E
:102BB0002929292952525252525252525252525299
:102BC00052525252525252525252525252525252E5
:102BD0005252060652525252FFFF292952FF060650
:102BE00029292929FF29292929292929292929297F
:102BF00029292929525252062929292952FF062911
:102C000029292929FF29292929292929292929295E
:102C10002929292929292929292929292929292924
:102C20002929292929292929292929292929292914
:102C30002929292952525252525252525252525218
:102C40005252525252525252525252525252525264
:102C50005252525252525252525252525252525254
:102C60005252525252525252525252520606060674
:102C7000060606060000000000000000000000003C
:102C80000000000000000000000000000000000044
:102C90000000000000000000000000000000000034
:102CA0000000000000000000000000000000000024
:102CB0000000000000000000000000003F3F000096
:102CC000000000003F3F00003F0000000000003F08
:102CD0000000000000003F0000000000003F000076
:102CE000000000003F00003F3F0000000000003FE8
:102CF0003F00000000000000000000000000000095
:102D0000FFFF0000000000FF000000000000FF00C7
:102D1000000000000000FF00000000000000FF00B5
:102D200000000000000000FF0000000000000000A4
:102D3000FFFF000000000000000000000000FFFF97
:102D40000000000000000000FF0000000000000084
:102D500000FF00000000000000FF00000000000075
:102D600000FF000000000000FF0000000000FFFF67
:102D70000000000000000000000000000000FFFF55
:102D8000FF00000000FFFF00FFFF0000FFFF00004A
:102D900000FFFF00FFFF000000FFFF00FFFFFFFF3D
:102DA000FFFFFF00FFFF000000FFFF00FFFF00002C
:102DB00000FFFF000000000000000000FFFFFFFF19
:102DC000FFFF0000FFFF000000FFFF00FFFF00000B
:102DD00000FFFF00FFFFFFFFFFFF0000FFFF0000FD
:102DE00000FFFF00FFFF000000FFFF00FFFFFFFFED
:102DF000FFFF000000000000000000000000FFFFD7
:102E0000FFFF000000FFFF0000FFFF00FFFF0000CA
:102E100000000000FFFF000000000000FFFF0000B6
:102E20000000000000FFFF0000FFFF000000FFFFA8
:102E3000FFFF00000000000000000000FFFFFFFF98
:102E4000FF000000FFFF0000FFFF0000FFFF000089
:102E500000FFFF00FFFF000000FFFF00FFFF00007A
:102E600000FFFF00FFFF0000FFFF0000FFFFFFFF6C
:102E7000FF0000000000000000000000FFFFFFFF57
:102E8000FFFFFF00FFFF000000000000FFFF000049
:102E900000000000FFFFFFFFFFFF0000FFFF00003A
:102EA00000000000FFFF000000000000FFFFFFFF28
:102EB000FFFFFF000000000000000000FFFFFFFF19
:102EC000FFFFFF00FFFF000000000000FFFF000009
:102ED00000000000FFFFFFFFFFFF0000FFFF0000FA
:102EE00000000000FFFF000000000000FFFF0000E6
:102EF0000000000000000000000000000000FFFFD4
:102F0000FFFFFF0000FFFF0000000000FFFF0000C8
:102F100000000000FFFF0000FFFFFF00FFFF0000B8
:102F200000FFFF0000FFFF0000FFFF000000FFFFA9
:102F3000FFFFFF000000000000000000FFFF000096
:102F400000FFFF00FFFF000000FFFF00FFFF000089
:102F500000FFFF00FFFFFFFFFFFFFF00FFFF00007C
:102F600000FFFF00FFFF000000FFFF00FFFF000069
:102F700000FFFF00000000000000000000FFFFFF56
:102F8000FFFFFF00000000FFFF000000000000FF47
:102F9000FF000000000000FFFF000000000000FF35
:102FA000FF000000000000FFFF00000000FFFFFF27
:102FB000FFFFFF000000000000000000000000FF15
:102FC000FFFFFF0000000000FFFF00000000000006
:102FD000FFFF000000000000FFFF000000000000F5
:102FE000FFFF0000FF000000FFFF000000FFFFFFE9
:102FF000FF0000000000000000000000FFFF0000D4
:1030000000FFFF00FFFF0000FFFF0000FFFF00FFC9
:10301000FF000000FFFFFFFF00000000FFFFFFFFB9
:10302000FF000000FFFF00FFFFFF0000FFFF0000A8
:10303000FFFFFF00000000000000000000FFFF0095
:103040000000000000FFFF000000000000FFFF0084
:103050000000000000FFFF000000000000FFFF0074
:103060000000000000FFFF000000000000FFFFFF65
:10307000FFFFFF00000000000000000000003F3FD5
:103080003F000000003F00003F3F00003F3F0000C6
:10309000003F3F003F3F0000003F3F003F3F000038
:1030A000003F3F00003F3F00003F000000003F3F67
:1030B0003F00000000000000000000000000003F92
:1030C0003F00000000003F3F3F0000000000003FC5
:1030D0003F0000000000003F3F0000000000003FF4
:1030E0003F0000000000003F3F000000003F3F3F66
:1030F0003F3F3F000000000000000000003F3F3F56
:103100003F3F00003F3F0000003F3F000000000045
:103110003F3F3F0000003F3F3F3F0000003F3F3F39
:103120003F0000003F3F3F00000000003F3F3F3FA7
:103130003F3F3F000000000000000000003F3F3F15
:103140003F3F3F00000000003F3F00000000003F05
:103150003F00000000003F3F3F3F00000000000034
:10316000003F3F003F3F0000003F3F00003F3F3F28
:103170003F3F000000000000000000000000003F92
:103180003F3F000000003F3F3F3F0000003F3F0047
:103190003F3F00003F3F00003F3F00003F3F3F3FB9
:1031A0003F3F3F00000000003F3F000000000000E4
:1031B0003F3F000000000000000000003F3F3F3F95
:1031C0003F3F00003F3F0000000000003F3F3F3F07
:1031D0003F3F000000000000003F3F0000000000F3
:1031E000003F3F003F3F0000003F3F00003F3F3FA8
:1031F0003F3F0000000000000000000000003F3FD3
:103200003F3F0000003F3F00000000003F3F000044
:10321000000000003F3F3F3F3F3F00003F3F0000B6
:10322000003F3F003F3F0000003F3F00003F3F3F67
:103230003F3F000000000000000000003F3F3F3F14
:103240003F3F3F003F3F0000003F3F0000000000C5
:103250003F3F00000000003F3F00000000003F3FF4
:103260000000000000003F3F0000000000003F3F62
:10327000000000000000000000000000003F3F3F91
:103280003F0000003F3F0000003F00003F3F3F0085
:10329000003F0000003F3F3F3F0000003F00003F75
:1032A0003F3F3F003F000000003F3F00003F3F3FE7
:1032B0003F3F00000000000000000000003F3F3FD3
:1032C0003F3F00003F3F0000003F3F003F3F000006
:1032D000003F3F00003F3F3F3F3F3F0000000000F6
:1032E000003F3F00000000003F3F0000003F3F3F25
:1032F0003F0000000000000000000000000000008F
:10330000000000000000FFFF000000000000FFFFC1
:103310000000000000000000000000000000FFFFAF
:10332000000000000000FFFF00000000000000009F
:10333000000000000000000000000000FFFF00008F
:1033400000FFFF00FFFFFF00FFFFFF00FFFFFFFF89
:10335000FFFFFF00FFFFFFFFFFFFFF00FFFF00FF7A
:1033600000FFFF00FFFF000000FFFF00FFFF000065
:1033700000FFFF000000000000000000FFFF000051
:1033800000FFFF00FFFFFF0000FFFF00FFFFFFFF48
:1033900000FFFF00FFFFFFFFFFFFFF00FFFF00FF39
:1033A000FFFFFF00FFFF0000FFFFFF00FFFF000027
:1033B00000FFFF00000000000000000000FFFFFF12
:1033C000FFFF0000FFFF000000FFFF00FFFF000005
:1033D00000FFFF00FFFF000000FFFF00FFFF0000F5
:1033E00000FFFF00FFFF000000FFFF0000FFFFFFE6
:1033F000FFFF00000000000000000000FFFFFFFFD3
:10340000FFFF0000FFFF000000FFFF00FFFF0000C4
:1034100000FFFF00FFFF000000FFFF00FFFFFFFFB6
:10342000FFFF0000FFFF000000000000FFFF0000A2
:1034300000000000000000000000000000FFFFFF8F
:10344000FFFF0000FFFF000000FFFF00FFFF000084
:1034500000FFFF00FFFF000000FFFF00FFFF00FF75
:10346000FFFFFF00FFFF0000FFFF000000FFFFFF66
:10347000FF00FF000000000000000000FFFFFFFF52
:10348000FFFF0000FFFF000000FFFF00FFFF000044
:1034900000FFFF00FFFF0000FFFFFF00FFFFFFFF37
:1034A000FF000000FFFF00FFFFFF0000FFFF000024
:1034B000FFFFFF00000000000000000000FFFFFF12
:1034C000FF000000FFFF0000FFFF0000FFFF000003
:1034D0000000000000FFFFFFFFFF000000000000F1
:1034E00000FFFF00FFFF000000FFFF0000FFFFFFE5
:1034F000FFFF0000000000000000000000FFFFFFD1
:10350000FFFFFF00000000FFFF000000000000FFC1
:10351000FF000000000000FFFF000000000000FFAF
:10352000FF000000000000FFFF000000000000FF9F
:10353000FF0000000000000000000000FFFF00008E
:1035400000FFFF00FFFF000000FFFF00FFFF000083
:1035500000FFFF00FFFF000000FFFF00FFFF000073
:1035600000FFFF00FFFF000000FFFF0000FFFFFF64
:10357000FFFF00000000000000000000FFFF00004F
:1035800000FFFF00FFFF000000FFFF00FFFF000043
:1035900000FFFF00FFFFFF00FFFFFF0000FFFFFF36
:1035A000FFFF00000000FFFFFF000000000000FF21
:1035B000000000000000000000000000FFFF00000D
:1035C00000FFFF00FFFF000000FFFF00FFFF00FF04
:1035D00000FFFF00FFFFFFFFFFFFFF00FFFFFFFFF8
:1035E000FFFFFF00FFFFFF00FFFFFF00FFFF0000E6
:1035F00000FFFF000000000000000000FFFF0000CF
:1036000000FFFF00FFFFFF00FFFFFF0000FFFFFFC5
:10361000FFFF00000000FFFFFF00000000FFFFFFB2
:10362000FFFF0000FFFFFF00FFFFFF00FFFF0000A4
:1036300000FFFF00000000000000000000FFFF008E
:1036400000FFFF0000FFFF0000FFFF0000FFFF0082
:1036500000FFFF000000FFFFFFFF0000000000FF71
:10366000FF000000000000FFFF000000000000FF5E
:10367000FF0000000000000000000000FFFFFFFF4F
:10368000FFFFFF0000000000FFFFFF00000000FF41
:10369000FFFF00000000FFFFFF00000000FFFFFF32
:1036A00000000000FFFFFF0000000000FFFFFFFF21
:1036B000FFFFFF0000000000000000FF0000FFFF10
:1036C000FF00FF0000FFFF00FFFF0000FFFF000002
:1036D00000FFFF00FFFF000000FFFF00FFFFFFFFF4
:1036E000FFFFFF00FFFF000000FFFF00FFFF0000E3
:1036F00000FFFF00FEFE05050505FEFEFE05FF05B9
:1037000005FF05FE00050505050505000005FFFF91
:10371000FFAD0500FE05FFFFADAD05FE000505058B
:10372000050505000005FFFFFFAD0500FE050505C9
:10373000050505FEFEFE000005FFFEFEFEFE00FF85
:10374000FF0505FE000005FFFFFF05FF000505055D
:10375000FFFFAD0505FFFF0505ADAD000505FFAD9C
:1037600005050000FE0505AD0500FEFEFEFE050593
:103770000000FEFEFE0000FE0000FEFE0505050541
:10378000050505FE05FF05FFFF05FF0505FF05FF14
:10379000FF05050505FF05FFAD05050505AD05ADF3
:1037A000AD05FF0505050505050505FEFE0000FE46
:1037B0000000FEFEFEFE05050000FEFEFE0505AD56
:1037C0000500FEFE0505FFAD0505000005FFFF0530
:1037D00005ADAD0000050505FFFFAD05000005FFC7
:1037E000FFFF05FFFEFE00FFFF0505FEFEFE0000D9
:1037F00005FFFEFEFE050505050505FE0005FFFFAC
:10380000FFAD05000005050505050500FE05FFFFE8
:10381000FFAD05FE0005FFFFADAD05000005050588
:1038200005050500FE05FF0505FF05FEFEFE050575
:103830000505FEFEFEFE7F7F7F7FFEFEFE7FFF7F93
:103840007FFF7FFE007F7F7F7F7F7F00007FFFFF06
:10385000FFAD7F00FE7FFFFFADAD7FFE007F7F7F6E
:103860007F7F7F00007FFFFFFFAD7F00FE7F7F7FB8
:103870007F7F7FFEFEFE00007FFFFEFEFEFE00FF5C
:10388000FF7F7FFE00007FFFFFFF7FFF007F7F7FC6
:10389000FFFFAD7F7FFFFF7F7FADAD007F7FFFAD7F
:1038A0007F7F0000FE7F7FAD7F00FEFEFEFE7F7FFC
:1038B0000000FEFEFE0000FE0000FEFE7F7F7F7F18
:1038C0007F7F7FFE7FFF7FFFFF7FFF7F7FFF7FFF89
:1038D000FF7F7F7F7FFF7FFFAD7F7F7F7FAD7FADEE
:1038E000AD7FFF7F7F7F7F7F7F7F7FFEFE0000FEBB
:1038F0000000FEFEFEFE7F7F0000FEFEFE7F7FAD2D
:103900007F00FEFE7F7FFFAD7F7F00007FFFFF7F98
:103910007FADAD00007F7F7FFFFFAD7F00007FFFA9
:10392000FFFF7FFFFEFE00FFFF7F7FFEFEFE000029
:103930007FFFFEFEFE7F7F7F7F7F7FFE007FFFFF9A
:10394000FFAD7F00007F7F7F7F7F7F00FE7FFFFFD7
:10395000FFAD7FFE007FFFFFADAD7F00007F7F7F6B
:103960007F7F7F00FE7FFF7F7FFF7FFEFEFE7F7FEA
:103970007F7FFEFE0002060000FB00FF0002090040
:1039800000F100FF0002090000FE00FF0001050039
:1039900000E219010302050000FF0001000000E23F
:1039A00032010102050000FF0001280000FEFA01BB
:1039B0000102050000FF0001000000FB9601030268
:1039C000050000FF0001000000E20F0103020500F6
:1039D00000FF0001030000F64B010302050000FF99
:1039E0000001020000EC1901FF03050000FF0001C7
:1039F000FF0000CE0501FF03050000FF00020800E4
:103A0000085504085A0000F8000990000A1E320503
:103A10000000FF0000007439000000000000007C7E
:103A2000390000000000000084390000000001009F
:103A3000008C39000000000100009A3900000000ED
:103A4000010000A83900000000010000B6390000A4
:103A50000000010000C43900000000010000D2395C
:103A600000000000010000E039000000000100003B
:103A7000EE3900000000000000FC390000000000EA
:103A8000FF06015300B0077F005C00000B7F00C001
:103A9000010090214000B1077F005C00000B7F0017
:103AA000C10000912D400F902140009130400F90B7
:103AB0002140009132400F902140009134401090FD
:103AC0002140009145400F902140009148400F90C7
:103AD00021400091404010902140009143400F90C0
:103AE0002140009132400F902140009134401090CD
:103AF0001F40009137400F901E40009139400F90B9
:103B0000214000913C401090214000913E400F9098
:103B10002140009137400F90214000913940109092
:103B20002140009140400F902140009143400F9070
:103B3000214000914540109021400F2140009145C7
:103B4000400F9021400091484010901F400F1E40B0
:103B5000009148400F90214000914A401090214030
:103B60000F21400F214010214000914A400F902129
:103B700040009149400F9021400091484010902111
:103B800040009147400F902140009145400F902107
:103B9000400091444010901F40009143400F901E00
:103BA00040009140400F90214000913E40109021F4
:103BB0004000913C400F9021400F21401021400FC8
:103BC00021400F21401021400F2140009145400F1E
:103BD0009021400091484010901F40009140400FBC
:103BE000901E40009143400F32400F33401034404C
:103BF0001E41401042400F43400F44401048400FC8
:103C000045402E9021400F21401021400F21400FB0
:103C100021401021400F21400F21401021400F2151
:103C2000400F1F40101E400F21400F214010214027
:103C30000F21400F21401021400F21400F21401043
:103C400021400F21400F1F40101E400F21400091C6
:103C50002B400F90214000912D4010902140009169
:103C600030400F902140009132400F902140009150
:103C7000454010902140009143400F902140009119
:103C800040400F90214000913E4010902140009113
:103C900030400F902140009132400F901F40009122
:103CA00034400F901E400091374010902140009109
:103CB00040400F90214000913E400F9021400091E4
:103CC00039401090214000913C400F9021400091DC
:103CD00034400F90214000913740109021400091D6
:103CE00039400F90214000913C400F9021400091BD
:103CF00039401090214000913C400F901F400091AE
:103D000034400F901E4000913740109021400091A8
:103D10002D400F90214000912E400F9021400091A6
:103D20002F4010902140009130400F902140009191
:103D300032400F902140009133401090214000917B
:103D400034400F902140009137400F902140009166
:103D50003940109021400F1F400F1E40102140009D
:103D60009139400F90214000913C400F902140102C
:103D700021400F214000913C400F90214000913F95
:103D800040109021400F21400F21401021400F1F73
:103D9000400F1E401021400F21400F2140102140B4
:103DA0000F21400F21401021400F21400F21400FD3
:103DB0002140101F400F1E400F214000913740103E
:103DC000902140009139400F902140009137400FE1
:103DD00090214000913940109021400F21400F2147
:103DE000401021400F2140009140400F90214000A1
:103DF00091404010901F40009140400F901E4000A5
:103E00009140400F9021400091434010902140008C
:103E10009143400F902140009143400F902140007A
:103E200091434010902140009145400F9021400067
:103E30009145400F90214000914540109021400055
:103E40009145400F902140009148400F9021400043
:103E500091484010901F40009148400F901E400034
:103E60009148400F90214000914A4010902140001D
:103E7000914A400F90214000914A400F902140000C
:103E8000914A401090214000914C400F90214000F9
:103E9000914E400F90214000914F401090214000E2
:103EA0009151400F9021400F2140101F400F1E40A4
:103EB0000FFF06014500FF2F0000B0076F005C00F8
:103EC000000B7F00C00000FF06015300902D400052
:103ED000B1077F005C00000B7F00C1020091214010
:103EE0000F902D400F3440009124400F902D400042
:103EF00091214010902D40009121400F902D4000C5
:103F00009121400F9034400091284010902D4000A6
:103F1000912B400F9042400091214004904040037B
:103F20003E40043B40043B400439400437400436E3
:103F3000400334400091244004903240042D400856
:103F40009121400F214008902B40079121401028DB
:103F5000400790374004394004374000912B40041B
:103F6000903240043440033240042D4000912140FF
:103F70000F902D40103440009124400F902D4000B0
:103F80009121400F902D400091214010902D400034
:103F90009121400F903440009128400F902D400017
:103FA000912B4010902D40009121400F902D400FFB
:103FB0002D400091244008902F40072D4000912172
:103FC0004008902F400832400091214007902F4038
:103FD000083240009121400890344007324000915F
:103FE00028400890344008364000912B4007903418
:103FF00040082D40009121400F902D400F3440008B
:1040000091244010902D40009121400F902D4000B0
:104010009121400F902D400091214010903440009C
:104020009128400F902D4000912B400F904240006E
:1040300091214004904040043E40043B40043B40FA
:104040000339400437400436400434400091244092
:1040500004903240032D40089121400F21400890E8
:104060002B40089121400F284008903740033940E9
:1040700004374000912B4004903240043440043215
:1040800040042D40009121400F902D400F344000FE
:104090009124400F902D400091214010902D400020
:1040A0009121400F902D40009121400F903440000D
:1040B00091284010902D4000912B400F902D4000F2
:1040C0009121400F902D40102D40009124400790E9
:1040D0002F40082D400091214007902F400832408A
:1040E0000091214008902F40073240009121400864
:1040F0009034400832400091284007903440083600
:104100004000912B400890344007344000912140FA
:104110003D90324000911F403E90314000911E4042
:104120003D90284000911C401E902B4000911F4064
:104130001F903440009121403D90324000911F403B
:104140003D90314000911E403D90284000911C4020
:104150001F902B4000911F401F9039400091264036
:104160003D903B40009128403D903E4000912B40C7
:104170003D90404000912D403D90394000912640B7
:104180003E903B40009128403D903E4000912B40A6
:104190003D90404000912D403D902D4000912140A8
:1041A0000F902D40103440009124400F902D40007E
:1041B0009121400F902D40009121400F902D400003
:1041C00091214010903440009128400F902D4000E4
:1041D000912B400F904240009121400490404004B8
:1041E0003E40043B40043B40033940043740043622
:1041F000400434400091244004903240042D400794
:1042000091214010214007902B40089121400F2818
:10421000400890374004394003374000912B400458
:10422000903240043440043240042D40009121403B
:104230000F902D400F34400091244010902D4000ED
:104240009121400F902D40009121400F902D400072
:104250009121400F9034400091284010902D400053
:10426000912B400F902D40009121400F902D401038
:104270002D400091244007902F40082D40009121AF
:104280004008902F400732400091214008902F4075
:10429000083240009121400790344008324000919C
:1042A00028400790344008364000912B4008903455
:1042B00040072D400091214010902D400F344000C8
:1042C0009124400F902D400091214010902D4000EE
:1042D0009121400F902D40009121400F90344000DB
:1042E0009128400F902D4000912B401090424000AB
:1042F00091214004904040033E40043B40043B4039
:1043000004394004374004364003344000912440CF
:1043100004903240042D40089121400F2140089024
:104320002B40079121401028400790374004394026
:1043300004374000912B4004903240033440043253
:1043400040042D40009121400F902D40103440003A
:104350009124400F902D40009121400F902D40005E
:1043600091214010902D40009121400F9034400049
:104370009128400F902D4000912B400F902D400030
:1043800091214010902D400F2D4000912440089025
:104390002F40072D400091214008902F40083240C7
:1043A0000091214007902F400832400091214008A1
:1043B000903440073240009128400890344007363E
:1043C0004000912B40089034400834400091214037
:1043D0003D90324000911F403D90314000911E4081
:1043E0003D90284000911C401F902B4000911F40A1
:1043F0001E903440009121403E90324000911F4079
:104400003D90314000911E403D90284000911C405D
:104410001F902B4000911F401E9039400091264074
:104420003D903B40009128403E903E4000912B4003
:104430003D90404000912D403D90394000912640F4
:104440003D903B40009128403D903E4000912B40E4
:104450003D90404000912D403E90434000912140CE
:104460001E904340009124400F2140109043400093
:104470009121400F21400F90404000912840102B87
:10448000400F903E40009124401E904040009128F3
:10449000401024400F904340009124400F244010CE
:1044A00090404000912B400F2F400F903E400091D4
:1044B00026401F90404000912A400F26400F904315
:1044C00040009126401026400F90404000912D4022
:1044D0000F304010903940009126403D9030400010
:1044E0009124401E902F40009123401F9043400094
:1044F0009121401F904840009124400F21400F908F
:104500004A40009121400F21401028400F2B400FBE
:10451000904A40009124401F904840009128400F4D
:1045200024400F904340009124401024400F9040BD
:104530004000912B400F2F4010903E4000912640AC
:104540001E903C4000912A400F26401090374000BA
:104550009126400F26400F90394000912D40103099
:10456000400F903940009126403D9030400091240A
:10457000401F902F40009123401E90454000912104
:1045800040059043400540400645400543400540F6
:1045900040054540009124400590434005404005BA
:1045A00045400091214005904340054040054A4068
:1045B0000091214006904840054540054A40009141
:1045C000214005904840054540054A40009128405B
:1045D00005904840054540054A4000912B40059014
:1045E000484006454005484000912440059045401C
:1045F0000543400548400545400543400548400007
:1046000091284005904540054340064840009124CC
:104610004005904540054340054A4000912440052F
:10462000904840054540054A400091244005904887
:1046300040054540054A4000912B40069048400502
:104640004540054A4000912F4005904840054540AF
:1046500005454000912640059043400540400545F2
:104660004005434005404006454000912A400590E2
:104670004340054040054540009126400590434099
:10468000054040054A4000912640059048400545B8
:1046900040054A40009126400690484005454005A7
:1046A0004A4000912D4005904840054540054A404C
:1046B0000091304005904840054540054840009134
:1046C00026400590454006434005484005454005C5
:1046D00043400548400545400543400548400545E1
:1046E00040054340064A400091244005904840055B
:1046F0004540054A40054840054540054A4000916F
:10470000234005904840054540054A40054840067D
:104710004540054540009121407AFF06014500FFD4
:104720002F0000B00758005C00000B7F0090244071
:1047300000FF06015300C00100B1077F005C0000CC
:104740000B7F00C10013902440009140400E902444
:104750004005244000914040099024400A24400034
:104760009143400A90244000914540099027400021
:104770009145400A902740092740009147400A9000
:1047800027400A914740099027400A274000914757
:104790004013902940009147400A90294009294040
:1047A0000A29401329400A29400929400A294000C2
:1047B0009145400943400A902940009140400A43F6
:1047C0004009902440132440009140400F90244021
:1047D00005244000914040099024400A2440009163
:1047E000434009902440009145400A9027400091A1
:1047F00045400A902740092740009147400A9027EA
:1048000040099147400A9027400A274000914740BD
:104810001390294000914740099029400A29400AF5
:1048200029401329400929400A29400A29400091BA
:1048300045400947400A90294000914A40094740B5
:104840000A902440132440009140400F90244004DB
:104850002440009140400A9024400A2440009143A3
:104860004009902440009145400A9027400091451E
:1048700040099027400A2740009147400A9027406E
:10488000099147400A90274009274000914740146A
:1048900090294000914740099029400A2940092960
:1048A000401429400929400A29400929400091451E
:1048B000400A43400A902940009140400943400A81
:1048C000902440132440009140400E902440052441
:1048D00040009140400A9024400924400091434008
:1048E0000A902440009145400A902740009145409D
:1048F000099027400A274000914740099027400A25
:104900009147400A90274009274000914740139063
:104910002940009147400A9029400A29400929402E
:104920001329400A29400A29400929401329401423
:10493000244000914F40044C400548400543400549
:1049400090244000914840054C40044F400590247D
:104950004000914C40059024400091484005434060
:104960000590244000914840044C400590244000AC
:10497000914F40054C40059024400091484005432C
:10498000400490274000915240054F400590274039
:1049900000914B400546400590274000914B400454
:1049A0004F400590274000915240054F40054B4035
:1049B0000546400490274000914B40054F4005902C
:1049C000274000915240054F40054B4004464005AA
:1049D0009029400091544005514005902940009194
:1049E0004D400548400490294000914D40055140FC
:1049F0000590294000915440055140054D40044820
:104A0000400590294000914D4005514005902940B6
:104A1000009154400551400490294000914D4005BB
:104A2000484005902940009154400A51400990297E
:104A30004000914D400A48400990244000914F4069
:104A4000054C4005484005434005902440009148EE
:104A500040044C40054F400590244000914C4005D7
:104A60009024400091484005434004902440009128
:104A70004840054C400590244000914F40054C4073
:104A80000590244000914840044340059027400091
:104A9000915240054F400590274000914B400546FC
:104AA000400490274000914B40054F40059027401F
:104AB00000915240054F40054B4004464005902769
:104AC0004000914B40054F400590274000915240D7
:104AD000054F40044B400546400590294000915445
:104AE000400551400590294000914D400448400543
:104AF00090294000914D400551400590294000917A
:104B00005440055140044D4005484005902940005F
:104B1000914D400551400590294000915440045169
:104B2000400590294000914D40054840059029409E
:104B3000009154400951400A90294000914C400A8C
:104B40004F400990244000914F40054C400548409B
:104B50000543400490244000914840054C40054FD7
:104B6000400590244000914C40059024400091481D
:104B7000400443400590244000914840054C4005C6
:104B800090244000914F40054C40049024400091F7
:104B900048400543400590274000915240054F4052
:104BA0000590274000914B40044640059027400067
:104BB000914B40054F400590274000915240054FD2
:104BC00040044B400546400590274000914B40056E
:104BD0004F400590274000915240044F40054B4004
:104BE00005464005902940009154400551400490ED
:104BF000294000914D400548400590294000914DC5
:104C00004005514005902940009154400451400511
:104C10004D400548400590294000914D40055140C8
:104C200004902940009154400551400590294000CE
:104C3000914D40054840059029400091544009514C
:104C4000400A90294000914D400948400A90244074
:104C500000914F40054C40054840044340059024D6
:104C60004000914840054C40054F400590244000CD
:104C7000914C4004902440009148400543400590E9
:104C8000244000914840054C400590244000914F3D
:104C900040044C40059024400091484005434005A5
:104CA00090274000915240054F40049027400091CA
:104CB0004B400546400590274000914B40054F4032
:104CC0000590274000915240044F40054B40054657
:104CD000400590274000914B40054F4004902740ED
:104CE00000915240054F40054B4005464005902934
:104CF00040009154400451400590294000914D409E
:104D00000548400590294000914D400551400490D0
:104D1000294000915440055140054D40054840054B
:104D200090294000914D4004514005902940009148
:104D300054400551400590294000914D40054840A0
:104D40000490294014294013FF06014500FF2F005D
:104D500000B0077F005C00000B7F00C000009037B0
:104D60005F00B1077F005C00000B7F00C10108906D
:104D7000375F08375F08395F083B5F11375F083CD2
:104D80005F11375F00911F5F0890435F00912B5FB9
:104D900021235F08235F08FF2F0000B00767005C36
:104DA00000000B7F00C0000090515F0A495F0A4C71
:104DB0005F0A515F0A485F0A4C5F0B515F0A475F09
:104DC0000A4A5F0A515F0A465F0B495F0A475F1E46
:104DD000FF2F0000B1077F005C00000B7F00C100C7
:104DE00000FF0601530091265F00B0077F005C00C2
:104DF000000B7F00C0001091265F08245F09265F2A
:104E000010265F08245F09265F10265F08295F15BA
:104E1000295F15265F10265F08245F09265F10268C
:104E20005F08245F09265F10265F082B5F152B5F44
:104E300015265F10265F08245F09265F10265F088D
:104E4000245F09265F10265F08295F15295F152654
:104E50005F10265F08245F09265F10265F08245F25
:104E600009265F10265F082B5F152B5F15265F1044
:104E7000265F08245F09265F10265F08245F092645
:104E80005F10265F08295F15295F15265F10265FD2
:104E900008245F09265F10265F08245F09265F103B
:104EA000265F082B5F2A245F08265F10225F0924F3
:104EB0005F10245F09265F18215F09225F08265FC3
:104EC00008245F08265F09245F08295F08265F3AE7
:104ED000245F08265F11225F082E5F10245F0930CF
:104EE0005F18215F09225F08265F08245F08265F9C
:104EF00009245F08295F08265F3A245F08265F11AE
:104F0000225F08245F10245F09265F18215F0922B1
:104F10005F08265F08245F08265F09245F08245F76
:104F200008295F08265F32245F08265F11225F0888
:104F30002E5F10245F09305F18215F09225F08226D
:104F40005F08245F08225F09245F08225F08295F49
:104F500008265F321F5F00903F5F0891215F00903D
:104F60003E5F083C5F0991245F00903B5F08912100
:104F70005F21215F0090415F0891235F00903F5FB8
:104F8000093E5F0891265F00903C5F0891235F21F6
:104F90001F5F0090435F0891215F0090415F093FD0
:104FA0005F0891245F00903E5F0891215F21215F9F
:104FB0000090445F0891235F0090435F09415F08C0
:104FC00091265F00903F5F0891235F21235F00904F
:104FD0003F5F0891245F00903E5F093C5F08912786
:104FE0005F00903B5F0891245F21245F0090415F48
:104FF0000891265F00903F5F093E5F0891295F009E
:10500000903C5F0891265F21235F0090435F0891E9
:10501000245F0090415F093F5F0891275F00903E49
:105020005F0891245F21245F0090465F0891265F0E
:105030000090445F09435F0891295F0090415F0839
:1050400091265F21245F08265F11225F08245F11EB
:10505000245F08265F19215F08225F08265F082465
:105060005F09265F08245F08295F08265F3A245FEE
:1050700008265F11225F082E5F11245F08305F1938
:10508000215F08225F08265F08245F09265F082445
:105090005F08295F08265F3A245F09265F10225FB8
:1050A00008245F11245F08265F19215F08225F082A
:1050B000265F09245F08265F08245F08245F09290A
:1050C0005F08265F31245F09265F10225F082E5F8C
:1050D00011245F08305F19215F08225F08225F09F1
:1050E000245F08225F08245F08225F09295F0826E1
:1050F0005F31245F09265F10225F08245F11245F5F
:1051000008265F0890325F42305F4291245F092693
:105110005F08245F10265F09295F08265F10902E24
:105120005F322B5F10305F4391245F08265F0826B3
:105130005F08265F09245F08295F08265F11903207
:105140005F312B5F11305F4291245F08265F102290
:105150005F092E5F10245F08305F0990305F312BAC
:105160005F11355F10325F32FF06014500FF2F00EF
:105170000D1EC8D716E7F432000000000000103200
:10518000C87D0DD41FF30000000000001316DC02E0
:10519000CB7DEBFEF0E9000000001400CD7B7AEB44
:1051A0009A992900000000000C20FCEACDDEFA1FCD
:1051B0000000000000001D15DC010272E1E99B2BDC
:1051C0008EFAE8001514C829850C05E0F5FD0000ED
:1051D0000000112B917201DCE83200000000000099
:1051E0001C167BCC7DEB9AE9988C796F0000163207
:1051F000FCEAFF7CCDDF0BC81F000000555A45427A
:105200004F5800434F5252494441204E45424F535C
:105210004F53410050524553532053544152540070
:10522000284329203230313020464CC38156494F23
:10523000205A4156414E0028432920323032322034
:10524000444F4D494E494B204B52495354454E0013
:1052500031003200504C41594552530053494E479A
:105260004C452052414345004348414D50494F4E23
:1052700053484950004F5054494F4E5300545241E7
:10528000434B20454449544F520044494646494304
:10529000554C54593A0045415359004D45444955E0
:1052A0004D004841524400434F4C4C4953494F4EE6
:1052B000533A004E4954524F3A004F4E004F464623
:1052C000004D555349433A005346583A004C41501B
:1052D0005320534149534F4E3A00524143452053C6
:1052E0004149534F4E3A00454550524F4D20434C93
:1052F0004541524544005449454420200046495206
:10530000535420005345434F4E440057494E4E4599
:1053100052004C4F53455220004C3A203A004E3A2E
:1053200020202025005041555345440052455355F7
:105330004D4500515549540044454D4F0053454C8F
:10534000205245564552534500545241434B004369
:105350005553544F4D004C41505300545241434B10
:1053600020534156454420494E20534C4F54004E43
:105370004F204652454520534C4F54530052455000
:105380004C41434520435553544F4D2054524143C3
:105390004B0043414E43454C005341564500545247
:1053A00041434B20434F4D504C45544544005245DA
:1053B000443A0059454C4C4F573A00504F494E54CF
:1053C000532041465445522052414345202020203D
:1053D0004F46203130003A3A3A454E44204F46205D
:1053E000534149534F4E3A3A3A00524143452057B0
:1053F0004F4E00504F494E5453005245442049539C
:10540000204348414D50494F4E0059454C4C4F5751
:10541000204953204348414D50494F4E000011242C
:105420001FBECFEFD0E1DEBFCDBF12E0A0E0B1E004
:10543000E6EDF2EE02C005900D92A431B107D9F766
:105440001AE0A0E2B2E001C01D92AD3FB107E1F762
:1054500014BE88E10FB6F89480936000109260004B
:105460000FBEF89426EB30E0F90185919491FC0190
:10547000F07090832E5F3F4F80E0283E3807A1F701
:105480000E943835882311F40E949035E1ECF7E052
:1054900080E8819399E0ED3CF907D9F781EC97E03A
:1054A0009093CE098093CD091092CF0991E090930B
:1054B000E6099093E7099093E5091092D2091092BA
:1054C000D8091092DE091092E4091092A2071092F6
:1054D000A40782E18093A30780EE8093AA0784E16A
:1054E0008093A9071092AE071092AD071092B207F1
:1054F0001092B1079093D1090E94014078940E94C4
:1055000000400E94506F0C9469710C94000003E8F5
:105510000A95F1F700C000919107E8E7F7E023E072
:10552000029FE00DF11D209190073CE3321B300FEC
:10553000201751F000000000A191B1911C9111932E
:105540000C9303950217C0F313E01A95F1F700C00E
:105550003A95D1F7C0E2D2E0662717E01A95F1F745
:1055600000C040919F075091A00760909B077090EA
:105570009C07D3015E01762F00C030919E0730302A
:1055800009F0C8E609F0D5E009F0DA0115E01A954E
:10559000F1F78090AA0707E00093360001E000933E
:1055A000810001E000936F0008E0609F8D010050D2
:1055B0001240000D111D180108E715E0000D111D26
:1055C000280100E4E02E03E31AEFCF93DF93599113
:1055D00000C000C01FD32EE12A95F1F7109385007B
:1055E00000938400789400275E9D5830F10108F400
:1055F000F201001FE00DF11D1AE01A95F1F700000D
:10560000112700FF02C0000065C048C018B90F9004
:105610000F90DF91CF9103E00A95F1F700C06395F9
:105620008A94B1F0683029F007E00A95F1F700C0DC
:10563000BBCF66276E960491049100C03A9509F499
:10564000672F09F4E50100C000C009F4D301ACCF15
:1056500020E12A95F1F700E0009385000CE2009329
:105660008400D8D211240E94AF2CE091A40742E01C
:10567000E160E427E093A40707E00093360009E027
:105680000093810002E000936F000895059108B92E
:10569000020C0000059108B9131CF001059108B92E
:1056A00000C0059108B94991059108B900C005915C
:1056B00008B94E9D059108B948300000059108B918
:1056C00028F70000059108B9040C0000059108B9FD
:1056D000151CF0010000019108B9499100000191E9
:1056E00008B900004E9D019108B90491019108B9D3
:1056F0000491019108B9483000C0019108B950F4F3
:105700000000040C019108B9151C00000191F00182
:1057100008B9E0CF020C019108B9131C00000191F7
:10572000F00108B9BBCF20E4E0919B07F0919C0702
:10573000829FE00DF11DA8E7B5E0629FA00DB11DAD
:1057400015901D9215901D9215901D9215901D9209
:1057500015901D9215901D9215901D9215901D92F9
:1057600015901D9215901D9215901D9215901D92E9
:1057700015901D9215901D9215901D9215901D92D9
:1057800015901D9215901D9215901D9215901D92C9
:1057900015901D9215901D9215901D9215901D92B9
:1057A00015901D9215901D9215901D9215901D92A9
:1057B00015901D9215901D9215901D9215901D9299
:1057C00015901D9215901D9215901D9215901D9289
:1057D00015901D9215901D9215901D9215901D9279
:1057E00015901D9215901D9215901D9215901D9269
:1057F00015901D9215901D9215901D9215901D9259
:1058000015901D9215901D9215901D9215901D9248
:1058100015901D9215901D9215901D9215901D9238
:1058200015901D9215901D9215901D9215901D9228
:1058300015901D9215901D9215901D9215901D9218
:105840001124089520E4E8E7F5E0829FE00DF11DC2
:10585000A8E7B5E0629FA00DB11D11901D921190B7
:105860001D9211901D9211901D9211901D921190F8
:105870001D9211901D9211901D9211901D921190E8
:105880001D9211901D9211901D9211901D921190D8
:105890001D9211901D9211901D9211901D921190C8
:1058A0001D9211901D9211901D9211901D921190B8
:1058B0001D9211901D9211901D9211901D921190A8
:1058C0001D9211901D9211901D9211901D92119098
:1058D0001D9211901D9211901D9211901D92119088
:1058E0001D9211901D9211901D9211901D92119078
:1058F0001D9211901D9211901D9211901D92119068
:105900001D9211901D9211901D9211901D92119057
:105910001D9211901D9211901D9211901D92119047
:105920001D9211901D9211901D9211901D92119037
:105930001D9211901D9211901D9211901D92119027
:105940001D9211901D9211901D9211901D92119017
:105950001D9211901D9211901D9211240895E091B5
:1059600091078E2FEE0FE80FFF27E858F84F0090B1
:105970009007801930F4A191B19101900C92839518
:10598000D1F7089598E0799FA12DBB27AD56B84F68
:10599000ED91FD9190E4699FE00DF11D899FD0018B
:1059A000A858BA4F90E040FD09C0822F48E0421B42
:1059B00070FF0AC01796E80FF91F08C088E0821B25
:1059C000422F70FFF8CF1197A20FB91F68E028E0AF
:1059D000231B50FD09C0639FA00DB11D71FDE85C44
:1059E00071FDFF4F122E08C0132E1A9471FF122E54
:1059F000619DE00DF11D132E71FD409770FD05C0F6
:105A000057EF540F70E061E004C059EF541B7FEF73
:105A10006FEF3EEF042E469530F461F0259123138D
:105A20002C93A60FB71F259123132C93A60FB71FF6
:105A30004150A1F7259123132C931A9449F0E80FB4
:105A4000F91FA51BBF4F402D469568F739F7F2CFD8
:105A500008950F921F92EF93FF93FFB7E091840098
:105A6000FF93E2FD04C0E1FD02C0000000C0E0FFC2
:105A700000C0E091A307EA95E093A307F091A20785
:105A8000F0FD51C0EC3098F0F3E0F0938900FDE8B0
:105A9000F0938800E0FB289826F4E1E00E94E32ED2
:105AA000B2C0E5E1EA95F1F70000289AACC0E63013
:105AB00008F100C000C02898E0FBE4E016F40E9462
:105AC000E32EE4E0E0933600E6E0E0936F009BC055
:105AD000EF93E0918400E2FD04C0E1FD02C000000C
:105AE00000C0E0FF00C0E2E00000289AE0936F00F1
:105AF000EF91189500C0E0FB289826F4E1E00E94A1
:105B0000E32E05C0E5E1EA95F1F70000289AE0915F
:105B1000A307E03009F077C0EDEFE093A307E1E0E1
:105B2000E093A20770C0E7E0E0938900EBE1E09327
:105B3000880000C02898E2E000C00E94E32EFDEF3C
:105B40000090A907F019E091A307EF17D8F4FDEF33
:105B50000090A907F0190090AA07F019EF1790F02C
:105B6000EDE1FF2700800F92EA95E1F70FE10A953A
:105B7000F1F700C00E94872AE1E0FF270F90019211
:105B8000EE31E0F3E091A307E03009F03CC02F9341
:105B90003F934F935F936F937F938F939F93AF93B5
:105BA000BF9378941124EE27E093A207E2E1E093FB
:105BB000A3078091B3079091B40701968093B30730
:105BC0009093B407E091A507F091A607E115F105C0
:105BD00009F009950E94EA350E948B410E94152E1A
:105BE0001124E091A707F091A807E115F10509F04C
:105BF0000995BF91AF919F918F917F916F915F9127
:105C00004F913F912F91EF91EFBFFF91EF911F9037
:105C10000F9018952898E2E000C00E94E32EE091D2
:105C2000A307EA95E093A3070895E091D109E0FD69
:105C30000E94B7370090CF09002019F4A1ECB7E01B
:105C400002C0A7ECB8E021E002260092CF0922E0D2
:105C50002093D009E091D109E0FF08952F923F925F
:105C60004F925F926F927F928F929F92AF92BF926C
:105C7000CF92DF92EF92FF920F931F93CF93DF9318
:105C80005091E4096091E6097091E7098091E80973
:105C90002090D3093090D4094090D6095090D7096C
:105CA0006090D5091091D2097090D9098090DA09D5
:105CB0009090DB09A090DC09B090DD092091D80913
:105CC000C090DF09D090E009E090E209F090E3098C
:105CD0000091E1093091DE099FEF620C431CF20153
:105CE000449141030008C12DD02D970CA81CF5014B
:105CF000449142030008C10DD01D8A956AF4409179
:105D0000E509842F8695062E0694062600FA7695D8
:105D1000679576F940FF66F940E860FD4FE7450377
:105D20000008C10DD01D0024C038D0050CF0CFE70D
:105D30000A94C038D0050CF4C0E8C058CD939A95A9
:105D400009F0CBCF4091D0094A954093D00997E014
:105D500009F0C3CF6092D5094092D6099092DB0931
:105D6000A092DC090093E109E092E2096093E60960
:105D70007093E7098093E809DF91CF911F910F910C
:105D8000FF90EF90DF90CF90BF90AF909F908F905B
:105D90007F906F905F904F903F902F900895E0918B
:105DA000CD09F091CE09019100000093B30009E004
:105DB000ED3CF00701EC17E008F0F801E093CD09A5
:105DC000F093CE0908950F931F932F93EF93E091D3
:105DD000CD09F091CE0901910093B30009E0ED3CAB
:105DE000F00701EC17E008F0F801E093CD09F0931B
:105DF000CE09E8E0EA95F1F7EF912F911F910F910D
:105E0000E0FD289AE0FF01C00895F4E1FA95F1F76A
:105E100000C0E1FD289AE1FF00C00895EF92FF92D3
:105E20000F931F937B018C0120E030E040E05FE4A2
:105E30000E94903188238CF0C801B70120E030E047
:105E400040E05FE40E9486300E941E329B01AC015C
:105E5000205030404040504806C0C801B7010E9461
:105E60001E329B01AC01B901CA011F910F91FF9035
:105E7000EF900895A0E0B0E0E0E4FFE20C944F70F2
:105E8000DC012B01FA019C91923008F439C1EB013D
:105E90008881823008F433C1943069F4843009F089
:105EA0002FC111969C9111978981981709F428C1E7
:105EB000A8E0B1E025C1843009F421C18230A9F401
:105EC000923009F01DC19A01AD0188E0EA01099004
:105ED000AE01E90109929E018150C1F7E201898179
:105EE00011969C918923818308C1923009F407C1DE
:105EF00012962D903C901397EB018A819B8114960A
:105F0000AD90BD90CD90DC901797EC80FD800E8118
:105F10001F819101281B390BB90137FF04C0662787
:105F20007727621B730B603271050CF061C012168B
:105F300013066CF537014801062E04C09694879429
:105F4000779467940A94D2F721E030E040E050E083
:105F500004C0220F331F441F551F6A95D2F72150EA
:105F60003040404050402E213F21402351232115F5
:105F700031054105510521F021E030E040E050E0DD
:105F800079018A01E628F728082919293CC0232B22
:105F9000D1F1260E371E35014601062E04C0969417
:105FA0008794779467940A94D2F721E030E040E038
:105FB00050E004C0220F331F441F551F6A95D2F7CB
:105FC00021503040404050402A213B214C215D214E
:105FD000211531054105510521F021E030E040E077
:105FE00050E059016A01A628B728C828D9280BC053
:105FF000821593052CF01C01AA24BB24650103C063
:10600000EE24FF24870111969C91D20111968C9168
:10601000981709F445C0992339F0A80197012A1966
:106020003B094C095D0906C0A60195012E193F09DF
:10603000400B510B57FD08C011823382228224830A
:106040003583468357831DC081E08183338222825A
:1060500088279927DC01821B930BA40BB50B848343
:106060009583A683B7830DC0220F331F441F551F8E
:106070002483358346835783828193810197938359
:1060800082832481358146815781DA01C9010197D4
:10609000A109B1098F5F9F4FAF4FBF4328F30BC0DA
:1060A000918333822282EA0CFB1C0C1D1D1DE482AD
:1060B000F5820683178383E08083248135814681BE
:1060C000578157FF1AC0C901AA2797FDA095BA2F7B
:1060D00081709070A070B070569547953795279550
:1060E000822B932BA42BB52B84839583A683B78314
:1060F00082819381019693838283DF0101C0D20163
:10610000CD01CDB7DEB7E2E10C946B70A0E2B0E058
:10611000ECE8F0E30C945B7069837A838B839C8357
:106120002D833E834F835887E9E0EE2EF12CEC0E51
:10613000FD1ECE010196B7010E9496338E010F5EBF
:106140001F4FCE010596B8010E9496338A8991E0CF
:1061500089278A8BC701B801AE01475E5F4F0E9455
:106160003A2F0E94C132A096E6E00C947770A0E22C
:10617000B0E0EDEBF0E30C945B7069837A838B8382
:106180009C832D833E834F835887F9E0EF2EF12CBB
:10619000EC0EFD1ECE010196B7010E9496338E01D2
:1061A0000F5E1F4FCE010596B8010E949633C701BE
:1061B000B801AE01475E5F4F0E943A2F0E94C13284
:1061C000A096E6E00C947770A8E1B0E0EAEEF0E388
:1061D0000C94577069837A838B839C832D833E83D1
:1061E0004F835887B9E0EB2EF12CEC0EFD1ECE014B
:1061F0000196B7010E9496338E010F5E1F4FCE01AC
:106200000596B8010E9496332985223008F47EC095
:106210003989323010F4B8017CC08A859A8989277F
:106220008A87243011F0223031F4231709F06EC030
:1062300068E071E06EC0343039F41D861E861F861A
:10624000188A1C861B8604C0323021F484E08987BA
:10625000B7015FC02B853C858B899C89281B390B36
:106260003C872B87ED84FE840F851889AD88BE8816
:10627000CF88D88CEA14FB040C051D0540F4EE0C05
:10628000FF1C001F111F215030403C872B8720E04E
:1062900030E040E050E080E090E0A0E0B0E460E07A
:1062A00070E0EA14FB040C051D0540F0282B392B87
:1062B0004A2B5B2BEA18FB080C091D09B695A7951C
:1062C00097958795EE0CFF1C001F111F6F5F7F4F86
:1062D0006F31710531F7DA01C9018F779070A070C5
:1062E000B07080349105A105B10561F427FD0AC0A5
:1062F000E114F1040105110529F0205C3F4F4F4FD7
:106300005F4F20782D873E874F87588BBE01675F90
:106310007F4FCB010E94C1326896EAE00C94737003
:10632000A8E1B0E0E6E9F1E30C945B7069837A835D
:106330008B839C832D833E834F83588789E0E82E8F
:10634000F12CEC0EFD1ECE010196B7010E94963392
:106350008E010F5E1F4FCE010596B8010E94963345
:106360008985823040F08989823028F0C701B801E0
:106370000E940E3401C08FEF6896E6E00C947770AF
:10638000A8E0B0E0E6ECF1E30C9458709B01AC019E
:1063900083E08983DA01C9018827B7FD83959927AE
:1063A000AA27BB27B82E211531054105510519F43F
:1063B00082E089833AC08823A9F0203080E0380742
:1063C00080E0480780E8580729F460E070E080E04A
:1063D0009FEC30C0EE24FF248701E21AF30A040B7D
:1063E000150B02C079018A018EE1C82ED12CDC8206
:1063F000CB82ED82FE820F831887C801B7010E940D
:10640000723201971816190684F4082E04C0EE0C97
:10641000FF1C001F111F0A94D2F7ED82FE820F832A
:106420001887C81AD90ADC82CB82BA82CE010196BB
:106430000E94C1322896E9E00C947470ACE0B0E0A0
:10644000E4E2F2E30C945F7069837A838B839C832C
:10645000CE010196BE016B5F7F4F0E9496338D8106
:10646000823061F1823050F1843021F48E818823B2
:1064700051F12EC02F81388537FD20C06E812F311C
:1064800031051CF06623F9F023C08EE190E0821BF9
:10649000930B29853A854B855C8504C056954795B5
:1064A000379527958A95D2F76623B1F05095409598
:1064B000309521953F4F4F4F5F4F0EC020E030E0A9
:1064C00040E050E009C02FEF3FEF4FEF5FE704C01F
:1064D00020E030E040E050E8B901CA012C96E2E04B
:1064E0000C947B70EF92FF920F931F937B018C01B2
:1064F00080E0E81680E0F80681E0080780E01807F1
:1065000088F48FEFE816F1040105110531F028F049
:1065100088E090E0A0E0B0E017C080E090E0A0E06C
:10652000B0E012C080E0E81680E0F80680E00807DE
:1065300081E0180728F088E190E0A0E0B0E004C016
:1065400080E190E0A0E0B0E020E230E040E050E008
:10655000281B390B4A0B5B0B04C016950795F79463
:10656000E7948A95D2F7F701E05FFE4F8081281B00
:10657000310941095109C9011F910F91FF90EF9015
:106580000895DF92EF92FF920F931F93FC01E48036
:10659000F58006811781D1808081823048F480E0C7
:1065A00090E0A0E1B0E0E82AF92A0A2B1B2BA5C055
:1065B000843009F49FC0823021F4EE24FF24870147
:1065C00005C0E114F1040105110519F4E0E0F0E063
:1065D00096C0628173819FEF623879070CF05BC0CF
:1065E00022E83FEF261B370B2A3131052CF020E043
:1065F00030E040E050E02AC0B801A701022E04C0FC
:1066000076956795579547950A94D2F781E090E083
:10661000A0E0B0E004C0880F991FAA1FBB1F2A95F5
:10662000D2F70197A109B1098E219F21A023B1239F
:106630000097A105B10521F081E090E0A0E0B0E075
:106640009A01AB01282B392B4A2B5B2BDA01C901AC
:106650008F779070A070B07080349105A105B1055E
:1066600039F427FF09C0205C3F4F4F4F5F4F04C0F4
:10667000215C3F4F4F4F5F4FE0E0F0E02030A0E063
:106680003A07A0E04A07A0E45A0710F0E1E0F0E082
:1066900079018A0127C06038710564F5FB01E15872
:1066A000FF4FD801C7018F779070A070B070803411
:1066B0009105A105B10539F4E7FE0DC080E490E035
:1066C000A0E0B0E004C08FE390E0A0E0B0E0E80E0E
:1066D000F91E0A1F1B1F17FF05C016950795F79493
:1066E000E794319687E016950795F794E7948A9595
:1066F000D1F705C0EE24FF248701EFEFF0E06E2F05
:10670000679566276795902F9F77D794DD24D79458
:106710008E2F8695492F462B582F5D29B701CA0128
:106720001F910F91FF90EF90DF900895FC01DB0126
:10673000408151812281622F6F7770E0221F2227D2
:10674000221F9381892F880F822B282F30E0991FD9
:106750009927991F11969C93119721153105A9F539
:10676000411551056105710511F482E037C082E8D9
:106770009FEF13969C938E9312979A01AB0167E05B
:10678000220F331F441F551F6A95D1F783E08C9366
:106790000DC0220F331F441F551F12968D919C91DF
:1067A0001397019713969C938E931297203080E055
:1067B000380780E0480780E4580758F314962D9373
:1067C0003D934D935C93179708952F3F310579F4CE
:1067D000411551056105710519F484E08C93089504
:1067E00064FF03C081E08C9312C01C9210C02F572D
:1067F000304013963C932E93129783E08C9387E05E
:10680000440F551F661F771F8A95D1F77064149641
:106810004D935D936D937C93179708951F93DC01BF
:10682000FB019C91923008F447C08081823008F4CB
:1068300043C0943051F411961C91843099F58181B4
:10684000682F70E0611B71093FC0843021F09230E5
:1068500031F48230B9F18181882389F12DC01196FC
:106860001C9111978230F1F081811817D9F412969A
:106870002D913C911397828193818217930794F015
:1068800028173907BCF014968D919D910D90BC91FD
:10689000A02D2481358146815781281739074A0761
:1068A0005B0718F4112341F00AC082179307A4076D
:1068B000B50740F4112319F061E070E005C06FEFF7
:1068C0007FEF02C060E070E0CB011F9108958093DC
:1068D0009307909394070895E8E4F3E0A0E2B2E010
:1068E00068E06D933197E9F71124089550919D0761
:1068F000450F00C0992777272EE1629F080E191EC9
:10690000A0E2B2E0A00DB11D485F4C9311240895A0
:1069100080939D07089580939B0790939C0708950B
:106920008091A407817008952091A4072E7F209361
:10693000A4070895882329F48091AB079091AC07B0
:1069400008958091AF079091B0070895E0E6F0E0D8
:10695000808183FD089588E198E0F8948083908396
:106960007894FFCFF999FECF92BD81BD60BDF894B8
:10697000FA9AF99A78940895F999FECF92BD81BD5B
:10698000F894F89A80B578940895A0E0B0E0EBEC24
:10699000F4E30C9453703C014B015A01FB0111824A
:1069A0001082FFEF8F3F9F0711F481E02EC0DD249E
:1069B000F3E0CF2E00E0EE24FF24C7010E94BC3498
:1069C000182FC70101960E94BC34D82FC0E0CE0119
:1069D000810F911D8615970529F4F401F182E0825B
:1069E000CC240BC08F5F9F4F41F4DD2031F4A11404
:1069F000B10411F0F5010083D02E0F5F80E290E02A
:106A0000E80EF91E0034C9F68C2DCDB7DEB7EEE0E6
:106A10000C946F70A2E0B0E0E0E1F5E30C945A70E2
:106A2000162F072FBE016F5F7F4F40E050E00E949E
:106A3000C534D82E8823B9F4812F902F9C01890169
:106A4000A0E2EA2EF12CE20EF31E89819A810196D2
:106A50009A83898301970E94BC34F80181938F0146
:106A6000EE15FF0591F78D2D2296E7E00C947670D8
:106A70001F9380E090E00E94BC34182F81E090E0EA
:106A80000E94BC3490E0382F20E0210F311D2A55A0
:106A9000354509F491E0892F1F910895A3E0B0E0F6
:106AA000E4E5F5E30C945B708C011B821A82198279
:106AB000FC0180819181BE016E5F7F4FAE014F5F0F
:106AC0005F4F0E94C534882311F0833029F58A81F5
:106AD0009B81892B69F48981882311F482E01CC091
:106AE00090E025E0880F991F2A95E1F79B838A8320
:106AF000B0E2EB2EF12CE00EF11E8A819B81019613
:106B00009B838A830197F80161918F010E94B234BF
:106B10000E151F0591F780E02396E6E00C94777040
:106B2000CF93DF93C0E0D0E0FE01EA56FF4FE4913F
:106B3000CE016E2F0E94B2342196C032D105A1F74A
:106B4000C0E2D0E0CE016FEF0E94B234CE010196D8
:106B50006FEF0E94B234A09688E0C030D80791F75A
:106B6000DF91CF910895129AC895C895C895C89598
:106B7000129820E030E080E090E040E036952795E4
:106B800096958795C895C895C895C8951398009B04
:106B90003068019B9068139AC895C895C895C895A8
:106BA0004F5F403159F73093AC072093AB07909378
:106BB000B0078093AF078091AB079091AC070F9718
:106BC00031F08091AF079091B0070F9711F40E94B8
:106BD000A63408951092060A009903C081E08093BC
:106BE000060A019905C08091060A82608093060A10
:106BF0000E94B3350895FC016787089581E091E014
:106C00009093E7098093E6096093E5090895FC01F4
:106C100080818F7580830895FC01808180648083EA
:106C20000895FC0166870895FC0162870895FC01C0
:106C300063870895CF93DF93EC01462F898190E01D
:106C4000FC01EE0FFF1FEA55FB4825913491E62F1A
:106C5000FF27E7FDF095E80FF91FEE0FFF1FEA553C
:106C6000FB48859194916885821B930B70E00E948C
:106C7000FF6F9B016115710511F421E030E08A81FD
:106C800090E0FC01EE0FFF1FE80FF91FEE0FFF1F52
:106C9000EE52F64F81819281820F931F92838183FE
:106CA0003E832D838881886088838981840F8F83C8
:106CB000DF91CF910895FC0160870895FC01648302
:106CC0000895DC0114968C911497882331F1559620
:106CD000ED91FC915697662371F0262F332727FDFF
:106CE000309520953095C901880F991F820F931F09
:106CF000E80FF91F08C033973297849132968D3090
:106D000011F08F3FC1F75696FC93EE93559714966A
:106D10008C911497815014968C9308959093680ADF
:106D20008093670A8FE680936A0A1092C007E9E0B1
:106D3000FAE080E090E13FEF28E1828390831586BE
:106D40003487108A238790878F5F77968430A9F7DE
:106D500008952091090A2F772093090A3FEF309375
:106D60000C0A2091200A2F772093200A3093230ABF
:106D70002091370A2F772093370A30933A0A2091CF
:106D80004E0A2F7720934E0A3093510A0196909322
:106D90006F0A80936E0A9093080A8093070A909373
:106DA000710A8093700A10926C0A10926B0A10920A
:106DB000660A1092650A10926D0A1092690A81E0C3
:106DC0008093C00708958AEF8093180A80932F0A52
:106DD0008093460A80935D0A1092C007089581E06F
:106DE0008093C0070895DC01ED91FC911197AF01EC
:106DF0004F5F5F4F11965C934E93E4912E2F30E0DE
:106E0000E7FF13C02F7730703695322F2227379542
:106E10002795FA014F5F5F4FE4918E2F8F77280FF0
:106E2000311DE7FDF1CF4D935C93C9010895809327
:106E30006A0A0895FF920F931F938C01F62EFC01AE
:106E400082810E941F3AF801F1828081877F8083CE
:106E50001F910F91FF900895FC01862F6181681B9F
:106E6000618382810E941F3A0895FC018181680F2D
:106E7000618382810E941F3A08950F931F93CF93DD
:106E8000DF93EC01062F10E0888187FD11E01F865B
:106E90009FEF9E874D871C8A8881877B88831A860F
:106EA000198629831C829B838A81833069F411238C
:106EB00009F4022F81E091E09093E7098093E609BD
:106EC00081E08093E50907C0622F0E941F3A8A8102
:106ED00060E00E94363A112311F0098B01C0088B43
:106EE00089E0089FC0011124E091670AF091680AC7
:106EF000E80FF91F3396259134912115310519F4C6
:106F00001E8A1D8A08C01B8AF90184918A8B2F5F13
:106F10003F4F3E8B2D8BDF91CF911F910F910895A5
:106F2000CF93DF93342F97E1899FE0011124C75F4E
:106F3000D54F8881982F85FF02C087FD15C0222379
:106F400041F48F85882311F496FF1D8688818F7BFD
:106F50000AC018821E8A1D8ACE01422F232F0E944A
:106F60003D37888180628883DF91CF910895A0E0CA
:106F7000B0E0EDEBF7E30C945970A9E0BAE0C3ED93
:106F8000D9E01F968C911F978823B9F0282F3327BB
:106F900027FD30951E968C911E97280F311D2F3F8F
:106FA000310519F014F02FEF30E0C90137FF02C0AE
:106FB00080E090E01E968C931E978C9183FF26C0F4
:106FC00015964D915C91169728813981240F351FB4
:106FD0003983288317968C911797E82FF0E0EE0FEE
:106FE000FF1FEA55FB48859194911416150624F469
:106FF0002817390730F40AC0452B41F08217930750
:1070000028F0998388838C91877F8C935796269656
:107010004AE0A536B40709F0B4CF8091C0078823B1
:1070200009F0DEC0F1C0E0916E0AF0916F0ACF0165
:10703000019690936F0A80936E0A44914F3F69F5D1
:10704000AC014F5F5F4F50936F0A40936E0AFC0193
:1070500084918F3219F41092C007D0C0863009F0A5
:10706000B2C0FA013196CF01019690936F0A8093D6
:107070006E0AE491E33529F49093710A8093700AC3
:10708000A2C0E53409F09FC08091700A9091710A06
:1070900090936F0A80936E0A96C047FF02C0409398
:1070A000690A2091690A322F3F7047FF08C0019694
:1070B00090936F0A80936E0A0197FC014491822F8E
:1070C00090E0807F9070803B910531F1803C91058C
:1070D00009F46DC08039910509F075C0E0916E0A20
:1070E000F0916F0A3196F0936F0AE0936E0A319730
:1070F000E491832F90E08C9FD0018D9FB00D9C9FD9
:10710000B00D1124A75FB54FEE0F832F50966C91F1
:107110002E2F0E94903757C0E0916E0AF0916F0AAF
:107120003196F0936F0AE0936E0A319724914730BD
:1071300071F4832F90E08C9FF0018D9FF00D9C9F48
:10714000F00D1124E75FF54F220F24873CC04B3030
:1071500071F4832F90E08C9FF0018D9FF00D9C9F28
:10716000F00D1124E75FF54F220F23832CC04C351F
:1071700071F4832F90E08C9FF0018D9FF00D9C9F08
:10718000F00D1124E75FF54F220F22871CC0443613
:10719000D1F4832F90E08C9FF0018D9FF00D9C9F88
:1071A000F00D1124E75FF54F220F23870CC0832FCA
:1071B00090E08C9FF0018D9FF00D9C9FF00D1124AD
:1071C000E75FF54F408B8EE69AE00E94F33690938E
:1071D0006C0A80936B0A1092660A1092650A02C0CC
:1071E000C7E1D0E02091650A3091660A80916B0A70
:1071F00090916C0A2817390709F415CF2F5F3F4F7C
:107200003093660A2093650AC9E0DAE002ED19E0DE
:107210005FEFC52ED12C7E018881282F85FF39C0D4
:107220008D899E89892B09F434C026FF2BC031C07B
:10723000ED89FE89CF0101969E8B8D8B24912F3F86
:1072400031F488818F7788831E8A1D8A1FC001963A
:107250009E8B8D8B0197FC016491822F90E0880FAB
:10726000991F88519F4FFC0125913491C701F90165
:107270000995ED89FE893196FE8BED8B3197E4916E
:10728000EA8B1B8A9B898A89981791F28B898F5F79
:107290008B8B888185FD03C020E030E070C08C8935
:1072A0008F3F11F08F5F8C8B888187FF02C08FEF3B
:1072B00001C08C859D85992309F45BC02E8522230E
:1072C00009F457C0882309F454C040916A0A442342
:1072D00009F44FC0899FC001112480509F4F892F0E
:1072E000992730E0B901869F9001879F300D969FC6
:1072F000300D112420503F4F232F33278B8190E0F6
:10730000FC012E9FC0012F9F900D3E9F900D1124D8
:1073100080509F4F892F9927242F30E0AC01429F46
:10732000C001439F900D529F900D112480509F4F9C
:10733000292F33278A858823F1F0E985F0E0E05092
:10734000FA48E491E058E89FC001112480509F4F13
:10735000892F9927B601681B790B629FC001639F33
:10736000900D729F900D112480509F4F292F33272D
:1073700002C020E030E089859B85890F8987F8016C
:10738000208367960A5F1F4FFAE0C536DF0709F0D2
:1073900042CFCDB7DEB7E8E00C9475700F931F9322
:1073A000282F362F89E0289FC0011124E091670A19
:1073B000F091680AE80FF91F8491813011F483E09D
:1073C00021C0823011F484E01DC08091200A87FF23
:1073D00016C08091310A821711F4442381F4809100
:1073E000370A87FF0EC08091480A821711F44423A0
:1073F00041F49091340A80914B0A891710F481E08E
:1074000001C082E007E1809F80011124075F154FD2
:1074100080E8F8018083168A158AC801622F432FFD
:1074200020E50E943D37F8018081806280831F91B2
:107430000F910895FC0182810E94363A08959927A0
:107440007727833008F00895E6EAF4E7660F771FA0
:10745000E60FF71FA591B491E2EDF9E026E0289F31
:10746000E00DF11DA183B283112408959927772798
:10747000E2EDF9E026E0289FE00DF11D6E3F31F4CA
:107480006091E5096E7F6093E5090BC06F3F31F4B1
:107490006091E5096E6F6093E50903C076E7760FAA
:1074A00075831124089522002400260028002B0053
:1074B0002D0030003300360039003D00400044000C
:1074C00048004C00510056005B00600066006C00F4
:1074D000730079008100880090009900A200AC0040
:1074E000B600C100CC00D800E500F3000101100196
:1074F00021013201440157016C0181019801B00161
:10750000CA01E50102022102410264028802AE02C0
:10751000D7020303300361039403CB030504420441
:107520008304C70410055D05AF0505066106C206A4
:10753000290796070908830805098E09200ABA0A4F
:107540005D0B0A0CC10C840D510E2B0F121007118C
:107550000A121D1340147415BA1614188319071B48
:10756000A31C571E24200E22142439267F28E82A23
:10757000752D293006330F364539AD3C49401B4443
:107580002848734CFE50CF55EA5A51600C661D6C6A
:107590008B725A79928037885090E598FDA19FAB05
:1075A000D3B5A3C0000000000000000000000000F0
:1075B00000000000000000000000000000000000CB
:1075C00000000000000000000000000000000000BB
:1075D00000000000000000000000000000000000AB
:1075E000000000000000000000000000000000009B
:1075F000000000000000000000000000000000008B
:10760000000306090C101316191C1F2225282B2E07
:10761000313336393C3F414447494C4E515355581C
:107620005A5C5E60626466686A6B6D6F70717374D9
:10763000757678797A7A7B7C7D7D7E7E7E7F7F7F92
:107640007F7F7F7F7E7E7E7D7D7C7B7A7A79787678
:1076500075747371706F6D6B6A68666462605E5C8E
:107660005A585553514E4C494744413F3C393633A3
:10767000312E2B2825221F1C191613100C09060366
:1076800000FDFAF7F4F0EDEAE7E4E1DEDBD8D5D26D
:10769000CFCDCAC7C4C1BFBCB9B7B4B2AFADABA838
:1076A000A6A4A2A09E9C9A9896959391908F8D8C5B
:1076B0008B8A888786868584838382828281818182
:1076C0008181818182828283838485868687888A7C
:1076D0008B8C8D8F9091939596989A9C9EA0A2A446
:1076E000A6A8ABADAFB2B4B7B9BCBFC1C4C7CACD11
:1076F000CFD2D5D8DBDEE1E4E7EAEDF0F4F7FAFD2E
:10770000808182838485868788898A8B8C8D8E8F01
:10771000909192939495969798999A9B9C9D9E9FF1
:10772000A0A1A2A3A4A5A6A7A8A9AAABACADAEAFE1
:10773000B0B1B2B3B4B5B6B7B8B9BABBBCBDBEBFD1
:10774000C0C1C2C3C4C5C6C7C8C9CACBCCCDCECFC1
:10775000D0D1D2D3D4D5D6D7D8D9DADBDCDDDEDFB1
:10776000E0E1E2E3E4E5E6E7E8E9EAEBECEDEEEFA1
:10777000F0F1F2F3F4F5F6F7F8F9FAFBFCFDFEFF91
:10778000000102030405060708090A0B0C0D0E0F81
:10779000101112131415161718191A1B1C1D1E1F71
:1077A000202122232425262728292A2B2C2D2E2F61
:1077B000303132333435363738393A3B3C3D3E3F51
:1077C000404142434445464748494A4B4C4D4E4F41
:1077D000505152535455565758595A5B5C5D5E5F31
:1077E000606162636465666768696A6B6C6D6E6F21
:1077F000707172737475767778797A7B7C7D7E7F11
:1078000000020406080A0C0E10121416181A1C1E88
:1078100020222426282A2C2E30323436383A3C3E78
:1078200040424446484A4C4E50525456585A5C5E68
:1078300060626466686A6C6E70727476787A7C7E58
:107840007F7D7B79777573716F6D6B696765636138
:107850005F5D5B59575553514F4D4B494745434128
:107860003F3D3B39373533312F2D2B292725232118
:107870001F1D1B19171513110F0D0B090705030108
:10788000FFFDFBF9F7F5F3F1EFEDEBE9E7E5E3E1F8
:10789000DFDDDBD9D7D5D3D1CFCDCBC9C7C5C3C1E8
:1078A000BFBDBBB9B7B5B3B1AFADABA9A7A5A3A1D8
:1078B0009F9D9B99979593918F8D8B8987858381C8
:1078C00080828486888A8C8E90929496989A9C9EC8
:1078D000A0A2A4A6A8AAACAEB0B2B4B6B8BABCBEB8
:1078E000C0C2C4C6C8CACCCED0D2D4D6D8DADCDEA8
:1078F000E0E2E4E6E8EAECEEF0F2F4F6F8FAFCFE98
:107900007F7F7F7F7F7F7F7F7F7F7F7F7F7F7F7F87
:107910007F7F7F7F7F7F7F7F7F7F7F7F7F7F7F7F77
:107920007F7F7F7F7F7F7F7F7F7F7F7F7F7F7F7F67
:107930007F7F7F7F7F7F7F7F7F7F7F7F7F7F7F7F57
:107C00000309131E28313A40464C5054585B5E61BC
:107C1000636567696B6C6E6F70717273747576777C
:107C2000777879797A7A7B7B7C7C7C7D7D7D7E7EA2
:107C30007E7E7F7F7F7F7F7F7F7F7F7F7F7F7F7F56
:107C40007F7F7F7F7F7F7F7F7F7F7F7F7F7E7E7E47
:107C50007E7D7D7D7C7C7C7B7B7A7A797978777779
:107C6000767574737271706F6E6C6B696765636142
:107C70005E5B5854504C46403A31281E13090300AD
:107C8000C6CCD5DBDFE3E5E7E9EAEBECEDEEEFEFC1
:107C9000F0F0F0F1F1F1F1F2F2F2F2F2F2F2F2F3CD
:107CA000F3F3F3F3F3F3F3F3F3F3F3F3F3F3F3F3A4
:107CB000F3F3F3F3F3F3F3F3F3F3F3F3F3F3F3F394
:107CC000F3F3F3F3F3F3F3F3F3F3F3F3F3F3F3F384
:107CD000F3F3F3F3F3F3F3F3F3F3F3F3F3F3F3F374
:107CE000F2F2F2F2F2F2F2F2F1F1F1F1F0F0F0EF81
:107CF000EFEEEDECEBEAE9E7E5E3DFDBD5CCC60040
:107D000000283D42302D2C2B2C2D2E2F3032333598
:107D100037393B3D3F414345484A4C4E50535557F8
:107D2000595B5D5F61636567696B6C6E70717374DD
:107D3000757778797A7B7C7D7D7E7E7F7F7F7F7F84
:107D40007F7F7F7F7F7F7E7E7D7D7C7B7A7978776A
:107D500075747371706E6C6B69676563615F5D5B91
:107D600059575553504E4C4A484543413F3D3B3986
:107D700037353332302F2E2D2C2B2C2D30423D28F1
:107D800000E9E5FED4D7D7D7D6D4D2D0CECCCAC856
:107D9000C6C3C1BFBDBAB8B6B4B1AFADABA9A7A594
:107DA000A3A19F9E9C9A999795949391908F8D8C67
:107DB0008B8A898888878685858484848383838366
:107DC0008383838383848484858586878888898A5E
:107DD0008B8C8D8F909193949597999A9C9E9FA14F
:107DE000A3A5A7A9ABADAFB1B4B6B8BABDBFC1C367
:107DF000C6C8CACCCED0D2D4D6D7D7D7D4FEE5E920
:107E0000F9F8F9F5EBE1DDDEE0E2E4E5E6E5E4E2F0
:107E1000DED9D2CAC1B7ACA299918A86838180800B
:107E20008182838586888A8C8D8F90929395969790
:107E300098999A9B9B9C9D9D9D9E9E9E9F9F9F9F78
:107E40009F9F9F9E9E9E9D9D9D9C9B9B9A99989770
:107E500096959392908F8D8C8A8886858382818077
:107E6000808183868A9199A2ACB7C1CAD2D9DEE259
:107E7000E4E5E6E5E4E2E0DEDDE1EBF5F9F8F90062
:107E80000708070B151F2322201E1C1B1A1B1C1E74
:107E900022272E363F49545E676F767A7E7F7F7F3A
:107EA0007F7E7D7B7A7876747371706E6D6B6A6994
:107EB000686766656564646363626262616161618B
:107EC0006161616262626363636465656667686974
:107ED0006A6B6D6E7071737476787A7B7D7E7F7F4E
:107EE0007F7F7E7A766F675E54493F362E27221E4B
:107EF0001C1B1A1B1C1E2022231F150B0708070022
:107F00001F313D444E5354565A5F64696E747679FE
:107F10007C7F7F7F7F7F7F7F7F7F7F7F7F7F7F7F74
:107F20007F7F7F7F7F7F7F7F7F7F7F7F7F7F7F7F61
:107F30007F7F7F7F7F7F7F7F7F7F7F7F7F7F7F7F51
:107F40007F7F7F7F7F7F7F7F7F7F7F7F7F7F7F7F41
:107F50007F7F7F7F7F7F7F7F7F7F7F7F7F7F7F7F31
:107F60007F7F7F7F7F7F7F7F7F7F7F7F7F7F7F7F21
:107F70007F7F7F7F7F7F7F7F7F7F7F7C7871684C73
:107F80002C1C120C0A0B0A05FDF3E9DFD4CAC0B79A
:107F9000AEA69E97918B868582808080808080802F
:107FA00080808080808080808080808080808080D1
:107FB00080808080808080808080808080808080C1
:107FC00080808080808080808080808080808080B1
:107FD00080808080808080808080808080808080A1
:107FE0008080808080808080808080808080808091
:107FF000808080808087919DACC4CBD4DDF2FAFA7A
:108000000895E8E6F5E090EF80EE90838183349662
:1080100025E0E837F207C9F710929007109292070F
:1080200008958093730A1092760A81E08093750A0E
:10803000662321F08091750A8823E1F70895982F2F
:10804000882319F48FEF87B9089581E08093770A28
:108050008093740A892F0E9411400895982F8823D5
:1080600011F417B808958CE08093770A8FEF80930E
:10807000740A892F0E94114008958091750A8823FF
:10808000F9F08091760A8823C1F48091730A809375
:10809000760A8091770AE82FF0E0EB5FFE4FE491DB
:1080A000E7B99091740A980F9093770A992311F089
:1080B0009D3031F41092750A089581508093760AAC
:1080C00008950F931F93CF93DF938C01C0E0D0E00E
:1080D00007C00E9490348823E1F30E9494342196D3
:1080E000C017D107B4F3DF91CF911F910F9108957D
:1080F000A0E0B0E0EEE7F0E40C945470782E862E09
:108100005A016901780100E010E00CC0872D8C0F46
:10811000692DA7010E947A342196CA15DB05B4F3B4
:108120000F5F1F4F0C151D052CF4C0E0D0E0902E02
:10813000980CF3CFCDB7DEB7EDE00C947070A1E0F2
:10814000B0E0E5EAF0E40C945370882E962EFA0124
:10815000B4903196A490CB2CDD248F010F5F1F4F7C
:10816000FF2413C0F3014491892F880D6E2D50E038
:1081700099830E947A3499819F5F0894611C711CD5
:108180009B1580F3F3940C0D1D1DFA1428F438018F
:1081900090E0EF2CE90CF4CF2196EEE00C946F7098
:1081A000A0E0B0E0E6EDF0E40C944F70962F682F5D
:1081B00070E082FD8DC0A8E08A2E840E869486949D
:1081C00086948A94477019F0F2E02F2E02C0222480
:1081D0002394022F085F0695069506950150277097
:1081E00019F0E2E03E2E02C033243394D62ECC2484
:1081F000C90ED11C922F80E02C01440E511CEE249C
:10820000FF240C3108F05DC08EE1089F300111247D
:10821000982C80E09E2D9C01E9018DE1891508F4E0
:108220004BC05301A90CB11CF501E05EFD4F10815C
:1082300020E0183008F021E090E0809191071817B5
:1082400008F491E0222321F4992311F4212F2AC06C
:1082500060919007683010F0212F22C0222329F06E
:10826000812F88500E94932B05C0992319F0812FEC
:108270000E94222C20919007822F90E0FC01EE0FAB
:10828000FF1FE80FF91FE858F84FD501A05EBD4F5A
:10829000B183A08312832C932F5F209390072150EA
:1082A000283050F480919107281730F0822FB601C2
:1082B000AE0192010E94C22C93942196C21508F43B
:1082C000ACCF0894E11CF11C0F5FE31408F499CFC4
:1082D000CDB7DEB7E2E10C946B70CF93DF93809162
:1082E00000018823A9F080919207809391078093E1
:1082F0009007C8E6D5E08B816A81488129810E9478
:10830000D040249685E0C837D807A9F70E94AF2C43
:10831000DF91CF9108950E943D400E946D410895E4
:108320006AE00E94D26F892F08956AE00E94D26F9E
:108330000E94D26F892F0895A2E0B0E0E2EAF1E452
:108340000C944F701C016B01FB0180E090E007C0B2
:108350002101F1E0AF2EB12CE6E06E2E62C1108259
:10836000118212821382148215820196369686300B
:108370009105A9F7EDCF21E0A216B10411F49C01FB
:1083800003C0950121503040A816B90621F471E0D0
:10839000872E912C04C045010894811C911CC101B9
:1083A000820F931F9A838983FC01E0808E2D0E94A7
:1083B0009541782EF2010181802F0E949541F82E7F
:1083C000871560F4802F0E949041182FF101E80D6D
:1083D000F91D80810E949041181798F0820C931C1F
:1083E000F4018080882D0E949541982EF816D0F4D3
:1083F000802F0E949041182F8E2D0E9490411817B7
:1084000088F4802F0E94904190E0FC01EE0FFF1F46
:10841000E80FF91FEE0FFF1FEC0DFD1DEF0DF11D15
:1084200021E06BC0F71448F4802F0E949041182F70
:10843000882D0E949041811758F0F914D0F4802FB4
:108440000E949041182F8E2D0E949041811788F430
:10845000802F0E94904190E0FC01EE0FFF1FE80F7B
:10846000F91FEE0FFF1FEC0DFD1DEF0DF11D82E05A
:1084700067C07F1448F4802F0E949041182F882DE8
:108480000E949041181758F09F14D8F4802F0E9432
:108490009041182F8E2D0E949041181790F4802F34
:1084A0000E94904190E0FC01EE0FFF1FE80FF91FC2
:1084B000EE0FFF1FEC0DFD1DEF0DF11D93E09083FE
:1084C00040C08E2D0E949041E82E802F0E94904146
:1084D000182FE816A1F4882D0E9490418E1579F48A
:1084E00090E0FC01EE0FFF1FE80FF91FEE0FFF1FDA
:1084F000EC0DFD1DEF0DF11D25E0208322C07F1442
:1085000089F4971479F4812F90E0FC01EE0FFF1F9E
:10851000E80FF91FEE0FFF1FEC0DFD1DE90DF11D1A
:1085200060820FC0812F90E0FC01EE0FFF1FE80F6B
:10853000F91FEE0FFF1FEC0DFD1DEF0DF11D84E087
:108540008083F201F1808F2D0E949541182FE981DF
:10855000FA810081802F0E949541181791F58F2D87
:108560000E949041182F802F0E949041412F50E08F
:10857000282F30E0181770F48A010F5F1F4F790120
:108580004801880C991C800E911E880C991C8C0C3B
:108590009D1C13C089010F5F1F4F7A01F1CFF201BB
:1085A00081810E949541F401E80FF11D60820F5F07
:1085B0001F4F86E090E0880E991E0E151F0578F378
:1085C0002AC0412F50E0282F30E0181730F47A01EC
:1085D0000894E11CF11C89011BC079010894E11C7D
:1085E000F11C8A0115C0F20181810E94904190E046
:1085F000FC01EE0FFF1FE80FF91FEE0FFF1FEC0D40
:10860000FD1DEE0DFF1D25E020830894E11CF11CEB
:10861000E016F10640F30894A11CB11C0894411C1B
:10862000511CF101808190E08A159B0508F0A3CED2
:108630002296E2E10C946B70A4E1B0E0E2E2F3E494
:108640000C944F702B01FC013297EB30F105F8F4DC
:10865000E85CFF4F0C9486702CE831E524C048EFAD
:1086600059E019C02AE931E51EC028EA31E51BC0EE
:1086700026EB31E518C024EC31E515C022ED31E5DB
:1086800012C020EE31E50FC02EEE31E50CC00B9785
:1086900040F040E751E520E030E0BE016F5F7F4FE2
:1086A00014C020E731E580E090E0AE014F5F5F4FFE
:1086B000F901E80FF91FE491DA01A80FB91FEC9353
:1086C00001968E309105A1F70DC0FB01E20FF31F5B
:1086D000DA01A20FB31F8C9180832F5F3F4F2E30A2
:1086E000310599F7E980F201E082FA808F2D0E942E
:1086F0009541082F8F2D0E9490419AE0099F80019B
:108700001124800FF20181839E012D5F3F4F3A8B30
:10871000298B82E0C82ED12C82E090E0EE2DF0E093
:10872000FC8BEB8B31C19C012F5F3F4F388B2F8728
:10873000E989FA89B080F7ECFB1508F4BEC02B89F3
:108740003C89C216D30608F0A2C08B2D0E94954129
:10875000082F8B2D0E94904112012C0C3D1C3AE0F9
:10876000039F80011124F82EF00EF101F0824601E2
:108770000894811C911C6201C80CD91C8F2D0E9489
:108780009541082F8F2D0E949041FAE00F9F8001A4
:108790001124080FF6010083F10180810E949041AD
:1087A000182FF601329780810E949041181739F4F2
:1087B000F3E6FB1510F4015008C00F5F06C0F3E6A6
:1087C000FB1510F40A5001C0065FF60100830894FF
:1087D000811C911C2B893C898216930621F4B1E0FF
:1087E000AB2EB12C02C0AF84B8883201680C791C62
:1087F0000894810891086201C80CD91C0894811C56
:10880000911CF601F0808F2D0E949541082F8F2D2D
:108810000E949041FAE00F9F80011124080FF3019C
:108820000083F60180810E949041182FF101808120
:108830000E9490411817A1F421E030E02C0F3D1F59
:10884000A20EB31EF50180810E949041182F802F47
:108850000E949041181710F4015015C00F5F13C00B
:1088600021E030E02C0F3D1FA20EB31EF5018081E8
:108870000E949541182F802F0E949541181710F4DF
:108880000A5001C0065FF3010083640172C02B89A6
:108890003C89C216D30689F48B2D0E949541082F7E
:1088A0008B2D0E949041F201EC0DFD1D3AE0039FDB
:1088B00080011124800F80835CC08B2D0E94954124
:1088C000082F8B2D0E949041F201EC0DFD1D9AE0C6
:1088D000099F80011124800F808356010894A11CF8
:1088E000B11CF201808190E0A816B90621F4A1E044
:1088F000EA2EF12C02C0EF84F8886201CA0CDB1C5E
:10890000F60102916F010894C11CD11C802F0E94B6
:108910009041182FF601329780810E9490411817DC
:10892000B1F4802F0E949541082F21E030E02C0FF8
:108930003D1FE20EF31EF70180810E949041FAE094
:108940000F9F80011124800FF601808311C021E068
:1089500030E02C0F3D1FE20EF31EF70180810E94D4
:108960009541FAE08F9FC0011124180FF601108382
:1089700065010894C11CD11C29893A892F5F3F4F9A
:108980003A8B298B8F859889EB89FC89EC15FD053D
:1089900008F0C9CE06C04AEE59E07DCE2EE731E59B
:1089A00082CE6496E2E10C946B70CF93DF93EC017E
:1089B000888190E0019762E070E00E94FF6F9B0168
:1089C000DE01A60FB71F2AC0E881F0E03196E21B56
:1089D000F30BEC0FFD1F908112968C911297982744
:1089E00012969C931297E881F0E03196E21BF30B0C
:1089F000EC0FFD1F808189278083E881F0E03196AC
:108A0000E21BF30BEC0FFD1F12968C9112979081D5
:108A1000892712968C931297215030401197211577
:108A2000310591F6DF91CF910895AC016130710568
:108A300071F48BE290E0489FF001499FF00D589F40
:108A4000F00D1124E656F54F80818F5F0FC0672B24
:108A500071F48BE290E0489FF001499FF00D589F20
:108A6000F00D1124E656F54F8081815080838BE212
:108A700090E0489FF001499FF00D589FF00D1124A0
:108A8000E656F54F80818F3F19F487E0808303C05D
:108A9000883009F410828BE290E0489FF001499FF2
:108AA000F00D589FF00D1124E656F54F60819A01A4
:108AB000220F331F220F331FDA01AA0FBB1F6530AD
:108AC000A8F0F901E859FA4F81E08383AA0FBB1F90
:108AD000A659BA4F84E090E0861B9109880F991F30
:108AE000240F351F820F860F8C930895F901E859E2
:108AF000FA4F1382AA0FBB1FA659BA4F240F351F76
:108B0000620F6C930895CF92DF92EF92FF920F93D2
:108B10001F939C018BE290E0289FF001299FF00DAC
:108B2000389FF00D1124E656F54F8081E82FF0E0D4
:108B3000E830F10508F0FDC0ED5BFF4F0C94867046
:108B40008BE290E0289FF001299FF00D389FF00DF7
:108B50001124E656F54F13861486158616868389EA
:108B60009489A589B689B095A095909581959F4FD8
:108B7000AF4FBF4F62C08BE290E0289F8001299FDA
:108B8000100D389F100D11240656154FF801C3889B
:108B9000D488E588F688C701B60127E430E040E0D4
:108BA00050E00E94B36F24E630E040E050E00E94C5
:108BB0003470F8012387348745875687C701B6018B
:108BC00029EB3FEF4FEF5FEF66C08BE290E0289F0D
:108BD000F001299FF00D389FF00D1124E656F54F56
:108BE00083899489A589B68976C08BE290E0289F15
:108BF0008001299F100D389F100D11240656154F26
:108C0000F801638974898589968927E430E040E01A
:108C100050E07EC08BE290E0289FF001299FF00D8C
:108C2000389FF00D1124E656F54F138614861586ED
:108C3000168683899489A589B6898787908BA18BAD
:108C4000B28B77C08BE290E0289F8001299F100DA6
:108C5000389F100D11240656154FF801C388D4888B
:108C6000E588F688C701B60129EB3FEF4FEF5FEFCC
:108C70000E94B36F24E630E040E050E00E94347080
:108C8000F8012387348745875687C701B60127E453
:108C900030E040E050E00E94B36F24E630E040E076
:108CA00050E00E943470F80140C08BE290E0289FB1
:108CB000F001299FF00D389FF00D1124E656F54F75
:108CC00083899489A589B689B095A0959095819559
:108CD0009F4FAF4FBF4F83879487A587B68717866F
:108CE000108A118A128A25C08BE290E0289F8001A9
:108CF000299F100D389F100D11240656154FF801AD
:108D0000638974898589968929EB3FEF4FEF5FEF7F
:108D10000E94B36F24E630E040E050E00E943470DF
:108D2000F80123873487458756872787308B418B07
:108D3000528B1F910F91FF90EF90DF90CF9008958D
:108D40002BE230E0829FF001839FF00D929FF00DA7
:108D50001124E656F54F83859485A585B685278928
:108D6000308D418D528D820F931FA41FB51F878BAD
:108D7000908FA18FB28F87859089A189B289238D29
:108D8000348D458D568D820F931FA41FB51F838F81
:108D9000948FA58FB68F08952BE230E0829FF0016B
:108DA000839FF00D929FF00D1124E656F54F8389B5
:108DB0009489A589B6890296A11DB11D838B948BD8
:108DC000A58BB68B258130E040E050E028173907AD
:108DD0004A075B0724F4238B348B458B568B08950D
:108DE000EF92FF920F931F932BE230E0829FF001EE
:108DF000839FF00D929FF00D1124E656F54F2389C5
:108E00003489458956892250304040405040238B58
:108E1000348B458B568B8581869590E09095819516
:108E20009F4F7C010027F7FC0095102F2E153F0562
:108E30004007510724F4E38AF48A058B168B1F91AF
:108E40000F91FF90EF9008952BE230E0829FF001A8
:108E5000839FF00D929FF00D1124E656F54F838904
:108E60009489A589B689181619061A061B0644F4B2
:108E70000197A109B109838B948BA58BB68B0895BB
:108E80000097A105B10539F00196A11DB11D838B95
:108E9000948BA58BB68B089589E392E090937B0A1F
:108EA00080937A0A8091F90A9091FA0A83709070FF
:108EB000880F991F2091FC0A820F911D880F991F1E
:108EC0002091780A820F911D880F991F2091F30A33
:108ED000820F911D880F991F2091F80A820F911D12
:108EE000880F991F20910201332727FD3095820FAB
:108EF000931F880F991F8093980AEAEEF9E0ACE778
:108F0000BAE081918D9389E0E83FF807D1F7E8EF67
:108F1000F9E0AAE8BAE081918D938AE0E630F8079B
:108F2000D1F78AE79AE00E944E3508950F931F9378
:108F300080E090E060E070E043E050E02CE130E061
:108F400000E010E00E9478408BE190E060E070E08B
:108F500043E050E02CE130E00E94784082E090E075
:108F600066E070E041E050E026E030E00CE910E01F
:108F70000E9478408BE190E066E070E041E050E0D4
:108F800026E030E00E94784082E090E06CE070E003
:108F900041E050E023E030E00EE810E00E9478402D
:108FA0008BE190E06CE070E041E050E023E030E0E5
:108FB0000E9478401F910F910895FF920F931F9385
:108FC000CF93DF93EC011981812F0E949041082FEC
:108FD000FA808F2D0E949041081708F03FC0812F22
:108FE0000E949541202F30E0220F331F220F331FA4
:108FF000682F70E0660F771F660F771F6E5F7F4FD9
:10900000C901069641E050E024E030E001EA10E0BA
:109010000E94784082E080936A0587E080936E0525
:1090200010926B0510926F0589810E949041829584
:10903000880F807E885D8093680589810E949541B4
:109040008295880F807E8B5E8093690589810E945E
:1090500090418295880F807E885D48C0801708F017
:109060004FC0812F0E949541202F30E0220F331FE7
:10907000220F331F682F70E0660F771F660F771F70
:109080006E5F7F4FC901039641E050E024E030E07D
:1090900001EA10E00E94784082E080936A0587E050
:1090A00080936E0581E080936B0580936F058981C5
:1090B0000E94904190E0019625E0880F991F2A9523
:1090C000E1F78093680589810E9495418295880F18
:1090D000807E8B5E8093690589810E94904190E03B
:1090E000019605E0880F991F0A95E1F780936C05BA
:1090F00089810E9495418295880F807E8D5D94C004
:10910000812F0E949541182F8F2D0E949541202F6D
:1091100030E0612F70E0811708F040C0220F331F4C
:10912000220F331F660F771F660F771F6E5F7F4F0B
:10913000C901039644E050E021E030E001EA10E08C
:109140000E94784010926A0585E080936E05109227
:109150006B0510926F0589810E9490418295880F5E
:10916000807E835E8093680589810E949541829507
:10917000880F807E885E8093690589810E94904176
:109180008295880F807E855D80936C0589810E9421
:1091900095418295880F807E885E46C0220F331FDE
:1091A000220F331F660F771F660F771F6B5F7F4F8E
:1091B000C901039644E050E021E030E001EA10E00C
:1091C0000E94784084E080936A0589E080936E0570
:1091D00010926B0510926F0589810E9490418295D3
:1091E000880F807E835E8093680589810E94954107
:1091F00090E00196E5E0880F991FEA95E1F78093EA
:10920000690589810E9490418295880F807E855DE5
:1092100080936C0589810E94954190E0019675E0EC
:10922000880F991F7A95E1F780936D0583E090E0B0
:1092300060E070E048E150E022E030E00EE710E04E
:109240000E94784083E090E06AE170E048E150E0FD
:1092500022E030E00E947840CDB7DEB7E5E00C9424
:109260007870A0E0B0E0E7E3F9E40C945470F82ED5
:10927000E92E0E946C3483E090E062E070E048E107
:1092800050E028E130E00EE710E00E9478402F2DFA
:109290003E2DC9014C01A3E0EA2EF12C53C0F6018A
:1092A0008081833031F184303CF48130C1F08230F0
:1092B000DCF4882341F032C0853029F18530F4F0A8
:1092C000863061F525C0872D9A2DBE0144E050E01F
:1092D00024E030E00EE710E00E9478401FC08B2DA4
:1092E0006C2F48EC51E018C08B2D6C2F4AED51E0EB
:1092F00013C08B2D6C2F4CEE51E00EC08B2D6C2FBC
:109300004EEF51E009C08B2D6C2F40E152E004C0BC
:109310008B2D6C2F42E252E00E949F400894C11CAA
:10932000D11C2496CA31D10509F0B9CF86E090E06E
:10933000880E991EE4E0F0E0EE0EFF1EFBE1EF1652
:10934000F10439F07E2CAF2CBE2C6401C2E0D0E0D9
:10935000A6CFCDB7DEB7EDE00C94707082309105EA
:1093600069F08330910529F0019761F489EB9EE360
:1093700002C083ED9DE40E94A936089582E297E43D
:109380000E94A9360895AAE0B0E0E9ECF9E40C9453
:109390004F709A8789878091A50A9091A60AA0911B
:1093A000A70AB091A80A8D839E83AF83B887609087
:1093B000D00A7090D10A8090D20A9090D30AE0909F
:1093C000B10AF090B20A0091B30A1091B40AE80E03
:1093D000F91E0A1F1B1F8091DC0A9091DD0AA091E3
:1093E000DE0AB091DF0AE81AF90A0A0B1B0BE6182D
:1093F000F708080919098091A90A9091AA0AA09171
:10940000AB0AB091AC0A89839A83AB83BC8320906A
:10941000D40A3090D50A4090D60A5090D70A2091AD
:10942000B50A3091B60A4091B70A5091B80A280F90
:10943000391F4A1F5B1F8091E00A9091E10AA091B9
:10944000E20AB091E30A281B390B4A0B5B0B221985
:10945000330944095509CA01B9010E94B36F5B0180
:109460006C01C801B701A80197010E94B36FA60E55
:10947000B71EC81ED91EC601B5010E94C0310E9488
:10948000F17020E030E048EC52E40E94E4300E94A9
:109490000E2F693071058105910510F080E073C0D1
:1094A0008D819E81AF81B885680E791E8A1E9B1EB4
:1094B000C401B30122E030E040E050E00E9434708B
:1094C0002093A50A3093A60A4093A70A5093A80AAE
:1094D0002093D00A3093D10A4093D20A5093D30AF2
:1094E00089819A81AB81BC81280E391E4A1E5B1E80
:1094F000C201B10122E030E040E050E00E9434704F
:109500002093A90A3093AA0A4093AB0A5093AC0A5D
:109510002093D40A3093D50A4093D60A5093D70AA1
:10952000A985BA85AB2B71F58091EF0A882351F597
:1095300081E090E061E070E00E9415458091CA0AE8
:1095400090E0A0E0B0E08093D80A9093D90AA0936D
:10955000DA0AB093DB0A8091C40A882399F480E088
:1095600090E061E070E00E94154580919F0A90E0D4
:10957000A0E0B0E08093AD0A9093AE0AA093AF0A4A
:10958000B093B00A81E02A96E2E10C946B706F927E
:109590007F928F929F92AF92BF92CF92DF92EF9283
:1095A000FF920F931F935B016C0139014A01FF2465
:1095B00020E83CE0E29EC001E39E900DF29E900DFB
:1095C0001124AA2797FDA095BA2FA81AB90ACA0A8A
:1095D000DB0A10E0029FC001039F900D129F900DC7
:1095E0001124AA2797FDA095BA2F681A790A8A0A2A
:1095F0009B0AC601B501A60195010E94B36F7B01CC
:109600008C01C401B301A40193010E94B36FE60E63
:10961000F71E081F191FC801B7010E94C0310E9420
:10962000F17020E030E048EC52E40E94E4300E9407
:109630000E2F9B01AC01CA011F910F91FF90EF907B
:10964000DF90CF90BF90AF909F908F907F906F9062
:1096500008956F927F928F929F92AF92BF92DF9206
:10966000EF92FF920F931F93CF93DF935C01FB0167
:109670003A0149016BE270E0869FE001879FD00DBF
:10968000969FD00D1124C656D54F2E8130E0C901CA
:10969000880F991F820F931F880F991FE80FF91FDA
:1096A0008F81E80FF11DE081E53089F58B859C8580
:1096B000AD85BE852F8D38A149A15AA1820F931F78
:1096C000A41FB51F845F9140A040B0408C5F9840BC
:1096D000A040B04008F4C3C21B861C861D861E86AF
:1096E0008AE08816910408F4B7C282E090E08A19F3
:1096F0009B09869FF001879FF00D969FF00D112426
:10970000E656F54F1386148615861686A5C2E630F2
:1097100059F58F859889A989BA892BA13CA14DA1BA
:109720005EA1820F931FA41FB51F845F9140A040CC
:10973000B0408C5F9840A040B04008F490C21F86B3
:10974000188A198A1A8A8AE08816910408F484C251
:1097500082E090E08A199B09869FF001879FF00DB7
:10976000969FF00D112472C2E13009F091C06B8513
:109770007C858D859E852F8D38A149A15AA1620FC8
:10978000731F841F951F2BA13CA14DA15EA101E079
:10979000EE24E3940E94C74A6C317105810591055E
:1097A000C8F46B857C858D859E852F8D38A149A158
:1097B0005AA1620F731F841F951F2BA13CA14DA1BD
:1097C0005EA10E94C74A643071058105910510F0C1
:1097D000DD2426C02BE230E0A29EF001A39EF00D16
:1097E000B29EF00D1124E656F54F138614861586A9
:1097F00016868AE08816910488F082E090E08A1943
:109800009B09829FF001839FF00D929FF00D112420
:10981000E656F54F1386148615861686DD24D394F6
:109820008BE290E0A89EE001A99ED00DB89ED00DDD
:109830001124C656D54F6F8D78A189A19AA12F8585
:10984000388949895A89EBA0FCA00DA11EA12E0DD3
:109850003F1D401F511F01E0EE24E3940E94C74AC0
:109860006C3171058105910508F0D2C16F8D78A129
:1098700089A19AA12F85388949895A89EBA0FCA032
:109880000DA11EA12E0D3F1D401F511F01E025C13E
:10989000E23009F08FC06B857C858D859E852F8D8C
:1098A00038A149A15AA1620F731F841F951F2BA1D4
:1098B0003CA14DA15EA101E0EE240E94C74A6C319B
:1098C000710581059105C8F46B857C858D859E8524
:1098D0002F8D38A149A15AA1620F731F841F951FB4
:1098E0002BA13CA14DA15EA10E94C74A6430710525
:1098F0008105910510F0DD2426C02BE230E0A29E08
:10990000F001A39EF00DB29EF00D1124E656F54F26
:1099100013861486158616868AE08816910488F0C8
:1099200082E090E08A199B09829FF001839FF00DED
:10993000929FF00D1124E656F54F13861486158676
:109940001686DD24D3948BE290E0A89EE001A99EC8
:10995000D00DB89ED00D1124C656D54F6F8D78A16D
:1099600089A19AA12F85388949895A89EBA0FCA041
:109970000DA11EA12E0D3F1D401F511F01E0EE2421
:109980000E94C74A6C3171058105910508F040C1FC
:109990006F8D78A189A19AA12F85388949895A8923
:1099A000EBA0FCA00DA11EA12E0D3F1D401F511FBD
:1099B00001E026C1E33009F093C06B857C858D857D
:1099C0009E852F8D38A149A15AA1620F731F841F54
:1099D000951F2BA13CA14DA15EA100E0EE24E394D4
:1099E0000E94C74A6C31710581059105C8F46B85E9
:1099F0007C858D859E852F8D38A149A15AA1620F46
:109A0000731F841F951F2BA13CA14DA15EA10E9435
:109A1000C74A643071058105910510F0DD2426C028
:109A20002BE230E0A29EF001A39EF00DB29EF00D5D
:109A30001124E656F54F13861486158616868AE09D
:109A40008816910488F082E090E08A199B09829F31
:109A5000F001839FF00D929FF00D1124E656F54F13
:109A60001386148615861686DD24D3948BE290E047
:109A7000A89EE001A99ED00DB89ED00D1124C65617
:109A8000D54F6F8D78A189A19AA12F8538894989F1
:109A90005A89EBA0FCA00DA11EA12E0D3F1D401F59
:109AA000511F00E0EE24E3940E94C74A6C31710517
:109AB0008105910508F0ACC06F8D78A189A19AA1AC
:109AC0002F85388949895A89EBA0FCA00DA11EA1D8
:109AD0002E0D3F1D401F511F00E0EE24E39491C066
:109AE000E43009F0BCC06B857C858D859E852F8D0B
:109AF00038A149A15AA1620F731F841F951F2BA182
:109B00003CA14DA15EA100E0EE240E94C74A6C3149
:109B1000710581059105C8F46B857C858D859E85D1
:109B20002F8D38A149A15AA1620F731F841F951F61
:109B30002BA13CA14DA15EA10E94C74A64307105D2
:109B40008105910510F0DD2426C02BE230E0A29EB5
:109B5000F001A39EF00DB29EF00D1124E656F54FD4
:109B600013861486158616868AE08816910488F076
:109B700082E090E08A199B09829FF001839FF00D9B
:109B8000929FF00D1124E656F54F13861486158624
:109B90001686DD24D3948BE290E0A89EE001A99E76
:109BA000D00DB89ED00D1124C656D54F6F8D78A11B
:109BB00089A19AA12F85388949895A89EBA0FCA0EF
:109BC0000DA11EA12E0D3F1D401F511F00E0EE24D0
:109BD0000E94C74A6C31710581059105C8F46F8DEB
:109BE00078A189A19AA12F85388949895A89EBA042
:109BF000FCA00DA11EA12E0D3F1D401F511F00E016
:109C0000EE240E94C74A643071058105910540F534
:109C10002BE230E0A29EF001A39EF00DB29EF00D6B
:109C20001124E656F54F1786108A118A128A8AE0A7
:109C30008816910488F082E090E08A199B09829F3F
:109C4000F001839FF00D929FF00D1124E656F54F21
:109C50001786108A118A128ADD24D39401C0DD246C
:109C6000A614B704E8F0DD20D9F08BE290E0A89EBE
:109C7000E001A99ED00DB89ED00D1124C656D54F37
:109C80008AA5882369F4C50161E070E00E9415454A
:109C90008D8190E0A0E0B0E08B8B9C8BAD8BBE8B78
:109CA0008D2DDF91CF911F910F91FF90EF90DF905D
:109CB000BF90AF909F908F907F906F900895FF928C
:109CC0000F931F93F82E86E090E062E170E041E090
:109CD00050E028E030E000E010E00E94784085E0AD
:109CE00090E062E170E041E050E028E030E00E9466
:109CF000784082E1F80E86E06F2D4CE950E00E943A
:109D00007A3485E06F2D45E950E00E947A3485E190
:109D100090E062E170E041E050E028E030E00E9435
:109D2000784086E190E062E170E041E050E028E0B8
:109D300030E00E94784085E16F2D4CE950E00E94B0
:109D40007A3486E16F2D45E950E00E947A341F9104
:109D50000F91FF900895FF920F931F93F82E86E0C6
:109D600090E062E170E041E050E028E030E000E0A7
:109D700010E00E94784082E1F80E86E06F2D45E900
:109D800050E00E947A341F910F91FF90089589E36B
:109D900092E090937B0A80937A0A6AE77AE00E94C5
:109DA0000A354091980A842F90E09C0166E0369530
:109DB00027956A95E1F73093FA0A2093F90A4270E1
:109DC000409302019695879596958795282F217047
:109DD0002093F80A96958795282F21702093F30AEF
:109DE00096958795282F21702093780A96958795C8
:109DF00081708093FC0AECE7FAE0AAEEB9E0819169
:109E00008D938AE0EA38F807D1F7A8EFB9E081919D
:109E10008D938AE0E839F807D1F780918A0A882380
:109E200021F480918B0A882319F08CE090E00DC01A
:109E300080917C0A882321F480917D0A882319F07F
:109E40008BE090E002C08AE090E09093F70A809364
:109E5000F60A08954F925F926F927F928F929F922F
:109E6000AF92BF92CF92DF92EF92FF921F93DF9358
:109E7000CF93CDB7DEB72E970FB6F894DEBF0FBEE7
:109E8000CDBF5C012B016A01FE0131968EE0DF013E
:109E90001D928A95E9F7A982FA0180818A83E3E01D
:109EA000EE2EF12CEC0EFD1EA1E0B0E03501089481
:109EB000610871087EEF872E7FEF972E8A0C9B1C1E
:109EC00093C0A615B70539F4F601EA0FFB1F808190
:109ED000F701808385C0F601EA0FFB1FA815B905BD
:109EE00008F079C01081319780816AE00E94D26FBA
:109EF000282F812F0E94D26F412F50E0BD016F5F4C
:109F00007F4F281749F5CA010A97F601E60FF71F98
:109F1000208130E08217930751F41296F601EA0F80
:109F2000FB1F8081282F30E0CA01099728C0CA0191
:109F30000A968217930709F049C01296F601EA0FB4
:109F4000FB1F8081282F30E0CA010B9628173907A4
:109F5000B1F1475F5F4F30C0CA010197F601E60FCC
:109F6000F71F208130E08217930799F41296F601CB
:109F7000EA0FFB1F8081282F30E0CA0109962817BD
:109F8000390729F04B50504024173507D9F41C5994
:109F900016C0CA01019682179307C1F41296F60102
:109FA000EA0FFB1F8081282F30E0CA010B9628178B
:109FB000390729F0495050402417350719F4F701A3
:109FC00010830EC01853D7011C9303C01853F70118
:109FD0001083DB0105C080818853F70180831196CF
:109FE00011960894E11CF11CAA15BB0508F469CF71
:109FF000FBE04F16510499F420E030E0AE014F5FD2
:10A000005F4FF901E651F64FDA01A20FB31F8C91B1
:10A0100080832F5F3F4F2E30310599F712C020E02B
:10A0200030E0AE014F5F5F4FF901E850F64FDA01C3
:10A03000A20FB31F8C9180832F5F3F4F2E303105CD
:10A0400099F70E944C470E94C74E2E960FB6F8947F
:10A05000DEBF0FBECDBFCF91DF911F91FF90EF907C
:10A06000DF90CF90BF90AF909F908F907F906F9038
:10A070005F904F900895A0E0B0E0E1E4F0E50C942B
:10A080005A708C01EB01F42ED22EEE24FF2011F435
:10A09000EE2051F48F2D6AE00E94D26F985E802FDF
:10A0A0006C2F492F0E947634DD2011F0219702C0D9
:10A0B00001501040E39483E0E81631F08F2D6AE000
:10A0C0000E94D26FF82EE2CFCDB7DEB7E7E00C9456
:10A0D000767080919C0A40910501481710F440E089
:10A0E00002C04F5F481B82E090E060E170E021E039
:10A0F0000E943B508091C70A40910501481710F417
:10A1000040E002C04F5F481B8BE190E060E170E0EF
:10A1100021E00E943B500895A0E0B0E0E2E9F0E5C4
:10A120000C9458707C018B018BE290E0E89EF0016A
:10A13000E99EF00DF89EF00D1124E656F54F43818F
:10A14000423020F0C42FD0E0219704C0DB018C9175
:10A15000C82FD0E0F8018081481718F0E1E0F0E066
:10A1600003C0E42FF0E031968BE290E0E89ED0014E
:10A17000E99EB00DF89EB00D1124A656B54F179666
:10A180009C9117978AE0989F9001112416968C91C4
:10A190001697280F311DE00FF11F808190E02817DE
:10A1A000390721F44F5F13964C9320C0F801EC0F50
:10A1B000FD1F808190E028173907C1F412968C9119
:10A1C0001297882339F0413029F48F5F12968C93CF
:10A1D0000E9469508BE290E0E89EF001E99EF00D4C
:10A1E000F89EF00D1124E656F54FC3838BE290E004
:10A1F000E89EF001E99EF00DF89EF00D1124E65660
:10A20000F54F9381D8018C91891718F481E08383ED
:10A2100081A78BE290E0E89EE001E99ED00DF89ED8
:10A22000D00D1124C656D54FCA80CC2009F46FC07A
:10A2300089A5882309F46BC0F801B2808B2D0E9498
:10A240009541D82ED80111960C91802F0E949541EE
:10A25000D81658F48BA19CA1ADA1BEA1845F9140FA
:10A26000A040B0400CF440C00BC08D1548F48BA149
:10A270009CA1ADA1BEA189529A40A040B040A4F5D6
:10A280008B2D0E949041182F802F0E94904118170B
:10A29000A8F48BE290E0E89EF001E99EF00DF89EB4
:10A2A000F00D1124E656F54F878D90A1A1A1B2A122
:10A2B000845F9140A040B040BCF029C0811738F5C0
:10A2C0008BE290E0E89EF001E99EF00DF89EF00D23
:10A2D0001124E656F54F878D90A1A1A1B2A1895214
:10A2E0009A40A040B0409CF08BE290E0E89E800154
:10A2F000E99E100DF89E100D11240656154FCA94B4
:10A30000D8011296CC920E946950F80111A6CDB7DF
:10A31000DEB7E9E00C9474700F931F9382E090E035
:10A3200066E170E041E050E023E030E000E010E062
:10A330000E9478408BE190E066E170E041E050E0FF
:10A3400023E030E00E94784040919B0A469582E0ED
:10A3500090E068E170E021E00E943B504091C60A25
:10A3600046958BE190E068E170E021E00E943B506F
:10A370001F910F9108952BE230E0829FF001839F9F
:10A38000F00D929FF00D1124E656F54F8181882340
:10A3900091F08150818386E985836B35710510F0DA
:10A3A0000E948C518091780A882329F48AE060E425
:10A3B00041E00E94CE390895A0E0B0E0E2EEF1E580
:10A3C0000C9458707C018B016A01B22EC0E0D0E081
:10A3D000F601EC0FFD1F21964491433C19F42196A0
:10A3E00041E31DC0453211F449E019C0842F885261
:10A3F000823018F44F774E5112C0842F81548C3024
:10A4000018F44F7745530BC0842F8D548E3018F4B9
:10A410004F774A5204C0442389F04F774851BB20FC
:10A4200031F48E2D0894E11CF11C602F04C0602FC4
:10A430000F5F1F4F8E2D0E947634CACFCDB7DEB787
:10A44000E9E00C9474700E946C3486E090E062E065
:10A4500070E043E052E520E00E94DC5185E066E0D8
:10A4600042E151E00E949F40089582E090E00E9406
:10A47000AE4982E060E00E941F400E946C3480EF91
:10A480008093680580936C0586E090E062E070E060
:10A4900046ED53E520E00E94DC518AE090E066E062
:10A4A00070E043EF53E520E00E94DC5182E190E050
:10A4B00066E070E04AEE53E520E00E94DC5182E065
:10A4C00090E06AE070E04EEA53E520E00E94DC5143
:10A4D00082E090E06CE070E043EB53E520E00E9406
:10A4E000DC518CE090E06AE070E04091F20A21E0FB
:10A4F0000E943B508CE090E06CE070E04091790A63
:10A5000021E00E943B5086E190E06AE070E04091DB
:10A51000FB0A21E00E943B5086E190E06CE070E095
:10A520004091F00A21E00E943B509091F20A809104
:10A53000790A89174CF486E090E062E170E04AEF16
:10A5400053E520E00E94DC519091790A8091F20A53
:10A5500089174CF486E090E062E170E04AE054E54F
:10A5600020E00E94DC519091F20A8091790A9817BC
:10A57000F1F49091FB0A8091F00A89174CF486E07F
:10A5800090E062E170E04AEF53E520E00E94DC5188
:10A590009091F00A8091FB0A89174CF486E090E0D4
:10A5A00062E170E04AE054E520E00E94DC518AE07C
:10A5B00090E069E170E044E152E520E00E94DC5166
:10A5C00080E00E949A340897D9F70E94E3360C94F1
:10A5D000000008950E946C3488EE80936805109204
:10A5E0006C0582E3809369058EEA80936D0582E0B5
:10A5F00080936A0587E080936E0581E080936B0508
:10A6000010926F0513C081E090E00E94614080913C
:10A61000680582508093680580916C058E5F8093F9
:10A620006C05809170058E5F809370058091680540
:10A63000893648F784E080936A0510926B0585E0BF
:10A6400080936E050EC081E090E00E946140809191
:10A6500069058E5F8093690580916D0582508093B6
:10A660006D05809169058C3670F38BE06FEF41E0EA
:10A670000E94CE3980EF8093680580936C058CE052
:10A6800090E06EE070E04CEF51E520E00E94DC517C
:10A6900088E790E00E94614008950F931F93809196
:10A6A0009C0A882331F020E030E08091C70A88239B
:10A6B00011F421E030E08901000F111F80919E0A02
:10A6C0009801280F311DA901A3E0440F551FAA9539
:10A6D000E1F7421B530B4A505D4A82E090E063E091
:10A6E00070E021E00E94DC518091C90A080F111D21
:10A6F000A801F3E0440F551FFA95E1F7401B510BF9
:10A700004A505D4A8BE190E063E070E021E00E94F6
:10A71000DC511F910F910895CF92DF92FF920F931A
:10A720001F93CF93DF93DC016B01EA0100919C0A38
:10A73000F090C70A0F1521F00F1508F08DC082C0E8
:10A740009091C30A8091EE0A981721F0992309F499
:10A7500083C078C090919D0A8091C80A981721F013
:10A76000891708F079C06EC08C91981719F4E1E050
:10A77000F0E003C0E92FF0E03196EA0FFB1F1081F3
:10A78000812F0E9495419091A10A981788F42091F9
:10A79000B50A3091B60A4091B70A5091B80A809133
:10A7A000E00A9091E10AA091E20AB091E30A45C063
:10A7B000891788F42091B50A3091B60A4091B70AFA
:10A7C0005091B80A8091E00A9091E10AA091E20AC2
:10A7D000B091E30A17C0812F0E9490419091A00A86
:10A7E0008917D8F42091B10A3091B20A4091B30A86
:10A7F0005091B40A8091DC0A9091DD0AA091DE0AA2
:10A80000B091DF0A281739074A075B07DCF0821787
:10A810009307A407B5073CF51FC02091B10A3091FA
:10A82000B20A4091B30A5091B40A8091DC0A909127
:10A83000DD0AA091DE0AB091DF0A82179307A40710
:10A84000B5072CF481E080939E0A82E009C02817A6
:10A8500039074A075B073CF482E080939E0A81E057
:10A860008093C90A04C010929E0A1092C90A80916E
:10A870009E0A90E08C159D05C9F00023B9F0FF20D9
:10A88000A9F00E944D53C130D10529F48091C90A25
:10A89000813061F402C0CD2B49F48091780A88237D
:10A8A00029F489E06FEF41E00E94CE39DF91CF912A
:10A8B0001F910F91FF90DF90CF9008950F931F93FA
:10A8C00080E090E060E070E043E050E02CE130E0B8
:10A8D00000E010E00E9478408BE190E060E070E0E2
:10A8E00043E050E02CE130E00E9478400EE113E5B7
:10A8F00082E090E064E170E0A80121E00E94DC5178
:10A900008BE190E064E170E0A80121E00E94DC515D
:10A9100009E113E582E090E06EE070E0A80121E03B
:10A920000E94DC5182E090E062E170E0409105011C
:10A9300021E00E943B508BE190E06EE070E0A801C6
:10A9400021E00E94DC518BE190E062E170E04091F7
:10A95000050121E00E943B500E944D530E948C5102
:10A960000E9469501F910F9108950F931F93CF93E9
:10A97000DF93EC0180E090E060E070E043E050E0C5
:10A980002CE130E000E010E00E9478408BE190E0A4
:10A9900060E070E043E050E02CE130E00E9478405D
:10A9A000CB30D10550F082E090E062E070E04FE4FF
:10A9B00053E521E00E94DC512A9782E090E069E0B3
:10A9C00070E049E453E521E00E94DC5182E090E030
:10A9D00060E170E04C2F21E00E943B508BE190E061
:10A9E00062E070E04DE353E521E00E94DC518BE131
:10A9F00090E066E170E046E553E521E00E94DC511D
:10AA00008BE190E064E170E04091050121E00E945B
:10AA10003B50DF91CF911F910F910895A0E0B0E0DE
:10AA2000E4E1F5E50C945670982E0E94E33680E040
:10AA300090E00E94AB4E88E090E060E170E045E27B
:10AA400053E520E00E94DC5188E090E062E170E094
:10AA50004CE253E520E00E94DC5188E090E063E1A5
:10AA600070E043E353E520E00E94DC5118E0C12E82
:10AA7000D12CC0E0D0E081E090E00E946140892DBF
:10AA80000E949A348C01B82EA12E892D0E949A34EE
:10AA90007601E826F926E022F122E4FE06C020979E
:10AAA00021F02197CE010E94AB4EE5FE08C0209711
:10AAB00031F481E090E00E94AB4EC1E0D0E08B2DFC
:10AAC0009A2D9C016901F0FED6CFCD2B11F081E0CB
:10AAD00007C08091FC0A882311F40E94EF3680E0C1
:10AAE000CDB7DEB7EBE00C947270A3E9B0E0EBE712
:10AAF000F5E50C944F704DE3C42ED12CCC0EDD1E29
:10AB000084E2F60111928A95E9F77E010894E11C2E
:10AB1000F11C8EE1F70111928A95E9F70E94E33664
:10AB20000E946C3483E090E062E070E048E150E025
:10AB300028E130E00EE710E00E9478408FE090E0DE
:10AB40006AE070E044E050E024E030E00EE810E01D
:10AB50000E9478400E94DD7063E070E00E94FF6F09
:10AB600001960E94AE4933E0A32EB12C22E0822E42
:10AB7000912CC257DF4F19821882CE58D040C3574C
:10AB8000DF4F1882CD58D0409FEF292E312C00E0A6
:10AB900011E012C0CB57DF4F08811981C558D04052
:10ABA000C257DF4F19830883CE58D040C557DF4FB7
:10ABB00008811981CB58D04081E090E00E9461402B
:10ABC00080E00E949A34C057DF4F99838883C05930
:10ABD000D04080E00E949A3480279127C057DF4FF1
:10ABE00028813981C059D04082239323C757DF4F32
:10ABF00099838883C958D04087FF56C135E0A31692
:10AC0000B10408F051C1A5014F5F5F4FFA01EE0F8B
:10AC1000FF1FE40FF51FEE0FFF1F61E070E06C0FE8
:10AC20007D1FE60FF71FE80DF91D84AD18168CF493
:10AC3000C401880F991F9401B3E0220F331FBA9506
:10AC4000E1F7820F931F480F591F4215530509F072
:10AC50002BC1C257DF4F88819981CE58D0400297CF
:10AC6000D8F0C1016AE070E00E94EB6F9B01EFEF4A
:10AC7000FFEFEC0FFD1FC257DF4F08811981CE583F
:10AC8000D040E00FF11F80816AE00E94D26F90E017
:10AC90002817390709F408C1C501880F991F880FC3
:10ACA000991F7401EE0CFF1CB7016F5F7F4F660F99
:10ACB000771F039644E050E024E030E00EE710E018
:10ACC0000E947840840163E0000F111F6A95E1F74C
:10ACD0000E0D1F1D4981642E7724C8018A0D9B1D0E
:10ACE0008615970559F4C1016AE070E00E94EB6F88
:10ACF000A816B90618F00894A108B108C801019671
:10AD00008A0D9B1D8215930549F524E0A216B10416
:10AD100010F5C1016AE070E00E94EB6F9B01C10178
:10AD20006AE070E00E94EB6F0196FC01EE0FFF1FDE
:10AD3000E80FF91FEE0FFF1F61E070E06C0F7D1F41
:10AD4000E60FF71FE20FF31F84AD181624F00894E6
:10AD5000A11CB11C03C00894A108B108C257DF4F61
:10AD600088819981CE58D040019771F595E0A91658
:10AD7000B10450F5C1016AE070E00E94EB6F6B0115
:10AD8000C1016AE070E00E94EB6F0196FC01EE0FDA
:10AD9000FF1FE80FF91FEE0FFF1F21E030E02C0F1F
:10ADA0003D1FE20FF31FEC0DFD1D84AD882369F0FC
:10ADB000C8018A0D9B1D91012150304082179307D5
:10ADC00019F40894A108B10864010894A11CB11CED
:10ADD000C257DF4F68817981CE58D040623071050B
:10ADE00008F44CC07601EE0CFF1CC60163E0880F2E
:10ADF000991F6A95E1F7E80EF91EEA0CFB1CE614B0
:10AE0000F70411F40C941E64842F6AE00E94D26F40
:10AE1000682F70E0E6EFFFEF6E9FC0016F9F900D0F
:10AE20007E9F900D1124840F911D880F991F880F0C
:10AE3000991F660F771F660F771F6E5F7F4F039610
:10AE400044E050E024E030E00FE710E00E9478405A
:10AE50000C941E64C501880F991F880F991FB601B5
:10AE6000660F771F660F771F6E5F7F4F039644E074
:10AE700050E024E030E005E910E013C0C501880F80
:10AE8000991F880F991FB601660F771F660F771FEE
:10AE90006E5F7F4F039644E050E024E030E00EE820
:10AEA00010E00E94784001C06401C757DF4FF8816D
:10AEB000C958D040F6FF53C1A114B10409F44FC1E1
:10AEC000A50141505040FA01EE0FFF1FE40FF51F9E
:10AED000EE0FFF1F01E010E00C0F1D1FE00FF11F30
:10AEE000EC0DFD1D84AD18168CF4C601880F991F5A
:10AEF000960163E0220F331F6A95E1F7820F931FDB
:10AF0000480F591F4215530509F029C1C257DF4F99
:10AF100028813981CE58D04022303105D8F0C10186
:10AF20006AE070E00E94EB6F9B01EFEFFFEFEC0F28
:10AF3000FD1FC257DF4F48815981CE58D040E40FE2
:10AF4000F51F80816AE00E94D26F90E028173907D0
:10AF500009F405C1C501880F991F880F991F760153
:10AF6000EE0CFF1CB7016F5F7F4F660F771F0396D4
:10AF700044E050E024E030E00EE710E00E9478402A
:10AF80008601B3E0000F111FBA95E1F70E0D1F1DEA
:10AF90004981642E7724C8018A0D9B1D861597056B
:10AFA00059F4C1016AE070E00E94EB6F8A159B05BD
:10AFB00018F00894A11CB11CC80101978A0D9B1DB3
:10AFC0008215930541F552E0A516B10408F1C101BF
:10AFD0006AE070E00E94EB6F9B01C1016AE070E0E3
:10AFE0000E94EB6FFC01EE0FFF1FE80FF91FEE0F41
:10AFF000FF1F61E070E06C0F7D1FE60FF71FE20F8F
:10B00000F31F86A9181624F00894A108B10803C0FC
:10B010000894A11CB11CC257DF4F88819981CE587A
:10B02000D040019761F5A114B10449F1C1016AE072
:10B0300070E00E94EB6F4B01C1016AE070E00E947A
:10B04000EB6FFC01EE0FFF1FE80FF91FEE0FFF1F64
:10B0500021E030E02C0F3D1FE20FF31FE80DF91D3A
:10B0600086A9882369F0C8018A0D9B1D91012F5F75
:10B070003F4F8217930719F40894A11CB11C460195
:10B080000894A108B108C257DF4F68817981CE5872
:10B09000D0406230710508F44CC07401EE0CFF1C06
:10B0A000C40123E0880F991F2A95E1F7E80EF91EE5
:10B0B000EA0CFB1CE614F70411F40C942764842FAB
:10B0C0006AE00E94D26F682F70E0E6EFFFEF6E9F9C
:10B0D000C0016F9F900D7E9F900D1124840F911DD4
:10B0E000880F991F880F991F660F771F660F771FAC
:10B0F0006E5F7F4F039644E050E024E030E00FE7BE
:10B1000010E00E9478400C942764C501880F991FB5
:10B11000880F991FB401660F771F660F771F6E5F48
:10B120007F4F039644E050E024E030E005E910E072
:10B1300013C0C501880F991F880F991FB401660FAE
:10B14000771F660F771F6E5F7F4F039644E050E0D6
:10B1500024E030E00EE810E00E94784001C0460193
:10B16000C757DF4FF881C958D040F5FF6FC105E0E0
:10B170008016910408F06AC1F501EE0FFF1FEA0D79
:10B18000FB1DEE0FFF1F21E030E02C0F3D1FE20FF3
:10B19000F31FE80DF91D85AD18169CF4C5010A963C
:10B1A0009401220F331FA40103E0440F551F0A9599
:10B1B000E1F7240F351F820F931F8215930509F0C5
:10B1C00045C1C257DF4F48815981CE58D0404230E7
:10B1D000510510F1EFEFFFEFEC0FFD1FE40FF51F2E
:10B1E0004081C1016AE070E00E94EB6F9C01842FF6
:10B1F0006AE00E94D26F90E0BC01E6EFFFEF6E9F25
:10B20000C0016F9F900D7E9F900D1124840F911DA2
:10B210002817390709F41AC1C501880F991F880F2B
:10B22000991F7401EE0CFF1CB7016F5F7F4F660F13
:10B23000771F039644E050E024E030E00EE710E092
:10B240000E9478401981612E7724C401F3E0880FB1
:10B25000991FFA95E1F7E80EF91EEA0CFB1CE614BB
:10B26000F70459F4C1016AE070E00E94EB6F8616A2
:10B27000970618F0089481089108C5010A96940170
:10B28000220F331FA40173E0440F551F7A95E1F795
:10B29000240F351F820F931F8215930541F5F4E0AB
:10B2A0008F16910408F5C1016AE070E00E94EB6F0F
:10B2B0009B01C1016AE070E00E94EB6FFC01EE0FA0
:10B2C000FF1FE80FF91FEE0FFF1F41E050E04C0F8A
:10B2D0005D1FE40FF51FE20FF31F85AD181624F074
:10B2E0000894811C911C03C0089481089108C257DE
:10B2F000DF4F68817981CE58D04061307105B9F552
:10B3000075E08716910498F5C1016AE070E00E942B
:10B31000EB6F6C01C1016AE070E00E94EB6FF60117
:10B32000EE0FFF1FEC0DFD1DEE0FFF1F81E090E003
:10B330008C0F9D1FE80FF91FE60FF71F85AD8823BF
:10B34000B9F0C401880F991F940103E0220F331F45
:10B350000A95E1F7820F931F8A0D9B1D91012A50D8
:10B3600030408217930719F4089481089108650109
:10B370000894811C911CC257DF4FE881F981CE5897
:10B38000D040329708F44CC07401EE0CFF1CC4018D
:10B39000A3E0880F991FAA95E1F7E80EF91EEC0CBF
:10B3A000FD1CE614F70411F40C943064812F6AE05C
:10B3B0000E94D26F682F70E026EF3FEF629FC001BE
:10B3C000639F900D729F900D1124810F911D880F26
:10B3D000991F880F991F660F771F660F771F6E5F83
:10B3E0007F4F039644E050E024E030E00FE710E0A8
:10B3F0000E9478400C943064C601880F991F880F12
:10B40000991FB401660F771F660F771F6E5F7F4F1E
:10B41000039644E050E024E030E005E910E013C07A
:10B42000C601880F991F880F991FB401660F771FF7
:10B43000660F771F6E5F7F4F039644E050E024E075
:10B4400030E00EE810E00E94784001C06501C75767
:10B45000DF4F3881C958D04034FF5FC18114910457
:10B4600009F45BC1F601EE0FFF1FEC0DFD1DEE0FA1
:10B47000FF1F41E050E04C0F5D1FE40FF51FE80D8A
:10B48000F91D83AD18169CF4C6010A979401220F8A
:10B49000331FA40113E0440F551F1A95E1F7240F41
:10B4A000351F820F931F8215930509F036C1C257CD
:10B4B000DF4F68817981CE58D0406230710510F13C
:10B4C000EFEFFFEFEC0FFD1FE60FF71F4081C1010B
:10B4D0006AE070E00E94EB6F9C01842F6AE00E949A
:10B4E000D26F90E0FC0106EF1FEFE09FC001E19FEB
:10B4F000900DF09F900D1124840F911D281739078E
:10B5000009F40BC1C601880F991F880F991F740198
:10B51000EE0CFF1CB7016F5F7F4F660F771F03961E
:10B5200044E050E024E030E00EE710E00E94784074
:10B530004981642E7724C401E3E0880F991FEA95BE
:10B54000E1F7E80EF91EEC0CFD1CE614F70459F4C3
:10B55000C1016AE070E00E94EB6F6815790518F090
:10B560000894811C911C8401000F111FC40163E029
:10B57000880F991F6A95E1F7080F191F0C0D1D1D03
:10B58000C8010A978215930569F522E08216910495
:10B5900008F1C1016AE070E00E94EB6F9B01C101FC
:10B5A0006AE070E00E94EB6FFC01EE0FFF1FE80FF6
:10B5B000F91FEE0FFF1F61E070E06C0F7D1FE60FBB
:10B5C000F71FE20FF31F83AD181624F008948108CB
:10B5D000910808C0C1010A960817190719F40894C0
:10B5E000811C911CC257DF4F88819981CE58D04071
:10B5F000019719F58114910401F1C1016AE070E02D
:10B600000E94EB6F5C01C1016AE070E00E94EB6F89
:10B61000F501EE0FFF1FEA0DFB1DEE0FFF1F01E00E
:10B6200010E00C0F1D1FE00FF11FE60FF71F83AD99
:10B63000882321F00894811C911C560108948108EC
:10B640009108C257DF4F28813981CE58D04022302F
:10B65000310508F44CC07401EE0CFF1CC40123E05A
:10B66000880F991F2A95E1F7E80EF91EEA0CFB1CDA
:10B67000E614F70411F40C943964842F6AE00E94F4
:10B68000D26F682F70E0E6EFFFEF6E9FC0016F9FF3
:10B69000900D7E9F900D1124840F911D880F991F8E
:10B6A000880F991F660F771F660F771F6E5F7F4F9A
:10B6B000039644E050E024E030E00FE710E00E9401
:10B6C00078400C943964C501880F991F880F991F21
:10B6D000B401660F771F660F771F6E5F7F4F03966B
:10B6E00044E050E024E030E005E910E013C0C5017B
:10B6F000880F991F880F991FB401660F771F660F77
:10B70000771F6E5F7F4F039644E050E024E030E007
:10B710000EE810E00E94784001C05601C401880F75
:10B72000991F340153E0660C771C5A95E1F7680EB7
:10B73000791E13012A0C3B1C2501440C551C440C9A
:10B74000551C7501EE0CFF1CBC016F5F7F4FC2578B
:10B75000DF4F08811981CE58D040012B39F5660F93
:10B76000771FC201039644E050E024E030E00FE789
:10B7700010E00E947840EA0CFB1CEE0CFF1C21E05C
:10B7800030E02C0F3D1FE20EF31EE80CF91C8FEF8A
:10B79000F70184AFF5E0AF16B10420F40894A11CC2
:10B7A000B11C25C30894A108B10821C38B01000F67
:10B7B000111FC957DF4F19830883C758D040C201F2
:10B7C0000396B80144E050E024E030E00CE910E0DA
:10B7D0000E94784097012A0D3B1D220F331FE1E0A4
:10B7E000F0E0EC0FFD1FE20FF31FE80DF91D11E073
:10B7F00014AFC257DF4FC880D980CE58D0400894CC
:10B80000C108D108E1E0F0E0EC0FFD1FEC0DFD1DDB
:10B81000E0818E2F6AE00E94D26F90E08816990630
:10B8200009F081C0F0E026EF3FEF829EC001839EC9
:10B83000900D929E900D11248E0F9F1F8A159B05CF
:10B84000D0F57301EE1AFF0A0894E108F108EA0C3A
:10B85000FB1CC5018E199F098C01000F111F080FD9
:10B86000191F000F111F080D191D4DE350E04C0F5B
:10B870005D1F040F151F880F991F880F991F73E014
:10B88000772E780E14C026E0F8012083872DC95743
:10B89000DF4F6881C758D04042E252E00E949F408B
:10B8A0000894E108F1080A5F1F4F34E0730EE114B9
:10B8B000F10449F79AC07C010894E108F108EA18FC
:10B8C000FB08C7018A0D9B1D8C01000F111F080F7B
:10B8D000191F000F111F080D191D4DE350E04C0FEB
:10B8E0005D1F040F151F880F991F880F991F33E0E4
:10B8F000732E780E14C026E0F8012083872DC957D7
:10B90000DF4F6881C758D04042E252E00E949F401A
:10B910000894E108F108065010403CEF730EE11462
:10B92000F10449F762C08815990578F57C01E09427
:10B93000F094E80CF91CC4018E199F098901080FC5
:10B94000191F4DE350E04C0F5D1F040F151F880FAA
:10B95000991F880F991FB2E07B2E780EA3E06A2E04
:10B96000640C0FC0F80125E021938F01862D672D0F
:10B9700040E152E00E949F400894E108F10834E061
:10B98000730EE114F10471F730C07C010894E108F2
:10B99000F108E818F908C701880D991D8901080FF9
:10B9A000191F4DE350E04C0F5D1F040F151F880F4A
:10B9B000991F880F991FE2E07E2E780E73E0672EA4
:10B9C000640C10C025E0F8012083862D672D40E12E
:10B9D00052E00E949F400894E108F1080150104095
:10B9E0003CEF730EE114F10469F7C257DF4F488151
:10B9F0005981CE58D0404230510508F43DC1E1E0B4
:10BA0000F0E0EC0FFD1FEC0DFD1D2081822F6AE0A0
:10BA10000E94D26F382FA82FB0E066EF7FEFA69F6D
:10BA2000A001A79F500DB69F500D1124420F511D2C
:10BA3000EFEFFFEFEC0FFD1FC257DF4F88819981B9
:10BA4000CE58D040E80FF91F2081822F6AE00E9473
:10BA5000D26FE82F90E006EF1FEF809FB001819F2B
:10BA6000700D909F700D1124620F711D46175707BE
:10BA70001CF4A815B90528F04A155B05D0F53E174A
:10BA8000C0F5440F551F440F551FAA0FBB1FAA0F27
:10BA9000BB1F1296842F8D5F6A2F48EC51E00E94E5
:10BAA0009F40E1E0F0E0EC0FFD1FEC0DFD1D40813B
:10BAB000842F6AE00E94D26F90E066EF7FEF869F4E
:10BAC0009001879F300D969F300D1124240F311D5A
:10BAD000F901EE0FFF1FE20FF31FEE0FFF1F01E052
:10BAE00010E00C0F1D1FE00FF11FE80FF91F11E010
:10BAF00044C0641775072CF4832F90E088159905CE
:10BB000028F0A416B506D8F53E17C8F5440F551F02
:10BB1000440F551FAA0FBB1FAA0FBB1F1296842FDD
:10BB20008D5F6A2F4AED51E00E949F40E1E0F0E016
:10BB3000EC0FFD1FEC0DFD1D4081842F6AE00E947B
:10BB4000D26F90E066EF7FEF869F9001879F300D68
:10BB5000969F300D1124240F311DF901EE0FFF1FA8
:10BB6000E20FF31FEE0FFF1F01E010E00C0F1D1F8F
:10BB7000E00FF11FE80FF91F12E014AF7DC0461768
:10BB800057072CF4832F90E08816990628F04A1561
:10BB90005B05D0F5E317C0F5440F551F440F551F43
:10BBA000AA0FBB1FAA0FBB1F1296842F8D5F6A2F8F
:10BBB0004CEE51E00E949F40E1E0F0E0EC0FFD1FF1
:10BBC000EC0DFD1D4081842F6AE00E94D26F90E051
:10BBD00066EF7FEF869F9001879F300D969F300D17
:10BBE0001124240F311DF901EE0FFF1FE20FF31F87
:10BBF000EE0FFF1F01E010E00C0F1D1FE00FF11F03
:10BC0000E80FF91F13E0B9CF440F551F440F551F1C
:10BC1000AA0FBB1FAA0FBB1F1296842F8D5F6A2F1E
:10BC20004EEF51E00E949F40E1E0F0E0EC0FFD1F7D
:10BC3000EC0DFD1D4081842F6AE00E94D26F90E0E0
:10BC400066EF7FEF869F9001879F300D969F300DA6
:10BC50001124240F311DF901EE0FFF1FE20FF31F16
:10BC6000EE0FFF1F01E010E00C0F1D1FE00FF11F92
:10BC7000E80FF91F84E084AFC1016AE070E00E9420
:10BC8000EB6F8B0121E030E02C0F3D1FC20ED31E65
:10BC9000F60180816AE00E94D26F90E008171907D0
:10BCA000E1F5FAE02F163104E0F0C1016AE070E03E
:10BCB0000E94EB6FFC01EE0FFF1FE80FF91FEE0F64
:10BCC000FF1FE20FF31FE00FF11F83AD181624F0E2
:10BCD00008948108910860C022E32216310408F01C
:10BCE00055C0C1016AE070E00E94EB6F9C01220F19
:10BCF000331F280F391F220F331F41E050E04C0F34
:10BD00005D1F240F351F020F131FF80185AD181694
:10BD1000ECF10894811C911C3FC0C1016AE070E005
:10BD20000E94EB6F9C0185309105D0F40196FC01D7
:10BD3000EE0FFF1FE80FF91FEE0FFF1F41E050E06D
:10BD40004C0F5D1FE40FF51FE00FF11F84AD1816B7
:10BD500024F00894A11CB11C1FC021153105B1F0BD
:10BD6000F901EE0FFF1FE20FF31FEE0FFF1F61E05F
:10BD700070E06C0F7D1FE60FF71FE00FF11F86A923
:10BD8000181624F00894A108B10806C071E0C35742
:10BD9000DF4F7883CD58D040C257DF4F88819981DB
:10BDA000CE58D040029718F1B401660F771F940166
:10BDB00043E0220F331F4A95E1F7260F371F2A0D64
:10BDC0003B1D898190E02817390789F4C501880F48
:10BDD000991F880F991F6F5F7F4F660F771F03961C
:10BDE00044E050E024E030E005E910E013C0C50174
:10BDF000880F991F880F991FB401660F771F660F70
:10BE0000771F6E5F7F4F039644E050E024E030E000
:10BE10000EE810E00E947840E1E0F0E0EC0FFD1F3A
:10BE2000C257DF4F08811981CE58D040E00FF11F73
:10BE300020820F5F1F4FCB57DF4F19830883C558F0
:10BE4000D040C357DF4F1881CD58D040112349F45B
:10BE50008091780A882329F483E06FEF41E00E9403
:10BE6000CE39C757DF4F2881C958D04023FD0DC0B8
:10BE7000C057DF4F48815981C059D040C557DF4F67
:10BE800059834883CB58D04090C080E090E00E9416
:10BE90000E55882309F026C5CE01CD960E94314962
:10BEA000CB57DF4F68817981C558D040672B09F4A3
:10BEB0005FC02981822F6AE00E94D26F682F70E0F4
:10BEC000E6EFFFEF6E9FC0016F9F900D7E9F900D7C
:10BED0001124820F911D880F991F880F991F660FDB
:10BEE000771F660F771F6E5F7F4F039644E050E029
:10BEF00024E030E00FE710E00E947840CB57DF4F9E
:10BF000008811981C558D0400130110589F1E1E05F
:10BF1000F0E0EC0FFD1FC257DF4F28813981CE586A
:10BF2000D040E20FF31F2081822F6AE00E94D26F7F
:10BF3000682F70E046EF5FEF649FC001659F900D32
:10BF4000749F900D1124820F911D880F991F880FE7
:10BF5000991F660F771F660F771F6E5F7F4F0396DF
:10BF600044E050E024E030E00CE910E00E9478402A
:10BF7000C501880F991F880F991FB401660F771F9D
:10BF8000660F771F6E5F7F4F039644E050E024E01A
:10BF900030E00EE810E00E94784060E071E0C557A4
:10BFA000DF4F79836883CB58D040E1E0F0E0EC0FBD
:10BFB000FD1FC257DF4F88819981CE58D040E80FCE
:10BFC000F91F90818981981709F06DC1CB57DF4F18
:10BFD000E881F981C558D040329708F464C10E94C5
:10BFE0006C3487E090E062E070E04EE953E520E0D9
:10BFF0000E94DC5188E090E062E170E042E953E5A4
:10C0000020E00E94DC518091F60A9091F70A0C978B
:10C0100061F588E090E064E070E04FE653E520E0F1
:10C020000E94DC5188E090E063E170E04DE753E569
:10C0300020E00E94DC5188E090E064E170E04DE790
:10C0400053E520E00E94DC518EE190E063E170E076
:10C0500041E020E00E943B508EE190E064E170E01E
:10C0600042E020E00E943B5009C088E090E063E19C
:10C0700070E049E953E520E00E94DC5180E090E067
:10C080000E94AB4E81E090E00E94614080E00E94FF
:10C090009A348C01782E612E80E00E949A34C55724
:10C0A000DF4F28813981CB58D040282739272023DA
:10C0B0003123C757DF4F39832883C958D040C9017E
:10C0C0008071907025FF10C08091F60A9091F70A58
:10C0D0008C30910511F00C9750F481E090E00E94B3
:10C0E000AB4E01E010E005C0892B09F4F1C300E07C
:10C0F00010E08091F60A9091F70A0C9709F059C068
:10C1000001301105A1F48BE090E0BE01615E7F4F2C
:10C110000E941C43CE014F96BE016F597F4F0E9473
:10C120009C41CE018F599F4F0E94314902C00E940D
:10C130006C3487E090E062E070E04EE953E520E087
:10C140000E94DC5188E090E062E170E042E953E552
:10C1500020E00E94DC5188E090E064E070E04FE66F
:10C1600053E520E00E94DC5188E090E063E170E05C
:10C170004DE753E520E00E94DC5188E090E064E167
:10C1800070E04DE753E520E00E94DC518EE190E045
:10C1900063E170E041E020E00E943B508EE190E0DE
:10C1A00064E170E042E020E00E943B50C8010E9440
:10C1B000AB4E0115110509F48BC34091F60A50915D
:10C1C000F70A4C30510540F40130110561F47A0151
:10C1D0000894E11CF11C1FC00130110521F43BE063
:10C1E000E32EF12C78C32CE0E22EF12C74C3CE01A7
:10C1F000CD960E943149872D962D9C01C557DF4F62
:10C2000039832883CB58D04031E0C357DF4F388380
:10C21000CD58D04048C0C257DF4F88819981CE5851
:10C22000D040B701AE014F5F5F4F0E942A4F0E947E
:10C230006C3482E090E06FE070E04BE553E520E085
:10C240000E94DC514E2D4A508AE190E06FE070E090
:10C2500020E00E943B508CE390E00E94614080E02F
:10C260000E949A3482FF3EC30E946C3402E010E0C8
:10C270004BE0E416F10421F4F801E851F64F03C055
:10C28000F801EA50F64F87E090E0B801408120E0E5
:10C290000E943B500F5F1F4F0031110549F780E0AE
:10C2A0000E949A34FCCFC757DF4F5881C958D040FD
:10C2B00051FD09C0C357DF4F6881CD58D040662378
:10C2C00011F40C94CA55CB57DF4F88819981C5581A
:10C2D000D040892B11F40C94CA55AA0CBB1CAA0C93
:10C2E000BB1C880C991C880C991CE2E0F0E08E0EB7
:10C2F0009F1EC5010396B40144E050E024E030E005
:10C300000EE710E00E947840C1016AE070E00E94F0
:10C31000EB6F7C015C01C1016AE070E00E94EB6F91
:10C320006B014B01F701EE0FFF1FEE0DFF1DEE0F2E
:10C33000FF1F01E010E00C0F1D1FE00FF11FE60FC3
:10C34000F71F14AE2701440C551C440C551C23E068
:10C3500030E0420E531E12013B01660C771C660C46
:10C36000771C42E050E0640E751ECE56DF4F6882A7
:10C37000C259D040CD56DF4F7882C359D040C20158
:10C38000B30144E050E024E030E00EE710E00E940A
:10C390007840CB57DF4F68817981C558D0406330F2
:10C3A000710560F1EFEFFFEFEC0FFD1FE60FF71FD8
:10C3B0002081822F6AE00E94D26F682F70E0E6EF42
:10C3C000FFEF6E9FC0016F9F900D7E9F900D112417
:10C3D000820F911D880F991F880F991F660F771F75
:10C3E000660F771F6E5F7F4F039644E050E024E0B6
:10C3F00030E00CE910E00E9478400DC0CB57DF4FD1
:10C4000008811981C558D0400130110521F46FEF22
:10C41000262E312C90C1CB57DF4F88809980C5588C
:10C42000D0402EEF3FEF820E931EE1E0F0E0EC0FE4
:10C43000FD1FE80DF91DE0818E2F6AE00E94D26F8A
:10C4400090E0C816D90609F099C0F0E046EF5FEF1A
:10C45000C49EC001C59E900DD49E900D11248E0FD8
:10C460009F1F8E159F0508F04AC0C601880F991FAF
:10C47000960143E0220F331F4A95E1F7820F931F85
:10C48000BF01681B790BCB0101967C01EE0CFF1CF0
:10C49000E80EF91EEE0CFF1CEC0CFD1CEDE3F0E0C9
:10C4A000EC0FFD1FEE0EFF1E6C01CC0CDD1CCC0C46
:10C4B000DD1C03E010E0C00ED11E1DC0F70110828C
:10C4C000C601CE56DF4F6881C259D040CD56DF4FEE
:10C4D0007881C359D04044E050E024E030E00EE7DA
:10C4E00010E00E94784006E010E0E00EF11E24E02B
:10C4F00030E0C20ED31EC414D50401F7C3C10197A6
:10C500008E199F098E0D9F1D7C01EE0CFF1CE80EFD
:10C51000F91EEE0CFF1CEC0CFD1C4DE350E04C0F23
:10C520005D1FE40EF51E6C01CC0CDD1CCC0CDD1C7B
:10C5300063E070E0C60ED71E1DC0F7011082C60171
:10C54000CE56DF4F6881C259D040CD56DF4F78813B
:10C55000C359D04044E050E024E030E00EE710E062
:10C560000E9478400AEF1FEFE00EF11E2CEF3FEF24
:10C57000C20ED31EC414D50401F784C19701220F43
:10C58000331F8C159D05B0F55C01A094B094AC0CE4
:10C59000BD1CC6018A199B09E20EF31EEE0CFF1C9E
:10C5A000E80EF91E4DE350E04C0F5D1FE40EF51E42
:10C5B0006C01CC0CDD1CCC0CDD1C62E070E0C60E06
:10C5C000D71E14C0F70111927F01C101B60144E0EA
:10C5D00050E024E030E00EE710E00E94784008943C
:10C5E000A108B10804E010E0C00ED11EA114B104EE
:10C5F00049F748C101978C199D098C0D9D1DE20ECC
:10C60000F31EEE0CFF1CE80EF91E2DE330E02C0F9C
:10C610003D1FE20EF31E6C01CC0CDD1CCC0CDD1CAE
:10C6200042E050E0C40ED51E13C0F7011082C101D4
:10C63000B60144E050E024E030E00EE710E00E9454
:10C6400078400894E108F1080CEF1FEFC00ED11EEE
:10C65000C614D70451F716C1C1016AE070E00E9408
:10C66000EB6F8B01EEEFFFEFEC0FFD1FCB57DF4FB2
:10C6700028813981C558D040E20FF31F80816AE0DC
:10C680000E94D26F90E00817190729F53AE02316A7
:10C690003104E0F0C1016AE070E00E94EB6F9C01A0
:10C6A000220F331F280F391F220F331F41E050E0A4
:10C6B0004C0F5D1F240F351F020F131FF80183ADB0
:10C6C000181624F008948108910835C04701089491
:10C6D000811C911C30C0C1016AE070E00E94EB6FC8
:10C6E0008530910528F50196FC01EE0FFF1FE80F3C
:10C6F000F91FEE0FFF1F21E030E02C0F3D1FE20F6E
:10C70000F31FE00FF11F84AD181694F00DC0CB5746
:10C71000DF4F48815981C558D0404230510559F406
:10C7200055E0A516B10420F40894A11CB11C03C067
:10C730000894A108B1082981822F6AE00E94D26F73
:10C74000682F70E0E6EFFFEF6E9FC0016F9F900DC6
:10C750007E9F900D1124820F911D880F991F880FC5
:10C76000991F660F771F660F771F6E5F7F4F0396C7
:10C7700044E050E024E030E00FE710E00E94784011
:10C78000CB57DF4F08811981C558D04001301105C2
:10C7900019F1B401660F771F940153E0220F331F84
:10C7A0005A95E1F7260F371F2A0D3B1D898190E02E
:10C7B0002817390789F4C501880F991F880F991F19
:10C7C0006F5F7F4F660F771F039644E050E024E0D1
:10C7D00030E005E910E013C0C501880F991F880FEC
:10C7E000991FB401660F771F660F771F6E5F7F4F2B
:10C7F000039644E050E024E030E00EE810E00E94B0
:10C800007840E1E0F0E0EC0FFD1FC257DF4F2881D8
:10C810003981CE58D040E20FF31F10828091780A00
:10C82000882329F484E06FEF41E00E94CE39C3579A
:10C83000DF4F1882CD58D0400C94D655898190E0B6
:10C84000E816F90611F00C943E570C942A5789818A
:10C8500090E0E816F90611F00C9499580C9485585C
:10C86000898190E0E816F90611F00C94105A0C94A6
:10C87000FC59898190E0E816F90611F00C94775B79
:10C880000C94635B41E050E04C0F5D1F840E951EDD
:10C89000F4018081282E33246AE00E94D26FE82EB2
:10C8A000FF2406EF1FEFE09E5001E19EB00CF09ECA
:10C8B000B00C1124A20CB31C4701CB57DF4F2881C9
:10C8C0003981C558D0402330310508F0C5CE1FCF7F
:10C8D000EE24EA94FE2C3FEFE3163FEFF30609F453
:10C8E00086CC99CCCD56DF4FE2E10C946B70ADE174
:10C8F000B0E0EDE7F4E60C944F709F8B8E8B798F50
:10C90000688F5B8F4A8F0E94964728E635E0EAE9F8
:10C91000FAE0AF01455F5F4F60E0FF24F39408EC5D
:10C9200010E074E6D90113968C911397880F880F45
:10C9300012969C91890F861B8083DA011D921D92AD
:10C940001D921C9213971786108A118A128A138AD5
:10C95000148A158A168A148210868091F30A8F250C
:10C9600090E0DC01A09FC001A19F900DB09F900DB1
:10C9700011248183809105018283F382D9018C91F6
:10C98000879FC0011124AA2797FDA095BA2F878BF6
:10C99000908FA18FB28FD90111968C91879FC00182
:10C9A0001124AA2797FDA095BA2F838F948FA58F66
:10C9B000B68FDA015E961C925E975D961C921E926F
:10C9C0005C972C5F3F4F6B5FBB96455D5F4F6A3056
:10C9D00009F0A8CFEA8DFB8DEF2B49F48DE090E0B4
:10C9E0006CE070E048E353E520E00E94DC518CE30A
:10C9F00090E00E94614082E090E066E070E041E0FB
:10CA000050E023E030E00FE710E00E9478408BE137
:10CA100090E066E070E041E050E023E030E00E940A
:10CA200078408091780A882329F487E06FEF41E00D
:10CA30000E94CE398CE390E00E94614082E090E059
:10CA400069E070E041E050E023E030E00FE710E003
:10CA50000E9478408BE190E069E070E041E050E0B6
:10CA600023E030E00E9478408091780A882329F4FE
:10CA700087E06FEF41E00E94CE398CE390E00E94A6
:10CA8000614082E090E06CE070E041E050E023E043
:10CA900030E005E910E00E9478408BE190E06CE026
:10CAA00070E041E050E023E030E00E947840809167
:10CAB000780A882329F486E06FEF41E00E94CE399E
:10CAC0001A8219821C821B821E821D8218861F8276
:10CAD0001A8619861C861B861C8A1A8A198A2224A1
:10CAE00033248A8D9B8D01979D8F8C8F81E090E000
:10CAF0000E9461409AE52916310481F40E945E5437
:10CB00008091FC0A882371F40E94DD7063E070E07C
:10CB10000E94FF6F01960E94AE4904C0ABE52A1641
:10CB2000310418F40894211C311CF8E6AF2EF5E00E
:10CB3000BF2E0FE91AE0EE24FF24CC24DD248E2D35
:10CB40000E949A349C01E1E0F0E0EC0FFD1FEC0D37
:10CB5000FD1D91838083A5E0B0E0AC0FBD1FAC0D3F
:10CB6000BD1D20953095E9E0F0E0EC0FFD1FEC0DC8
:10CB7000FD1D80819181282339232D933C93F5015C
:10CB8000808190E0449760E270E00E94FF6FE62FA2
:10CB9000D80111966C93D50111968C9190E00C9769
:10CBA00060E270E00E94FF6FD80112966C931297BA
:10CBB00052962D913D914D915C915597205D374056
:10CBC00040405040F0E0A0E8BCE0EA9FC001EB9F8D
:10CBD000900DFA9F900D1124AA2797FDA095BA2FCA
:10CBE000281B390B4A0B5B0BF801228F338F448FC4
:10CBF000558F26893789408D518D205B34404040C8
:10CC0000504070E0A0E8BCE06A9FC0016B9F900DAF
:10CC10007A9F900D1124AA2797FDA095BA2F281B63
:10CC2000390B4A0B5B0B268F378F40A351A38C8D9A
:10CC30009D8D8E159F0588F48091F90A9091FA0ACE
:10CC40008130910521F49BE49093CA0A09C00297B0
:10CC500021F4AAE6A093CA0A03C044E6F80140837F
:10CC6000C7016E897F890E948C500894E11CF11CD9
:10CC700082E090E0C80ED91EA4E0B0E0AA0EBB1E70
:10CC8000055D1F4FB2E0EB16F10409F058CF80911B
:10CC9000C70A8823A9F480919C0A882389F08C898B
:10CCA00063E00E94DE6F992329F48091F40A8F5F7C
:10CCB0008093F40AEC89EF5FEC8BEB300CF01C8A6C
:10CCC00080919C0A8823C1F48091C70A8823A1F02F
:10CCD00081E08093F50A8C8963E00E94DE6F9923DE
:10CCE00029F48091F10A8F5F8093F10AFC89FF5F3C
:10CCF000FC8BFB300CF01C8A8A8D9B8D019779F0A0
:10CD000080919C0A8823E9F48091C70A8823C9F49A
:10CD10009BEF2916310490F0A1E0AB8B13C08091FA
:10CD20009C0A882371F48091C70A882351F4BBEFD1
:10CD30002B16310418F0E1E0EB8B80C00894211C25
:10CD4000311C1B8AFBE52F16310451F460919E0AB9
:10CD50008E899F8970E04A8D5B8D0E948C536EC0D6
:10CD60004CE52416310409F069C00E944D538091AE
:10CD7000FC0A882309F062C00E94E3368A8D9B8DED
:10CD8000019709F065C080919C0A882371F5809114
:10CD9000F50A813051F580E59DE40E94A936909115
:10CDA000F20A9F5F9093F20A8091FB0A8F5F809353
:10CDB000FB0A8091F10A8253823318F49F5F9093AB
:10CDC000F20A8091F10A8456843628F48091F20A9E
:10CDD0008E5F8093F20A8091F10A883C78F180910D
:10CDE000F20A8D5F8093F20A29C08AE99DE40E94CD
:10CDF000A9369091790A9F5F9093790A8091F00A01
:10CE00008F5F8093F00A8091F40A8253823318F482
:10CE10009F5F9093790A8091F40A8456843628F4AF
:10CE20008091790A8E5F8093790A8091F40A883C18
:10CE300028F08091790A8D5F8093790AE5E0AE2E23
:10CE4000B12CAC0EBD1E0DEA1AE0EE24FF24DEC0AC
:10CE500080E59DE40E94A936F1CFDE2C8E2D0E9444
:10CE60009A3493FF05C0C701B1010E94BB5180C035
:10CE7000F801248935892A303105C1F480819181F6
:10CE8000A281B3814396A11DB11D8797A105B1056C
:10CE900068F0C70161E070E00E94154581E090E014
:10CEA000D80155969C938E93549767C0265F3F4F49
:10CEB000C9F4F80180819181A281B3814396A11DBB
:10CEC000B11D8797A105B10568F0C70160E070E06A
:10CED0000E941545EFEFFFEFD8015596FC93EE93B6
:10CEE00054974BC08D2D0E949A3487FF1DC0D801E6
:10CEF00054968D919C915597892B89F48D919D9194
:10CF00000D90BC91A02D4396A11DB11D8797A10541
:10CF1000B10528F0C70161E070E00E941545F801F5
:10CF200084899589019621C08D2D0E949A3486FFAF
:10CF30001FC0D80154968D919C915597892B89F4E7
:10CF40008D919D910D90BC91A02D4396A11DB11D79
:10CF50008797A105B10528F0C70160E070E00E9445
:10CF60001545F801848995890197958B848B05C0B7
:10CF7000D80155961C921E9254978D2D0E949A347A
:10CF800090FF04C0C7010E94CC460CC08D2D0E94AA
:10CF90009A3481FF04C0C7010E94F04603C0C70154
:10CFA0000E942447F50180819181089731F5C701DE
:10CFB0000E940E558B8B882351F08091790A8F5FE8
:10CFC0008093790A8091F00A8F5F8093F00A888DB0
:10CFD000998D0E9431498E899F890E94DD470E9468
:10CFE0005E5480E090E062E070E00E94154581E0D0
:10CFF00090E062E070E00E9415450894E11CF11C8D
:10D0000082E090E0A80EB91E055D1F4FAA8DBB8D72
:10D01000EA16FB0608F421CFFE013796F88BEF875E
:10D020007FEC872E7AE0972E66EFC62E6FEFD62E16
:10D03000C80CD91C51E0452E512C75C1D4019096D5
:10D040001C92F6018085853009F41086D601189669
:10D050008C91882339F40E94DD70F60181878085E8
:10D060008F5F8087D60119966C90A62CBB24B3E005
:10D07000AB22BB24E091F90AF091FA0AFE87ED8712
:10D08000329729F4F2E0AF16B10448F40CC08D8554
:10D090009E85892B41F493E0A916B10421F4AEEFEB
:10D0A000BFEFAA0EBB1EF6019381AE89BF898C919A
:10D0B000981718F0E1E0F0E003C0E92FF0E03196B6
:10D0C0008E899F89E80FF91F90819D8B892F0E947F
:10D0D0009041D60116969C9116979817A0F57C90D2
:10D0E000B2E07B1609F464C0F401618D728D838D0A
:10D0F000948D24E630E040E050E00E9434707901E5
:10D100008A01C501880F991F0796A0E0B0E08E152F
:10D110009F05A007B1070CF04BC08CE090E08A1986
:10D120009B09880F991FA0E0B0E0E816F9060A07EE
:10D130001B07F4F560E070E0FEEF7F0E43E047155B
:10D1400008F0A7C0A4C0891798F5D6017C90B6E076
:10D150007B1671F1F401618D728D838D948D24E6BF
:10D1600030E040E050E00E94347079018A01C5014E
:10D17000880F991F0796A0E0B0E08E159F05A007C5
:10D18000B107B4F48CE090E08A199B09880F991FCD
:10D19000A0E0B0E0E816F9060A071B074CF460E0CF
:10D1A00070E0FDEF7F0E42E0471508F472C06FC0DB
:10D1B0008D890E949541D60117969C9117978917E2
:10D1C000A0F57C90772009F46EC05F966D917D91FB
:10D1D0008D919C91929724E630E040E050E00E94CF
:10D1E000347079018A01C501880F991F0796A0E064
:10D1F000B0E08E159F05A007B1070CF054C08CE07D
:10D2000090E08A199B09880F991FA0E0B0E0E8160A
:10D21000F9060A071B070CF046C060E070E0BBEFA0
:10D220007B0EE2E0E715A8F132C09817E0F5D601D1
:10D230007C90B4E07B16B9F1F601678D70A181A1F5
:10D2400092A124E630E040E050E00E943470790181
:10D250008A01C501880F991F0796A0E0B0E08E15DE
:10D260009F05A007B107FCF48CE090E08A199B09A8
:10D27000880F991FA0E0B0E0E816F9060A071B071F
:10D2800094F460E070E07A94F2E0F71510F061E059
:10D2900070E0C2010E941545E1E0D401EC93F1E099
:10D2A0009096FC9323C0D4018C91882349F0669416
:10D2B0006694F601618680858F5F80871C9216C018
:10D2C0008D859E85029791F4F60183899489A589BD
:10D2D000B68984369105A105B10544F0FBE52F160A
:10D2E000310420F0C201B1010E94BB51C2010E9471
:10D2F000CC468A8D9B8D892B41F4AF85B8898D9161
:10D300009C91089711F4B1E0BB8B08944108510837
:10D31000EF85F8893297F88BEF8785ED9FEF880EC0
:10D32000991EC80ED91EAA8DBB8D4A165B0630F019
:10D33000BFEF4B16BFEF5B0609F080CE80E090E0B8
:10D340000E94834581E090E00E9483458091F80A25
:10D35000882319F000E010E010C08A8D9B8D0E9498
:10D36000C349282F30E0890163E0000F111F6A953F
:10D37000E1F7220F331F020F131F80E090E0688D4A
:10D38000798D4A8D5B8D98010E94294B080F111DE4
:10D3900081E090E0688D798D4A8D5B8D98010E94C7
:10D3A000294B080F111D0115110571F0E989FA8942
:10D3B000EF2B89F488E06FEF41E00E94CE398AE0DC
:10D3C00090E09A8B898B07C0A989BA89109719F0C8
:10D3D0001197BA8BA98B80E090E00E94A04681E073
:10D3E00090E00E94A0466091B10A7091B20A8091CB
:10D3F000B30A9091B40A24E630E040E050E00E9485
:10D400003470209368056091B50A7091B60A8091D6
:10D41000B70A9091B80A24E630E040E050E00E945C
:10D420003470209369056091DC0A7091DD0A809167
:10D43000DE0A9091DF0A24E630E040E050E00E94EE
:10D44000347020936C056091E00A7091E10A80913C
:10D45000E20A9091E30A24E630E040E050E00E94C6
:10D46000347020936D0529813A818B819C81BB8921
:10D47000BB2329F43A8729879C878B8737CB6D9606
:10D48000E2E10C946B70A2E4B0E0E9E4FAE60C94FB
:10D490004F702C01C0900601D09007018E010F5FE4
:10D4A0001F4F8EE1F80111928A95E9F7C601B80184
:10D4B0000E941C439FE1E92EF12CEC0EFD1EC801D9
:10D4C000B7010E949C41C7010E943149C8010E94D6
:10D4D000DD47C6010E94B554A12C81E0B82EB9E009
:10D4E0002B2E332433944801370181E090E00E94D1
:10D4F000614080E00E949A347C018501009510957E
:10D500000823192302FF04C0C4010E94D54420C08F
:10D5100007FF0EC00894C11CD11C8091F60A90919F
:10D52000F70A8C159D0580F4A1E0CA2ED12C0CC001
:10D5300006FF19C00894C108D108C114D10421F410
:10D54000C090F60AD090F70AC601B4010E941C43AD
:10D55000C401B3010E949C41C3010E943149C4012E
:10D560000E94DD4717C004FF0AC0809105018F5F4C
:10D57000809305018A3070F0309205010BC005FFE1
:10D580000CC080910501815080930501882311F41E
:10D5900020920501C6010E94B554570108301105BB
:10D5A00009F0A3CF0E94E336D0920701C092060192
:10D5B000CE010196BE01615E7F4FA2010E94776499
:10D5C000CE5BDF4FE2E10C946B70A2E4B0E0EBEED7
:10D5D000FAE60C945B70162F7E010894E11CF11C96
:10D5E0002EE1F70111922A95E9F7B7010E941C4339
:10D5F000112319F0C7010E94D5442FE1E22EF12C2E
:10D60000EC0EFD1E8E010F5F1F4FC801B7010E9477
:10D610009C41C7010E943149C8010E94DD47C801F1
:10D62000B70140E050E00E947764CE5BDF4FE6E058
:10D630000C947770A2E4B0E0E0E2FBE60C94597041
:10D6400000910101112707FD10957E010894E11C4E
:10D65000F11C8EE1F70111928A95E9F7C801B70133
:10D660000E941C433FE1C32ED12CCC0EDD1EC7010E
:10D67000B6010E949C41C6010E943149C7010E9427
:10D68000DD47C8010E94B5548091030180930501D4
:10D690000E94E33680910101992787FD9095909330
:10D6A00007018093060182E060E00E941F40C701ED
:10D6B000B60141E050E00E94776482E060E00E94A1
:10D6C0001F400E946C3480EF8093680580936C0546
:10D6D00082E090E064E070E04BEB53E520E00E94D4
:10D6E000DC5185E190E064E070E04091060120E0CB
:10D6F0000E943B509091F20A8091790A981714F198
:10D700008BE090E06AE070E04EEA53E520E00E9492
:10D71000DC5183E190E06AE070E04091F20A21E0A0
:10D720000E943B508BE090E06CE070E043EB53E5EF
:10D7300020E00E94DC5183E190E06CE070E04091D9
:10D74000790A21C08BE090E06AE070E043EB53E59A
:10D7500020E00E94DC5183E190E06AE070E04091BB
:10D76000790A21E00E943B508BE090E06CE070E091
:10D770004EEA53E520E00E94DC5183E190E06CE04A
:10D7800070E04091F20A21E00E943B508AE090E074
:10D7900062E170E044E152E520E00E94DC5180E06B
:10D7A0000E949A340897D9F71092F40A1092F10A5D
:10D7B0001092F50A82E061E00E942E402091010162
:10D7C0002F5F20930101332727FD309580910401BD
:10D7D00090E02817390711F40E9435520E941A6B05
:10D7E000CE5BDF4FE8E00C947570A0E0B0E0EBEFAB
:10D7F000FBE60C9457700E94235288E090E062E1AF
:10D8000070E04CE552E520E00E94DC5188E090E0B9
:10D8100063E170E048E652E520E00E94DC5188E0D8
:10D8200090E064E170E045E752E520E00E94DC51C1
:10D8300088E090E065E170E04DE752E520E00E946D
:10D84000DC5180E090E00E945F4EC0E0D0E0CC244C
:10D85000DD2481E090E00E94614080E00E949A34E3
:10D860008C01B82EA12E80E00E949A347601E82621
:10D87000F926E022F122E5FE07C0C330D10520F4ED
:10D880002196CE010E945F4EE4FE06C0209721F053
:10D890002197CE010E945F4E8B2D9A2D9C0169012C
:10D8A000F0FED7CFCE01CDB7DEB7EAE00C947370AF
:10D8B0000F931F9386E190E062E170E048E050E052
:10D8C00026E030E000E010E00E9478408091F90A04
:10D8D0009091FA0A009739F486E190E062E170E0F5
:10D8E0004BE952E50FC0019739F486E190E062E11F
:10D8F00070E046E952E506C086E190E062E170E042
:10D9000042EA52E520E00E94DC5180910201882326
:10D9100039F486E190E063E170E040E552E506C04D
:10D9200086E190E063E170E042E552E520E00E948C
:10D93000DC51409104014A3098F486E190E064E1C2
:10D9400070E044E050E024E030E000E010E00E94AD
:10D95000784086E190E064E170E04091040104C009
:10D9600087E190E064E170E020E00E943B5086E1B6
:10D9700090E065E170E04091030120E00E943B509F
:10D980008091F80A882339F486E190E066E170E03E
:10D990004AEB52E506C086E190E066E170E04DEBAF
:10D9A00052E520E00E94DC518091F30A882339F48B
:10D9B00086E190E067E170E04AEB52E506C086E15F
:10D9C00090E067E170E04DEB52E520E00E94DC5111
:10D9D0008091FC0A882339F486E190E068E170E0E8
:10D9E0004AEB52E506C086E190E068E170E04DEB5D
:10D9F00052E520E00E94DC518091780A882339F4B6
:10DA000086E190E069E170E04AEB52E506C086E10C
:10DA100090E069E170E04DEB52E520E00E94DC51BE
:10DA20001F910F9108950E94235284E090E068E1D5
:10DA300070E040E252E520E00E94DC5183E090E09B
:10DA400069E170E047E352E520E00E94DC518091FB
:10DA5000FC0A882321F48FE79AE30E94A93680EF1D
:10DA60008093680580936C050895CF92DF92EF92C2
:10DA7000FF920F931F930E94136DCC24DD24760137
:10DA800047C081E090E00E946140C701B6012CE3ED
:10DA900030E040E050E00E94127061157105810590
:10DAA000910569F489E090E062E170E04BE050E0BC
:10DAB00021E030E000E010E00E94784016C0C7018D
:10DAC000B6012EE130E040E050E00E941270611596
:10DAD00071058105910549F489E090E062E170E00B
:10DAE00044E152E520E00E94DC5188E5C81682E05E
:10DAF000D80680E0E80680E0F80629F40E94E336C4
:10DB000021E030E00DC00894C11CD11CE11CF11CC7
:10DB100080E00E949A34089709F0B3CF20E030E00B
:10DB2000C9011F910F91FF90EF90DF90CF90089562
:10DB30000F931F930E94E33689E392E090937B0A50
:10DB400080937A0AECE7FAE011928AE0EA39F80762
:10DB5000D9F7CF0180970E944E350E94C74E809121
:10DB6000780A882329F485E06FEF41E00E94CE39DE
:10DB700088E090E061E170E047EE52E520E00E942D
:10DB8000DC5188E790E00E94614088E090E061E12C
:10DB900070E04EE050E021E030E000E010E00E9454
:10DBA00078401F910F9108958F929F92BF92CF92CC
:10DBB000DF92EF92FF920F931F93CF93DF930E9418
:10DBC000235288E090E062E170E04AE852E520E00C
:10DBD0000E94DC5188E090E063E170E044E552E5AA
:10DBE00020E00E94DC5188E090E064E170E04AEDC2
:10DBF00052E520E00E94DC5188E090E065E170E0B1
:10DC00004DEC52E520E00E94DC5188E090E066E1B6
:10DC100070E047EA52E520E00E94DC5188E090E0A5
:10DC200067E170E043EB52E520E00E94DC5188E0C0
:10DC300090E068E170E041EC52E520E00E94DC51A8
:10DC400088E090E069E170E048EC52E520E00E9455
:10DC5000DC5180E090E00E94AB4E80E090E00E94BA
:10DC6000586C00E010E0E12C51E0F52EBB24B39499
:10DC700042E0842E912C81E090E00E94614080E09F
:10DC80000E949A346C0180E00E949A34E701C82710
:10DC9000D927CC21DD21C5FF08C00730110528F4A4
:10DCA0000F5F1F4FC8010E94AB4EC4FF08C0011593
:10DCB000110541F001501040C8010E94AB4E011502
:10DCC000110581F5C7FFD5C08091F90A9091FA0A34
:10DCD000009729F49092FA0A8092F90A06C00197F7
:10DCE00021F41092FA0A1092F90A80E090E00E9462
:10DCF000586CBFC08091F90A9091FA0A009739F4E4
:10DD000081E090E09093FA0A8093F90A06C00297A6
:10DD100021F41092FA0A1092F90A80E090E00E9431
:10DD2000586C15C00130110591F49E01207C09F456
:10DD300067C080910201882319F4B092020102C0E9
:10DD40001092020180E090E00E94586C59C00230AD
:10DD5000110571F4C7FF90C0809104018A3018F456
:10DD60008F5F8093040180E090E00E94586C84C033
:10DD70000330110569F023C080910401882319F054
:10DD800081508093040180E090E00E94586C48C06C
:10DD9000C7FF75C080910301893018F48F5F8093AD
:10DDA000030180E090E00E94586C69C080910301FB
:10DDB000823008F444C081508093030140C0043095
:10DDC000110571F49E01207C09F43DC08091F80A90
:10DDD000882319F4B092F80A32C01092F80A2FC0C2
:10DDE0000530110569F49E01207C69F18091F30AE8
:10DDF000882319F4B092F30A22C01092F30A1FC0CC
:10DE00000630110569F49E01207CE9F08091FC0A3E
:10DE1000882319F4B092FC0A12C01092FC0A0FC0B9
:10DE20000730110581F49E01207C69F08091780A09
:10DE3000882319F4B092780A02C01092780A80E020
:10DE400090E00E94586C80E00E949A3480509D407F
:10DE500019F40E94986D18C088E0E822FF24C601DA
:10DE6000809590958E219F217601892B09F403CF0F
:10DE700009C0C6FD3FCF6BCFC6FD7ECFD1CFC6FD5B
:10DE800095CFE1CF0E944C47DF91CF911F910F9129
:10DE9000FF90EF90DF90CF90BF909F908F9008956C
:10DEA0000F931F930E94C74E83E19AE30E948E3620
:10DEB00080EB0E94173784E392E00E948B3481EA62
:10DEC0000E94883484EF96E30E9467340E94EA52ED
:10DED0008091990A90E00E94E2700E94DD70809328
:10DEE000990A8AE79AE00E944E350E94356D0097A4
:10DEF00019F0019769F723C00E94F56B81309105F5
:10DF0000A9F0823091051CF4892B39F0E1CF8230E1
:10DF1000910579F00397E1F60FC0809102019927EE
:10DF200087FD909501960E94436AD2CF0E941A6B9A
:10DF3000CFCF0E94D46DCCCF0E947555C9CF0E941F
:10DF4000DD706091F60A7091F70A0E94EB6F8C0108
:10DF50000F5F1F4F0E94DD70BC0161707070C801BF
:10DF60000E94E56AB5CF629FD001739FF001829F46
:10DF7000E00DF11D649FE00DF11D929FF00D839F58
:10DF8000F00D749FF00D659FF00D9927729FB00DF5
:10DF9000E11DF91F639FB00DE11DF91FBD01CF0108
:10DFA00011240895991B79E004C0991F961708F071
:10DFB000961B881F7A95C9F78095089587FB082ED0
:10DFC000062687FD819567FD6195ECDF0EF491953E
:10DFD00007FC81950895AA1BBB1B51E107C0AA1F2E
:10DFE000BB1FA617B70710F0A61BB70B881F991FFA
:10DFF0005A95A9F780959095BC01CD01089597FB9E
:10E00000092E07260AD077FD04D0E5DF06D00020D0
:10E010001AF4709561957F4F0895F6F79095819564
:10E020009F4F0895A1E21A2EAA1BBB1BFD010DC034
:10E03000AA1FBB1FEE1FFF1FA217B307E407F507B8
:10E0400020F0A21BB30BE40BF50B661F771F881F94
:10E05000991F1A9469F760957095809590959B012A
:10E06000AC01BD01CF01089597FB092E05260ED006
:10E0700057FD04D0D7DF0AD0001C38F450954095E6
:10E08000309521953F4F4F4F5F4F0895F6F790958C
:10E090008095709561957F4F8F4F9F4F08952F9278
:10E0A0003F924F925F926F927F928F929F92AF9228
:10E0B000BF92CF92DF92EF92FF920F931F93CF9375
:10E0C000DF93CDB7DEB7CA1BDB0B0FB6F894DEBF0C
:10E0D0000FBECDBF09942A88398848885F846E8432
:10E0E0007D848C849B84AA84B984C884DF80EE807C
:10E0F000FD800C811B81AA81B981CE0FD11D0FB685
:10E10000F894DEBF0FBECDBFED010895EE0FFF1FE7
:10E110000590F491E02D0994A0E0B0E0E2E9F0E789
:10E120000C945770EC01A880B980CA80DB80A114E0
:10E13000B104C104D10441F484E2A82E89EDB82EC3
:10E140008BE5C82E87E0D82EC601B5012DE133EF4F
:10E1500041E050E00E94347027EA31E440E050E0B2
:10E160000E94B36F7B018C01C601B5012DE133EF35
:10E1700041E050E00E943470CA01B9012CEE34EF46
:10E180004FEF5FEF0E94B36F6E0D7F1D801F911FD9
:10E1900097FF04C061507040804090486883798345
:10E1A0008A839B839B013F77C901CDB7DEB7EAE045
:10E1B0000C9473700E948C70089580E192E00E942C
:10E1C0008C700895A0E0B0E080931002909311024B
:10E1D000A0931202B0931302089511F40EF44DC0EF
:10E1E0003EC05DD0D0F39923D9F3CEF39F57550BA2
:10E1F00087FF46D00024A0E640EA9001805856955B
:10E20000979528F4805C660F771F881F20F02617EB
:10E210003707480730F4621B730B840B2029312920
:10E220004A2BA69517940794202531254A2758F79D
:10E23000660F771F881F20F026173707480730F42E
:10E24000620B730B840B200D311D411DA09581F7CE
:10E25000B901842F9158880F9695879508959F3F0F
:10E2600031F0915020F4879577956795B795880F91
:10E27000911D9695879597F908959FEF80EC0895E5
:10E2800091505040660F771F881FD2F7089557FDB1
:10E290009058440F551F59F05F3F71F04795880F14
:10E2A00097FB991F61F09F3F79F0879508951216AB
:10E2B00013061406551FF2CF4695F1DF08C0161657
:10E2C00017061806991FF1CF869571056105089408
:06E2D0000895F894FFCF51
:10E2D600010101090A03010000000000000000001E
:10E2E60000010202030303030404040404040404F7
:10E2F60005050505050505050505050505050505C8
:10E3060006060606060606060606060606060606A7
:10E316000606060606060606060606060606060697
:10E326000707070707070707070707070707070777
:10E336000707070707070707070707070707070767
:10E346000707070707070707070707070707070757
:10E356000707070707070707070707070707070747
:10E366000808080808080808080808080808080827
:10E376000808080808080808080808080808080817
:10E386000808080808080808080808080808080807
:10E3960008080808080808080808080808080808F7
:10E3A60008080808080808080808080808080808E7
:10E3B60008080808080808080808080808080808D7
:10E3C60008080808080808080808080808080808C7
:10E3D60008080808080808080808080808080808B7
:04E3E6000100000032
:00000001FF
